:100000000000032011420100B5380100A9370100AA
:10001000A9370100A9370100A9370100A93701005C
:10002000A9370100A9370100A9370100B53801003F
:10003000B5380100A937010061480100E54601001B
:10004000B5380100B5380100B5380100B5380100F8
:10005000B5380100B5380100B5380100B5380100E8
:10006000B5380100B5380100B5380100B5380100D8
:10007000B5380100B5380100B5380100B5380100C8
:10008000B5380100B5380100B5380100B5380100B8
:10009000B5380100B5380100B5380100B5380100A8
:1000A000D91D0100CD1D0100B5380100B538010092
:1000B000B5380100B5380100B538010079360100C6
:1000C000B5380100F5EA0000B53801002DEA00005E
:1000D000B538010065E90000B5380100B538010008
:1000E000B5380100B5380100B5380100B538010058
:1000F000B5380100B5380100B5380100B538010048
:10010000B5380100B5380100B5380100B538010037
:10011000B5380100F9EB0000B5380100B538010031
:10012000B5380100B5380100B5380100B538010017
:10013000B5380100B5380100B5380100B538010007
:100140009D480100B53801009DE80000B538010068
:10015000B5380100B5380100B5380100B5380100E7
:10016000B5380100B5380100C11D0100B5380100E6
:10017000B5380100B5380100B5380100B5380100C7
:10018000B5380100D1FB0000B5380100B5380100D9
:10019000B5380100B5380100C1E70000B5380100ED
:1001A000B5380100B5380100B5380100B538010097
:1001B000B5380100B5380100B5380100B538010087
:1001C000B5380100B5380100B5380100B538010077
:1001D000FFFFFFFFFFFFFFFFFFFFFFFFFFFFFFFF2F
:10040000FFFFFFFFFFFFFFFFFFFFFFFFDEF9FFFF23
:1004100010B5054C237833B9044B13B10448AFF33E
:1004200000800123237010BD00B0FF1F00000000FA
:1004300044070F00084B10B51BB108490848AFF33B
:1004400000800848036803B910BD074B002BFBD0A0
:10045000BDE81040184700BF0000000004B0FF1FB7
:1004600044070F005CA2FF1F000000002DE9F047C9
:100470004DF27446C1F6FF7682B04DF2784733688C
:100480000093C1F6FF77009B3A689B1AB3F5487F4B
:1004900043F6F04500F2B8824BF2EC14C2F20005CC
:1004A000C1F6FF744DF25440C1F6FF7016F074FDB2
:1004B0004DF21440C1F6FF7015F01AF92368984206
:1004C000804600F33884C0F22D83984520D049F24D
:1004D000D0295FFA88F3C1F6FF79184689F8003011
:1004E00017F00EFE4FF66820C0F2010017F0F8FB7F
:1004F00099F800000AF058FA43F6F420C2F200001E
:100500000AF0CCF80AF0B8F833680193019B3B601D
:100510004DF25447C1F6FF77C4F80080BB7B002B37
:1005200040F03E814DF60036C1F6FF764DF2644054
:10053000C1F6FF7016F030FD4DF23440C1F6FF7089
:1005400015F0D6F895F8AD3055F823305A7B03EB0B
:10055000820380465B68B34200F0A0824EF23442D0
:10056000C1F6FF72934200F0A6824EF22062C1F6FD
:10057000FF72934200F0ED834EF60C02C1F6FF725B
:10058000934200F0E5824EF6F812C1F6FF729342F4
:1005900000F07D844EF6E432C1F6FF72934200F023
:1005A000BB844EF6D052C1F6FF72934200F06F85C5
:1005B0004EF6BC72C1F6FF72934200F005844FF212
:1005C000A812C1F6FF72934200F0D6854FF2943222
:1005D000C1F6FF72934200F01D8640F23452C2F21F
:1005E0000002934200F0668640F22072C2F20002DE
:1005F000934200F0AD8640F60C12C2F20002934224
:1006000000F0F48640F6F822C2F20002934200F0B5
:100610003B8740F6E442C2F20002934200F06C874E
:1006200040F6D062C2F20002934200F0718741F2BC
:10063000BC02C2F20002934200F0A28741F2A8225B
:10064000C2F20002934200F0E28741F29442C2F209
:100650000002934201F0BB8041F28062C2F20002CC
:10066000934201F05D8041F66C02C2F200029342B7
:1006700001F0E98041F65822C2F20002934201F0F3
:100680002B8141F64442C2F20002934201F05581AF
:1006900042F21C02C2F20002934201F0318141F6A3
:1006A0003062C2F20002934201F0CC8242F2082290
:1006B000C2F20002934201F0A88242F2F432C2F286
:1006C0000002934201F0958242F2E052C2F200022F
:1006D000934201F0828242F2CC72C2F20002934253
:1006E00001F06F8242F6B812C2F20002934201F0AA
:1006F0005C8242F6A432C2F20002934200F0CE8144
:1007000043F68C42C2F20002934201F03D8243F272
:100710000412C2F20002934201F0F78143F2F02288
:10072000C2F20002934201F0A78143F2DC42C2F21E
:100730000002934201F07D8143F2C862C2F20002DE
:100740009342636801F01C814BF2EC199845C1F6A5
:10075000FF7901F30F8114DA4FF6B010C0F20100F7
:1007600017F0BEFA40460AF051FB5FFA88F099F89C
:1007700004100BF003F995F8AD3055F8230008F09C
:1007800093FCBA7FC4F804804DF25443C1F6FF7362
:100790001AB11F7F002F00F0128202B0BDE8F0876F
:1007A0003B7B002B7FF4BEAE4FF62C70C0F20100F5
:1007B00017F096FA95F8AD3055F823305A7B03EBD5
:1007C00082034DF600365B68C1F6FF76B34200F057
:1007D000F6834EF24822C1F6FF72934200F04C8439
:1007E0004EF23442C1F6FF72934200F073844EF22F
:1007F0002062C1F6FF72934200F077844EF60C023D
:10080000C1F6FF72934200F07B844EF6F812C1F6F7
:10081000FF72934200F07F844EF6E432C1F6FF721D
:10082000934200F0E1844EF6D052C1F6FF7293423B
:1008300000F0E5844EF6BC72C1F6FF72934200F000
:1008400009834FF2A812C1F6FF72934200F01C8593
:100850004FF29432C1F6FF72934200F0208540F2CD
:100860004832C2F20002934200F05C8540F23452FA
:10087000C2F20002934200F0608540F22072C2F2A0
:100880000002934200F09C8540F60C12C2F2000276
:10089000934200F0A08540F6F822C2F20002934293
:1008A00000F0DC8540F6E442C2F20002934200F020
:1008B000E08540F6D062C2F20002934200F0F0857B
:1008C00041F2BC02C2F20002934200F0F48541F210
:1008D000A822C2F20002934200F0038641F2944241
:1008E000C2F20002934200F0F18541F28062C2F24E
:1008F0000002934200F0238641F66C02C2F200022D
:10090000934200F0118641F65822C2F2000293424F
:1009100000F02B8641F64442C2F20002934200F0FE
:10092000198641F63062C2F20002934200F06486FA
:1009300042F21C02C2F20002934200F0A48642F28C
:100940000822C2F20002934200F0B38642F2F4326F
:10095000C2F20002934200F0A18642F2E052C2F2DB
:100960000002934200F0D18642F2CC72C2F2000241
:10097000934200F0BF8642F6B812C2F200029342E0
:1009800000F0AD8642F6A432C2F20002934200F0BB
:100990009B8643F68C42C2F20002934201F0AA8089
:1009A00042F61872C2F20002934201F0988043F2BC
:1009B0000412C2F20002934201F0868043F2F02258
:1009C000C2F20002934201F0748043F2DC42C2F2B0
:1009D0000002934200F04E8743F2C862C2F2000266
:1009E000934200F03C8743F6B402C2F20002934205
:1009F0007FF49CAD4FF6DC60C0F2010009F0C6FF49
:100A000006200AF039FF91E5C2F2000543F6A02264
:100A100095F8AD3055F82330597B03EB8103C2F2D2
:100A200000025B68934204D04BF2EC14C1F6FF74F1
:100A300038E54FF6F060C0F2010009F0A7FF4DF273
:100A40003440C1F6FF7014F053FE4BF2C018C1F6EB
:100A5000FF784BF2EC1488F829004DF66810C1F6C7
:100A6000FF7009F01BFE09F0A9FF4DF21442C1F618
:100A7000FF7298F90030C1F6FF7400210520636011
:100A8000906323EAE37382F83C10516372B68342A9
:100A9000A8BF03469B00D36262B603E5636898452E
:100AA0003FF46FAE49F2A423C1F6FF7383F80080D0
:100AB00009F0E2FD65E6636898453FF462AE4FF2E7
:100AC000F4705FFA88F90A21C0F2010016F026FCE2
:100AD00000220A21484617F00DF909F003FE07EE3F
:100AE000909A0023C4F2C62306EE903AB8EE676AE5
:100AF0000023C6EE267A07EE103A4BF22003C1F629
:100B0000FF7377EE877A18684368C3ED007A10F0B8
:100B1000BBFB49F2A823C1F6FF7383F8049009F0E8
:100B2000ABFD2EE64FF65C20C0F2010017F0D8F8BE
:100B3000B8F1000FC0F20981404600220A2117F0E7
:100B4000D9F809F0CFFD236898457FF4C0ACDFE405
:100B5000636898453FF415AE4FF610005FFA88F9C8
:100B60000D21C0F2010016F0D9FB00220A214846EF
:100B700017F0C0F809F0B6FD07EE909A0023C4F212
:100B8000C62306EE903AB8EE676A0023C6EE267AD0
:100B900007EE103A4BF22003C1F6FF7377EE877A27
:100BA00018684368C3ED027A10F06EFB49F2A8237F
:100BB000C1F6FF7383F8069009F05EFDE1E54FF69C
:100BC0000C70C0F2010009F0E1FE95F8AD3055F867
:100BD00023305A7B03EB820343F6F0495B68B34250
:100BE000C2F2000900F0DC8142F6A432C2F2000237
:100BF000934200F0EF8143F68C42C2F2000293422E
:100C000000F07C814EF24822C1F6FF72934200F060
:100C1000C38140F24832C2F20002934200F0D08019
:100C200042F61872C2F20002934200F02B833E4655
:100C3000B8464FF6F810C0F2010017F051F860689E
:100C4000304409F0E3FE4FF61420C0F2010017F023
:100C500047F860680028B6BF2D22002240420A21D2
:100C600017F048F84FF63420C0F2010017F038F8BA
:100C700000220A21384617F03DF809F033FD95F8B7
:100C8000AD3055F823707B7B07EB830343F6F049C7
:100C90005A6892F8511092F850308B42C2F2000913
:100CA00000F0E380636852F8212001334344DBB253
:100CB00001334BF2EC1A52F82330C1F6FF7A002BC5
:100CC00000F0D3809847386811F090F9384608F062
:100CD000EBF999F8AD3059F82340637B04EB8303BB
:100CE0005A6892F8511092F850308B420BD0DAF8D3
:100CF000043052F8212001334344DBB2013352F86F
:100D0000233003B19847206811F070F9204608F0AD
:100D1000CBF995F8AD3055F82330186811F066F925
:100D200095F8AD3055F82340206811F05FF9204662
:100D300008F0BAF931E54FF64C20C0F2010016F088
:100D4000CFFFB8F1000FBFF6F7AEC8F100002D22BB
:100D5000F4E6636898453FF414AD4FF600005FFA7F
:100D600088F90C21C0F2010016F0D8FA00220A21FD
:100D7000484616F0BFFF09F0B5FC07EE909A002335
:100D8000C4F2C62306EE903AB8EE676A0023C6EEB8
:100D9000267A07EE103A4BF22003C1F6FF7377EE86
:100DA000877A18684368C3ED017A10F06DFA49F24A
:100DB000A823C1F6FF7383F8059009F05DFCE0E419
:100DC0000F273E46B84634E7636898453FF4D9ACF0
:100DD0004FF648004FFA88F90921C0F2010016F0D9
:100DE0009DFAB9F1000FB4BF2D2200224FF00A0185
:100DF0004846B8BFC9F1000016F07CFF09F072FC4C
:100E000007EE909A0023C4F24823B8EEE77A07EE83
:100E1000903A0023C4F2C82306EE103A37EE277A40
:100E20000023C7EE067A06EE903A4BF22003C1F695
:100E3000FF7377EEA67A18684368C3ED097A10F05D
:100E400023FA49F2A823C1F6FF7383F80A9009F048
:100E500013FC96E44FF65430C0F2010009F096FD01
:100E60000D200AF0B7FCFFF761BB386811F0BEF83F
:100E7000384608F019F94FF61870C0F2010016F064
:100E80002FFF60680130304409F0C0FD85E46368DD
:100E900098453FF476AC4FF620005FFA88F90B21B5
:100EA000C0F2010016F03AFA00220A21484616F074
:100EB00021FF09F017FC07EE909A0023C4F2C62325
:100EC00006EE903AB8EE676A0023C6EE267A07EE81
:100ED000103A4BF22003C1F6FF7377EE877A186859
:100EE0004368C3ED037A10F0CFF949F2A823C1F6A5
:100EF000FF7383F8079009F0BFFB42E4B8F1010FDC
:100F000000F014814FF6E410C0F2010009F03EFD3C
:100F100004200AF0B1FC40E4636898453FF431AC2A
:100F20004FF62C004FFA88F90B21C0F2010016F0A1
:100F3000F5F9B9F1000FB4BF2D2200224FF00A01DC
:100F40004846B8BFC9F1000016F0D4FE09F0CAFB4C
:100F500007EE909A0023C4F2C62306EE903AB8EE4C
:100F6000E76A0023C6EE267A07EE103A4BF220031A
:100F7000C1F6FF7377EE877A18684368C3ED077A86
:100F800010F082F949F2A823C1F6FF7383F80890A4
:100F900009F072FBFFF7F5BB06273E46B84648E668
:100FA0004FF6BC10C0F2010016F09AFE09F09AFB51
:100FB00006F042FE01200AF05FFCFFF7EEBB4FF6A1
:100FC0007820C0F2010009F0E1FC01200AF054FC95
:100FD000FFF7ACBA4FF6C810C0F2010016F080FE61
:100FE00009F080FB4DF23440C1F6FF7014F080FB35
:100FF0004BF2C016C1F6FF76307143F6E040C2F204
:10100000000009F04BFB99F8AD3059F823E09EF849
:101010000C30D3B13D46384602240EEB85025168B0
:1010200091F850206AB1002351F823201471D07038
:101030009070013391F85020DBB29A42F4D89EF8B8
:101040000C300135EDB29D42E7D34DF21442C1F6AA
:10105000FF7296F928300021012023EAE3739063A0
:1010600082F83C10516372B68342A8BF03469B00CE
:10107000D36262B6FFF791BB4FF69020C0F2010039
:1010800009F084FC02200AF0F7FBFFF74FBA63680F
:1010900098453FF476AB4FF638004FFA88F9C0F226
:1010A000010016F01DFEB9F1000F4846BABF2D220F
:1010B000C9F1000000220A2116F01CFE09F012FB03
:1010C00049F2A823C1F6FF7383F8099009F0D4FA16
:1010D000FFF757BB4FF6A820C0F2010009F056FCFD
:1010E00007200AF077FBFFF721BA4FF6C420C0F2C1
:1010F000010009F04BFC08200AF06CFBFFF716BA60
:101100004FF6E020C0F2010009F040FC09200AF08F
:1011100061FBFFF70BBA4FF6FC20C0F2010009F0AB
:1011200035FC0A200AF056FBFFF700BA49F2A42466
:10113000C1F6FF744FF6D810C0F2010016F0D0FDD2
:101140003A460A21207816F0D5FD09F0CBFA4FF681
:10115000D810C0F2010016F0C3FD207809F024FC7D
:101160004BF2A4124BF21C03C1F6FF72C1F6FF73DF
:10117000217811701F70CBE6636898453FF401AB8E
:101180004FF654005FFA88F90B21C0F2010016F007
:10119000C5F800220A21484616F0ACFD09F0A2FA73
:1011A00007EE909A0023C4F2C62306EE903AB8EEFA
:1011B000676A0023C6EE267A07EE103A4BF2200348
:1011C000C1F6FF7377EE877A18684368C3ED0A7A31
:1011D00010F05AF849F2A823C1F6FF7383F80B9078
:1011E00009F04AFAFFF7CDBA4FF61830C0F2010005
:1011F00009F0CCFB0B200AF0EDFAFFF797B94FF698
:101200003430C0F2010009F0C1FB0C200AF0E2FA10
:10121000FFF78CB9636898453FF4B3AA4FF66000B6
:101220005FFA88F91321C0F2010016F077F8002266
:101230000A21484616F05EFD09F054FA07EE909A2E
:101240000023C4F2C62306EE903AB8EE676A002384
:10125000C6EE267A07EE103A4BF22003C1F6FF7372
:1012600077EE877A18684368C3ED067A10F00CF8B9
:1012700049F2A823C1F6FF7383F80C9009F0FCF93A
:10128000FFF77FBA2327D2E44FF66C30C0F201009B
:1012900009F07CFB0E200AF09DFAFFF747B94FF6E4
:1012A0008830C0F2010009F071FB0F200AF092FAB9
:1012B000FFF73CB9636898453FF463AA4FF67400A2
:1012C0005FFA88F91621C0F2010016F027F8002213
:1012D0000A21484616F00EFD09F004FA07EE909A2E
:1012E0000023C4F2C62306EE903AB8EE676A0023E4
:1012F000C6EE267A07EE103A4BF22003C1F6FF73D2
:1013000077EE877A18684368C3ED057A0FF0BCFF63
:1013100049F2A823C1F6FF7383F80D9009F0ACF9E8
:10132000FFF72FBA4FF6AC30C0F2010009F02EFBE8
:1013300003200AF0A1FAFFF7F9B84FF6C030C0F267
:10134000010009F023FB10200AF0F2F9FFF7EEB8D4
:10135000636898453FF415AA4FF68C005FFA88F948
:101360001321C0F2010015F0D9FF00220A214846DE
:1013700016F0C0FC09F0B6F907EE909A0023C4F20B
:10138000C62306EE903AB8EE676A0023C6EE267AC8
:1013900007EE103A4BF22003C1F6FF7377EE877A1F
:1013A00018684368C3ED047A0FF06EFF49F2A82372
:1013B000C1F6FF7383F80E9009F05EF9FFF7E1B90B
:1013C0004FF6E430C0F2010009F0E0FA11200AF013
:1013D000AFF9FFF7ABB84FF60440C0F2010009F0D7
:1013E000D5FA12200AF0A4F9FFF7A0B8636898456F
:1013F0003FF4C7A94FF6A0005FFA88F90E21C0F2AA
:10140000010015F08BFF00220A21484616F072FCFD
:1014100009F068F907EE909A0023C4F2C62306EE9D
:10142000903AB8EE676A0023C6EE267A07EE103AC5
:101430004BF22003C1F6FF7377EE877A1868436892
:10144000C3ED0B7A0FF020FF49F2A823C1F6FF731A
:1014500083F80F9009F010F9FFF793B94FF6204089
:10146000C0F2010009F092FA13200AF061F9FFF7C7
:101470005DB84FF63C40C0F2010009F087FA142035
:101480000AF056F9FFF752B8636898453FF479A916
:101490005FFA88F017F092F809F0EEF8FFF771B9EB
:1014A0004FF65C40C0F2010009F070FA15200AF016
:1014B0003FF9FFF73BB84FF67840C0F2010009F062
:1014C00065FA16200AF034F9FFF730B84FF6B44049
:1014D000C0F2010009F05AFA18200AF029F9FFF7C2
:1014E00025B84FF69840C0F2010009F04FFA1720D6
:1014F0000AF01EF9FFF71AB8636898453FF441A94E
:101500005FFA88F017F016F809F0B6F8FFF739B966
:10151000636898453FF435A95FFA88F016F0C6FF76
:1015200009F0AAF8FFF72DB94FF6F040C0F201001C
:1015300009F02CFA1A200AF0FBF8FEF7F7BF4FF675
:10154000D040C0F2010009F021FA19200AF0F0F8A9
:10155000FEF7ECBF4FF63050C0F2010009F016FA6A
:101560001C200AF0E5F8FEF7E1BF4FF61050C0F27C
:10157000010009F00BFA1B200AF0DAF8FEF7D6BFDB
:10158000636898453FF4FDA84FF6B00049F2A829DA
:10159000C1F6FF795FFA88FA1321C0F2010015F055
:1015A000BDFE00220A21504616F0A4FB09F09AF86D
:1015B00099F8153099F8122099F8111099F810003F
:1015C00001EE103A99F8143007EE903AB8EE411A4D
:1015D000F8EE677AF2EE040A81EE201AC7EEA00A4E
:1015E00007EE90AAB8EE670A09F056FB89F813A037
:1015F00009F042F8FFF7C5B84FF65450C0F20100A9
:1016000009F0C4F91D200AF093F8FEF78FBF636854
:1016100098453FF4B6A84FF6C40049F2A829C1F690
:10162000FF795FFA88FA1021C0F2010015F076FE0A
:1016300000220A21504616F05DFB09F053F899F894
:10164000153099F8122099F8111099F8100007EE4A
:1016500090AA01EE103A99F81330F8EE670A00EEFE
:10166000103AB8EE411AF2EE047A81EE271AC0EE73
:10167000A70AB8EE400A09F00FFB89F814A008F099
:10168000FBFFFFF77EB84FF67450C0F2010009F07F
:101690007DF91E200AF04CF8FEF748BF4FF6B8500F
:1016A000C0F2010009F072F920200AF041F8FEF7BB
:1016B0003DBF4FF69850C0F2010009F067F91F20B6
:1016C0000AF036F8FEF732BF4FF62860C0F201008C
:1016D00009F05CF904200AF0CFF8FEF727BF4FF6B7
:1016E0001060C0F2010009F051F923200AF020F83F
:1016F000FEF71CBF4FF6F850C0F2010009F046F9A2
:1017000022200AF015F8FEF711BF4FF6D850C0F2AC
:10171000010009F03BF921200AF00AF8FEF706BFA4
:10172000636898453FF42DA84FF6E80014215FFA4E
:1017300088F9C0F2010015F0F1FD00220A214846A7
:1017400016F0D8FA08F0CEFF07EE909A0023C4F204
:10175000C623F8EE676A07EE103AC6EE877A0023D2
:1017600006EE103A77EE867AF7EE006AF4EEE67A45
:10177000F1EE10FA40F3898044F21873C2F20003CC
:1017800045F2606247F670519952F0EE667A45F67E
:101790002943C4F20F6307EE103A67EE877A4AF6E0
:1017A000B811FDEEE77AC2F2000117EE903A45F269
:1017B000606049F2A82203F5B343C1F6FF72193302
:1017C0000B5282F8169008F057FFFEF7DABF6368F5
:1017D00098453EF4D6AF4FF6D80049F2A829C1F695
:1017E000FF795FFA88FA0F21C0F2010015F096FD2B
:1017F00000220A21504616F07DFA08F073FF99F88E
:10180000143099F8122099F8111099F8100007EE89
:1018100090AA00EE903A99F81330B8EE671A00EEED
:10182000103AF8EE600AF2EE047AC0EEA70A81EEF2
:10183000271AB8EE400A09F02FFA89F815A008F027
:101840001BFFFEF79EBF636898453EF49AAF5FFAB0
:1018500088F016F09FFD08F00FFFFEF792BF4FF6DD
:10186000C460C0F2010009F091F827200AF056F890
:10187000FEF75CBE4FF6A460C0F2010009F086F8E6
:1018800026200AF04BF8FEF751BE45F62943F4EE48
:10189000C67AC4F20F63F1EE10FA05EE903A54BF27
:1018A000B0EE677AB0EE467A27EE257A44F21872E7
:1018B000BDEEC77AC2F2000217EE103A45F260613F
:1018C00003F5B343F4EEE67A1933F1EE10FA53520E
:1018D0000EDDF0EE667A5AE7636898453EF451AF44
:1018E0005FFA88F008F07AFA08F0C6FEFEF749BF02
:1018F000F4EE467AF1EE10FA48BFF0EE467A46E78B
:10190000636898453EF43DAF4FF618101521C0F2BC
:10191000010015F003FD00220A215FFA88F016F09D
:10192000E9F908F0DFFE49F2A823C1F6FF7383F856
:101930001B8008F0A1FEFEF724BF636898453EF4C3
:1019400020AF4FF600101521C0F2010015F0E6FCA3
:1019500000220A215FFA88F016F0CCF908F0C2FEE6
:1019600049F2A823C1F6FF7383F8198008F084FEBA
:10197000FEF707BF4FF6A010C0F20100FEF7F0BE61
:1019800098453EF4FEAE4FF690105FFA88F90D21AF
:10199000C0F2010015F0C2FC00220A21484616F0F0
:1019A000A9F908F09FFE4BF22003C1F6FF7349F23C
:1019B000A8221868C1F6FF7247F2A40E80F81090B2
:1019C0004FF0000CC3F67D7E034682F8249000F5AC
:1019D0001C61C3F8D0C2C3F8D4E2343399424FF04B
:1019E0000002F6D100F6C8414FF0000EC4F2203ECE
:1019F000C1F800E000F6984E00F54B61002300F5B9
:101A0000496CC0F87C3CC0F88C3CCEF8002000F655
:101A1000944300F6AC4ECCF800200A604FF07E51A3
:101A2000CEF8002019600FF02FFC08F025FEFEF71D
:101A3000A8BE636898453EF4A4AE4FF67C105FFAEA
:101A400088F91321C0F2010015F068FC00220A2178
:101A5000484616F04FF908F045FE49F2A82319F15F
:101A60000009C1F6FF7318BF4FF0010983F82390F6
:101A700008F002FEFEF785BE636898453EF481AE2D
:101A80004FF668101121C0F2010015F047FC00224A
:101A90000A215FFA88F016F02DF908F023FE49F2CA
:101AA000A823C1F6FF7383F8228008F0E5FDFEF756
:101AB00068BE4FF68860C0F2010008F067FF25207D
:101AC00009F02CFFFEF732BD4FF67060C0F2010046
:101AD00008F05CFF242009F021FFFEF727BD4FF638
:101AE0005C60C0F2010008F051FF052009F0C4FE5F
:101AF000FEF71CBD4FF64060C0F2010008F046FF43
:101B0000042009F0B9FEFEF711BD636898453EF464
:101B100038AE4FF658105FFA88F90D21C0F2010077
:101B200015F0FCFB00220A21484616F0E3F808F005
:101B3000D9FD07EE909A0023C4F2C623F8EE675A47
:101B400006EE103A85EE867A002349F2A822C1F605
:101B5000FF7282F8219007EE903A4CF6CD43C3F61F
:101B60004C6306EE903A4BF22003C1F6FF7377EE1A
:101B7000277A1B6867EEA67A03F6DC43C3ED007A8A
:101B800008F07AFDFEF7FDBD636898453EF4F9ADB7
:101B90004BF21C0318F10002C1F6FF7318BF0122BB
:101BA0001A7008F069FDFEF7ECBD636898453EF4D5
:101BB000E8AD5FFA88F007F087FE08F05DFDFEF7FC
:101BC000E0BD636898453EF4DCAD5FFA88F007F04D
:101BD00049FF08F051FDFEF7D4BD636898453EF417
:101BE000D0AD5FFA88F008F009F808F045FDFEF77F
:101BF000C8BD636898453EF4C4AD5FFA88F008F04C
:101C000075F808F039FDFEF7BCBD636898453EF4F1
:101C1000B8AD4FF644101121C0F2010015F07EFB63
:101C200000220A215FFA88F016F064F808F05AFDE5
:101C300049F2A823C1F6FF7383F81C8008F01CFD4D
:101C4000FEF79FBD636898453EF49BAD4FF630109C
:101C50001121C0F2010015F061FB00220A215FFA98
:101C600088F016F047F808F03DFD49F2A823C1F6C8
:101C7000FF7383F81A8008F0FFFCFEF782BD00BFF7
:101C80002DE98048B9B002F0CBF942F649044DF293
:101C900074422646C1F6FF7244F230640292324624
:101CA0002746C2F2010244F2905301923A469E4600
:101CB000C2F200024BF2200305921A46C1F6FF72EF
:101CC00044F2D06300921A46C2F2000244F2F46376
:101CD00013921A46C2F2000248F2854312921A4643
:101CE000C0F2000242F63D0314921A46C2F201020B
:101CF00042F63E0310921A46C2F2010248F209432C
:101D000011921A46C0F2000242F2D0331D921A46D6
:101D1000C2F2010242F2104316921A46C2F20102C6
:101D200048F2A55315921A46C0F2000242F25C43F3
:101D30000E921A46C2F2010242F214430C921A4663
:101D4000C2F2010242F2154307921A46C2F20102A0
:101D500042F2184304921A46C2F2010242F2584378
:101D600008921A46C2F2010242F6E9130D921A468F
:101D7000C0F2010242F63C0318921A46C2F2010276
:101D800040F640731E921A46C2F201024FF64473A7
:101D90000B921A46C0F2010249F2A42317921A4686
:101DA000C1F6FF7240F6447319921A46C2F201025C
:101DB00049F2D0231A921A464EF60453CEF200038B
:101DC00040F63C7140F64870099348F2340343F6FC
:101DD000A05B43F6A06A41F679544EF20305C2F2C5
:101DE000000EC2F20101C2F20100C1F6FF72C4F29C
:101DF0000403CDF818E01C911F90C2F2000BC2F250
:101E0000000AC0F201041B920F93C4F20705069B5F
:101E1000D3F8983044F29056C2F20006002B00F03E
:101E20001A86059BD3F8983044F23066C2F2000659
:101E3000002B01F00A8172B64EF21803029ACEF21C
:101E400000031B681168099A126862B6520102D534
:101E5000322B88BF0131C3F52F331C9A03F21F3395
:101E600046F6174012689B08C1F2C160A0FB03034D
:101E7000C2EB93034FF47A7202FB013340F64B320C
:101E8000934240F2568172B64EF21803029ACEF295
:101E900000031B681168099A126862B6570102D5DF
:101EA000322B88BF0131029A1F9812682792C3F51E
:101EB0002F3303F21F3346F61747C1F2C167279E3F
:101EC00000689B084FF47A72A7FB037302FB01F2D0
:101ED00002EB9302301A41F288331C994DF2744799
:101EE00040F6487698420A60C1F6FF77C2F20106D2
:101EF00000F26F86069BD3F89830002B00F0EA8141
:101F000003F10408059BD3F89820002A00F0CD8146
:101F1000043272B64EF218030299CEF200031B6827
:101F20000F680999096862B64E0102D5322B88BF45
:101F3000013700990868C3F52F33066803F21F3391
:101F400046F6174EC1F2C16E9B08AEFB03E3414655
:101F50004FF47A7E36684FEA93080EFB07F7B047D6
:101F600072B64EF21803029A0999CEF200031B686A
:101F70001268096862B6480102D5322B88BF013267
:101F8000C3F52F3303F21F3346F617419B08C1F206
:101F9000C161A1FB0313C8EB9303DF1B4FF47A73FA
:101FA00003FB027340F65532934203D900994A6805
:101FB00001324A60009A11894BF22002C1F6FF7289
:101FC0008B4288BF138172B6139B1A7F44F2D06391
:101FD00002F0FF01C2F200030AB100221A7762B6D2
:101FE00061B372B6139E47F6FF734FF40041B6F922
:101FF0001E20F383B6F92030318462B6002AB8BFC0
:102000005242002BB8BF5B429342B8BF134607EE63
:10201000903A4FF47E43C4F2FF63F8EEE77A06EE9F
:10202000903A87EEA67AF7EE007AB4EEE77AF1EE10
:1020300010FA03DD009AD3680133D36072B6129BA5
:102040001A7F44F2F46302F0FF01C2F200030AB106
:1020500000221A7762B661B372B6129E47F6FF731A
:102060004FF40041B6F91E20F383B6F920303184D5
:1020700062B6002AB8BF5242002BB8BF5B429342FF
:10208000B8BF134607EE903A4FF47E43C4F2FF63A5
:10209000F8EEE77A06EE903A87EEA67AF7EE007A47
:1020A000B4EEE77AF1EE10FA03DD009AD36801335B
:1020B000D360069FD7F8980044F29053C2F2000311
:1020C000B8B193F89C1001311F29CABF0026CEB2C7
:1020D000314697F89D2044F290538A42C2F20003A1
:1020E000F7D00631002243F8210083F89C60C3F842
:1020F0009820059FD7F8980044F23063C2F200039D
:10210000B8B193F89C1001311F29CABF0026CEB286
:10211000314697F89D2044F230638A42C2F20003B0
:10212000F7D00631002243F8210083F89C60C3F801
:1021300098209BF84C7043F6A053102FC2F2000376
:1021400040F23A81009B1A694BF22006C1F6FF76F5
:10215000002A00F0568217885388990802EB810103
:102160000433BB428E6880F0F081538006F00F028A
:10217000A2F1080106294FEA162300F2BF8003F0FE
:102180000F03082A03F10100C6F3033300F04D8268
:10219000092A00F031840A2A40F021840A2B00F039
:1021A0004D87009BD3F880616EB1F76847B13B68FB
:1021B000DB68A342384600D098477F68002FF6D1ED
:1021C000B668002EF1D1BAF82E20BAF8303043F6B6
:1021D000A0619A42C2F200014BD0898D01338B423B
:1021E00080F0E6804FEA830E9EB2DAF824009AF877
:1021F000287050F80E90AAF8306043F6A060C2F242
:10220000000097B9C06880B19A4226BF01F1FF3142
:102210008A1AD243BAF820101344B3EB910F43F655
:10222000A062C2F2000280F00C844FEA192309F088
:102230000F0703F00F08A7F108020A9343F6A06600
:10224000C9F3031308F10101062A0391C2F2000643
:102250008AF838307CD8082FC9F3033300F0DD83C7
:10226000092F00F015840A2F40F0FE830A2B00F09E
:102270006287029B0B9A1B6825931268259B9B1A09
:102280004DF2744140F64072642BC1F6FF71C2F208
:10229000010200F2EE80019B1B78002B7FF4B7ADAA
:1022A00014F03CFFB3E514F039FF12F0F9FC059B84
:1022B000C3F8980050B9019B1B78002BF3D012F0A3
:1022C000EFFC059BC3F898000028F4D0021D20E61F
:1022D00014F024FF12F0E4FC069BC3F8980050B9F8
:1022E000019B1B78002BF3D012F0DAFC069BC3F89D
:1022F00098000028F4D000F1040803E6901E01289D
:10230000D9B240F23081052A00F02781042A00F07A
:102310002287501F022840F233840F2A7FF441AFF6
:10232000F72900F22081009AF029B2F8542002D057
:10233000002A3FF436AFB2F5917FBFF432AF009878
:1023400001461144013281F85830A0F8542028E7A2
:10235000BB1E012B9DF8288040F22481052F00F040
:102360001981042F00F04F847B1F022B40F2A983B8
:102370000F2F7FF47EAFB8F1F70F00F21381B8F1A1
:10238000F00FB6F8601102D000293FF472AFDAF80E
:102390008031002B01F0B684B1F5917F81F0A884E3
:1023A0004B1C9BB25144AAF8603181F83D8060E734
:1023B0000026B646334618E7986C149A03681B69E2
:1023C000934240F00184109B119A1B781078DBB285
:1023D000C0B2834238BF4033181A00283FF4B2AE6F
:1023E000DBF848001D9A03685B6943F6A0569342E8
:1023F000C2F2000640F00586109B119A1B781278F5
:10240000D9B2D2B242F63E0E9142C2F2010E01F0B2
:102410002E85531C3F2B40F23D84169B1878159B4C
:102420001E680023C0B28EF8003026B1CB1A1A2BDA
:1024300001DC00233370C3B203F0FB02F92A3FF43E
:1024400081AEDBF85810002940F040849BF84D2005
:102450008BF84F30110601F150815AB2002AC1F2B7
:10246000A2810023CBF85830CBF854308BF84D3094
:1024700068E60B682493249B1360FDF7F7FF009B2D
:1024800093F884214BF22003C1F6FF73002A40F039
:10249000DA80009B93F885314BF22002C1F6FF727F
:1024A000002B3FF4F8AE029B1A991B68239309682E
:1024B000239B5B1A41F288318B427FF6ECAE0123FD
:1024C000C4F20203002182F885111B781B9ADB07F6
:1024D000167840F12C864FF0A0531B789E4224D0F2
:1024E0000123C4F202031B78DF0741F199834FF007
:1024F000A0531B789E4218D02B78802B01F07D834F
:102500000022C4F20202137813F0700300D013709B
:102510004FF0A05301221E70C4F202021378D807B4
:10252000FCD52B78012B01F0C5834FF6D470222106
:10253000C0F2010014F0F2FE179B02211B88ADF8D7
:10254000A03028A814F0EAFEA5E6104614F016FE06
:1025500009F0DEFA009B186108E6F02940F21083CA
:10256000F72900F00D83F82900F04A8640F23983FC
:10257000FC2900F03E8600F29A84FA2900F07C855E
:10258000FB297FF40EAE009B5B6C002B3FF409AE81
:10259000984706E6B8F1F00F40F29382B8F1F70FD2
:1025A00000F08F82B8F1F80F01F0978340F25B835F
:1025B000B8F1FC0F01F0168300F22685B8F1FA0F8E
:1025C00001F0EF82B8F1FB0F7FF453AEDAF8A021EF
:1025D00043F6A063C2F20003002A00F0268590476C
:1025E000C9F307469DF828309DF80C808AF83A30E8
:1025F0004FEA19678AF839808AF83B608AF83C709C
:1026000037E61E9B1B78002B3FF4CBAD09F080FA18
:102610000246306100283FF4C4AD0788002F7FF4E4
:102620009BAD14F0ABFD3761BBE5082B7FF4B9AD72
:10263000009B5B69002B3FF4B4ADC0B2320EC6F311
:1026400007419847ADE51B68D3F87C3C002B7FF42D
:1026500020AF4FF6487EC0F2010EBEE80F0028AF53
:102660000FC7BEE80F000FC7BEE80F000FC79EE8F8
:102670000F0049F2AC2687E80F00C1F6FF764FF055
:10268000FF3316F8012B82EA030138A801F00F018D
:1026900000EB810151F8401C81EA131181EA121309
:1026A00003F00F0300EB830353F8402C82EA11136D
:1026B00049F2D022C1F6FF7296426FEA0303E0D1DD
:1026C0004FF68C70C0F20100282142F8283C14F02B
:1026D00025FE009B93F88421002A00F0EB824CF643
:1026E000CD40CCF6CC40A0FB0213DB0803EB83010A
:1026F000A2EB410230328DF8C120002B01F0228381
:102700002122A0FB0361C90801EB8106013AA3EB7A
:102710004603D2B238AE1644303306F8403C0B467E
:102720000029EED11046C2F1220128AB184414F062
:10273000F5FD4FF6B8701121C0F2010014F0EEFD66
:1027400049F2A823C1F6FF731968002900F0B88286
:10275000212000E0F0B201F00F03DAB2092B38AB10
:10276000034494BF30323732090900F1FF3603F8D1
:10277000402CEFD1C0F1220128AB184414F0CEFD5B
:102780004FF6CC70C0F20100062114F0C7FD009B8B
:1027900093F88431013B03EB8303DB0002332120F8
:1027A00000E0F0B203F00F02D1B2092A38AA0244C5
:1027B00094BF303137311B0900F1FF3602F8401C5D
:1027C000EFD128ABC0F12201184414F0A7FD179BEC
:1027D00002211B88ADF8A03028A814F09FFD009BB3
:1027E0004FF64877C0F2010793F884E10FCF28AE87
:1027F0000FC60FCF0FC60FCF0FC697E80F000EF111
:10280000FF3E86E80F000EEB8E0E49F2AC20C1F6BB
:10281000FF704FEACE034FF0FF3210F8011B81EA40
:10282000020638AF06F00F0607EB860656F8406C36
:1028300086EA121686EA111202F00F0207EB8202F4
:1028400052F8401C81EA161249F2D021C1F6FF71FC
:1028500088426FEA0202E0D149F2A826C1F6FF766B
:10286000C6F1A05909F10109012701F8282C994462
:10287000C4F2020798460394CDF828A049F2A82391
:10288000C1F6FF73C3F10102013642443244B2F58E
:10289000805F23D23B7816F801ACDA0775D516F8BD
:1028A00009309A4506EB090418D03B78DB076FD551
:1028B00023789A4512D02B78802B6CD00020C4F25C
:1028C0000200037813F0700300D0037084F800A0B6
:1028D0003B78DC07FCD52B78012B6ED049F2D02356
:1028E000C1F6FF739E42C9D101230099039CDDF814
:1028F00028A00022C4F2020381F884211B78199ACF
:10290000D807167840F196840123C1F200431B7862
:102910009E423FF4BEAD0123C4F202031B78D907E7
:1029200040F123850123C1F200431B789E423FF40E
:10293000B0AD2B78802B01F082810022C4F202021C
:10294000137813F0700300D013700122C1F200421B
:1029500001231670C4F202031A78D207FCD52B7833
:10296000012B7FF496AD4EF20103C4F207036022FF
:102970001A702B78802BFCD148F24403C4F2040374
:102980000022C0F206221A6083E510F0ABFA86E757
:1029900010F0A8FA8CE748F24400C4F204004EF2AA
:1029A00001030022C4F20703C2F2282202600020C1
:1029B00018702B78802BFCD080E74EF20103C4F214
:1029C000070360221A702B78802BFCD148F2440355
:1029D000C4F204030022C0F206221A607EE70B2A2A
:1029E00040F0F6830B2B7FF4DCAB009B1B6A002BC3
:1029F0007FF423AEFFF7D5BB092B7FF4D2AB320EA9
:102A0000009B00F007879B69002B3FF4CAABC6F31D
:102A10000741C0B29847FFF7C4BB082B7FF429AC2D
:102A2000D6F864319DF80C80802286F83A2053B3A2
:102A3000C9F307464FEA196740463A463146984778
:102A4000D8E572B61346128C5969D86813F06CFA3F
:102A500062B6FFF7EABB12F023F9C6F89800002827
:102A60007FF4DFA9FFF765BB0B2F40F065840B2BCC
:102A70007FF4FFABD6F870319DF80C80B02286F859
:102A80003A20002BD4D14FEA1967C9F30746B1E5C4
:102A9000092B7FF4EEAB5FEA196700F01C86D6F8CD
:102AA00068319DF80C80902286F83A20002B01F0C6
:102AB0002F81C9F30746FFB23A4631464046984750
:102AC00098E5DAF8803143F6A060C2F20000002BEE
:102AD00001F0AA80B0F86021B2F5917F80F0718397
:102AE000511C89B252449DF82830AAF8601182F82E
:102AF0003D30052F00F05B83DAF8803143F6A066A5
:102B0000C2F20006002B01F05780B1F5917F81F0F1
:102B10005F80481C0A4681B252444FEA194043F68E
:102B2000A066072FAAF8601182F83D00C2F20006E5
:102B300041F04980002B00F04982B1F5917F01F00E
:102B40008A814A1C92B2D7B2100A51444FEA1969DD
:102B500081F83D9011460026F0228AF83B708AF8F1
:102B60003C00AAF860618AF83A20002B00F03D8210
:102B700043F6DD600122C2F200009847FFF779BBFF
:102B80000099B1F854004BF2200EB0F5917FC1F6D8
:102B9000FF7E80F019820EEB0007411C052A87F8A2
:102BA000583089B241F0FF810098D0F87C31002282
:102BB000A0F85420002B3FF4F4AA4BF27800C1F6A1
:102BC000FF709847FFF7EDBA984700283FF4BAAA7C
:102BD00006E415F0D7F93B682693269B3360FFF790
:102BE00089B9F2293FF4DDAA40F21B83F32900F0F2
:102BF0000E83F6297FF4D5AA009B9B6B002B7FF4F4
:102C0000C7ACFFF7CEBAD6F88031002B01F02A808E
:102C1000B6F86011B1F5917F80F079824A1C701886
:102C200091B2B1F5917FA6F8601180F83D80C9F3AB
:102C3000074700F05C824A1C0AEB010091B2B1F533
:102C4000917F4FEA1969AAF8601180F83D7000F091
:102C500045824A1C92B20B465344AAF8602183F87D
:102C60003D90FFF706BBB8F1F20F00F0828340F20F
:102C7000E582B8F1F30F00F08E83B8F1F60F7FF420
:102C8000F8AADAF89431002B00F0D4819847C9F300
:102C90000746A7E4169AD05C159A1668DAB2C0B255
:102CA0008EF80020002E3FF4C6AB994238BF403169
:102CB000FFF7BCBB30238DF8C1300121212034E562
:102CC00030238DF8C1300121212055E5020600F1A5
:102CD000D0829BF84F2043F6A050C2F20000F02AA9
:102CE000426D00F0BA82461802F1FF3E8E4586F82A
:102CF0004F3000F2B98290F84FC0BCF1F00F3FF4B2
:102D0000B0AB1CF0800F40F0F28200238BF86630ED
:102D1000B02B00F00483A02B00F00183D02B00F037
:102D2000FE82E02B00F0FB82C02B00F0F882002036
:102D300043F6A056C2F20006032A08BF96F85120B7
:102D40009BF850108BF8650018BF002200264FF04A
:102D5000010EB02B8BF867108BF86820CBF8586009
:102D6000CBF854608BF8E9E000F0BC8200F2B3824B
:102D7000902B00F0B782A02B00F0B482802B00F0E3
:102D8000B18200238BF84D309BF86630902B75D0C4
:102D9000A3F18006F6B2602E43D9F12B47D04DD96E
:102DA000FA2B01F0F98073D8F32B01F01781C1F0F1
:102DB000B680F62B01F0AC80F82B03D1DBF8303075
:102DC00003B198479BF8642043F6A056D307C2F29C
:102DD00000067FF5B7A912F0FE0F3FF4B3A996F8ED
:102DE000661081F08003602B6ED896F865309F42A4
:102DF00000F03481002F00F031815208012A00F0E8
:102E00009282032A7FF49EA9084696F8682096F8D5
:102E1000671008F00BFEFFF795B980238BF866303A
:102E200000228742B9D0002FCCD1F12BB7D1DBF8EB
:102E30002030002BC6D008469847C3E7B02B01F0DE
:102E4000598040F22081D02B01F05B8040F2E88471
:102E5000E02B01F03680F02BB4D1DBF81C3043F6C8
:102E6000A050C2F20000002BACD0B0F8671080294F
:102E700000F1690028BF80219847A3E7002ACCD041
:102E80008742D0D1DBF80430002B9BD0984799E7DC
:102E9000FC2B00F04987C0F04087FE2B00F04B87E9
:102EA000FF2B8FD1DBF84430002B8AD18AE7FE2933
:102EB00000F0F880FF297FF474A9009B1B6D002BA4
:102EC0007FF466ABFFF76DB9F62900F0BE8500F21E
:102ED000B485F12900F0AF8440F2CC85F22900F0EE
:102EE0006382F3297FF42EA9B06C0E99026896F8DC
:102EF000676013688B4240F06D870F9B1B68590514
:102F00005CD50C9B1B680BB101221A70079B1F78C4
:102F100001373F2F2B4688BF4FF000084FF4204960
:102F2000254694BF5FFA87F84746C4F206091C4657
:102F3000049B1B78BB422CD1EFF31383002B40F092
:102F4000B880EFF31083002B40F0B380EFF30581DE
:102F5000002900F0AB860F2905D94EF2F033CEF2EE
:102F600000030B441B78EFF3118111B18B4228BF92
:102F70000B46402B40F29D80B3F5807FD8D1019B5A
:102F80001B78002BD4D114F0C9F8049B1B78BB42EA
:102F9000D2D008990D982346F322CA552C46012118
:102FA0001D464FF420430170C4F206030799BC226A
:102FB00081F80080DA70DBF848000268D36C06F014
:102FC0007F019847FFF7BEB80146EDE5B1F5917F67
:102FD0007FF4B7AD0B1200228AF83C30F0238AF858
:102FE0003B10AAF860218AF83A30DAF88431002BD5
:102FF0003FF43FA943F6DD60C2F200009847FFF7B7
:1030000038B99847FFF717BAB8F1FE0F00F05983A7
:10301000B8F1FF0F7FF42DA9DAF8AC2143F6A063D5
:10302000C2F20003002A7FF4DAAAD3F8B0310BB160
:1030300040469847C9F30746FFF7D4BA009BDB69BF
:10304000002B7FF4FAAAFFF7ACB811F029FEC6F8FE
:10305000980000287EF4EFAEFFF76BB89BF8642071
:10306000520843F6A056012AC2F2000600F05B8126
:10307000022A7FF467A8C7E6009B1B6C002B7FF435
:1030800087AAFFF78EB8902B3FF4FCAEA02B00F080
:103090009A86802B7FF496AEDBF80030002B7FF40D
:1030A000F5AE8FE6009BDB6C002B7FF471AAFFF777
:1030B00078B899F804301B067FF53AAF049B089A5C
:1030C0001B7801333F2B86BF00210B46D9B2D35C5E
:1030D000DBB289F80730049B197029E743F6DD60FD
:1030E0000022C2F20000984700230122B4E500222A
:1030F00006F13D009847D6F8802186F83D704FEAEA
:1031000019690123002A00F0CD851946A1E50022A6
:1031100006F13D009847D6F8803186F83D800122BF
:10312000C9F30747002B00F0B085114683E50FF087
:10313000D9FEFFF7D0B9D6F86C319DF80C80A022EB
:1031400086F83A20002B7FF473AC4FEA1967C9F375
:103150000746FFF74FBA009AB2F854004BF220022C
:10316000B0F5917FC1F6FF72BFF41BA8411C171880
:1031700089B2B1F5917F87F85830A2F85410C6F3A0
:1031800007473FF40EA85318811C89B2B1F5917F0F
:1031900083F85870A2F854103FF403A81144033088
:1031A000360EA2F8540081F85860FEF7FABFB8F165
:1031B000F70F7FF45EA8DAF88031CFB2C1F30720B1
:1031C000C9E411463D30002298470022012189E4DC
:1031D0000C2A40F052860C2B7EF4E3AF009B5B6A16
:1031E000002B3EF4DEAFC6F30741C0B29847FEF7AE
:1031F000D8BF009B9B6C002B7FF4CAA9FEF7D1BF00
:10320000009BDB6B002B7FF4C3A9FEF7CABF009BBA
:103210005B6B002B3EF4C5AFC6F307409847FEF743
:10322000C0BFF1297EF4BDAF009B1B6B002BF3D117
:10323000FEF7B7BF0FF056FEFFF766BBB8F1F10F10
:103240007FF417A8DAF88831C9F30746002B3FF45A
:10325000C9A930469847FFF7C5B90844013A8A42E0
:1032600080F869307FF6FDA80131CBF85810FEF7E1
:1032700069BFA3F1F70008283FF62BAD4FF0010E10
:103280000EFA00F212F4DD7F40F0AF8500287FF4E3
:1032900020AD9BF8693043F6A056F02BC2F2000631
:1032A0007FF4DFA84A1C06EB01084FF0F70CD1B2FF
:1032B000C2F3072286F8663086F8650086F8E9E0F2
:1032C000B065706586F84D0088F869C086F86710AB
:1032D00086F868205CE5D02B04D0E02B02D0C02B10
:1032E0007FF44FAD8BF84DC09BF866304EE50CF186
:1032F0000C03DBB2012B7FF608AD0CF0FB03F92BBE
:103300003FF403ADBCF1EF0F00F282850CF0F00347
:10331000802B80F8663002D0902B7FF4F9AC0CF053
:103320000F00013004E508469BF868209BF8671001
:1033300008F07CFBFEF706BF0C2F40F00A850C2B33
:103340007EF497AFD6F874319DF80C80C02286F8D1
:103350003A20002B3FF497ABC9F30746404631466D
:103360004FEA19679847FFF745B90FF0BBFDFFF724
:10337000D9BADAF88C21002A3FF45CAE4FEA19463C
:103380004FEA594306F07F0003F47E531843F6B228
:103390009047FFF727B9DAF89031C9F30746002BB9
:1033A0007FF457AFFFF71EB9B06C96F8672096F818
:1033B0006870D0F800E042EAC717DEF800300E9AD5
:1033C000934240F042850F9B1B685E055DD50C9BC8
:1033D0001B680BB101221A70079B1E7801363F2E25
:1033E0002B4688BF4FF000084FF42049254694BF74
:1033F0005FFA86F84646C4F206091C46049B1B7811
:10340000B3422CD1EFF31383002B40F01581EFF37F
:103410001083002B40F01081EFF30581002900F0AC
:1034200020810F2905D94EF2F033CEF200030B4470
:103430001B78EFF3118111B18B4228BF0B46402B53
:1034400040F2FA80B3F5807FD8D1019B1B78002B26
:10345000D4D113F063FE049B1B78B342D2D00899F9
:103460000D982346F2228A552C4601211D464FF421
:1034700020430170C4F206030799BC2281F8008042
:10348000DA70DBF84800D0F800E0DEF84830189A2F
:10349000934207F07F0140F0CF84DEF800205FFA0E
:1034A00081F80E998A4240F0B6840F9A126852054C
:1034B00062D50C9B1B680BB101221A70079B039508
:1034C0001E7801363F2E4FF42043524688BF4FF0FE
:1034D0000009C4F20603A24694BF5FFA86F94E467D
:1034E0001D461446049B1A78B2422CD1EFF3138286
:1034F000002A40F0BC80EFF31082002A40F0B78031
:10350000EFF30580002800F0AF800F2805D94EF2B8
:10351000F032CEF2000202441278EFF3118010B1C3
:10352000824228BF0246402A40F2A180B2F5807F45
:10353000D8D1019B1A78002AD4D113F0EFFD049B57
:103540001A78B242D2D02346089A0D9802F8068023
:10355000012154469A464FF420430170C4F20603F9
:103560000799039D81F80090BC22DA70DBF84800CF
:10357000D0F800E0DEF84830189A9342C7F3C6113D
:1035800040F05784DEF800300E9A9342CEB240F0FD
:1035900030850F9B1B6858057EF5D4AD0C9B1B68CE
:1035A0000BB101221A70079B1F7801373F2F2B4662
:1035B00088BF4FF000084FF42049254694BF5FFABA
:1035C00087F84746C4F206091C46049B1B78BB4299
:1035D00028D1EFF31383002B5FD1EFF31083002B7F
:1035E0005BD1EFF30581002954D00F2905D94EF2A4
:1035F000F033CEF200030B441B78EFF3118111B1CD
:103600008B4228BF0B46402B47D9B3F5807FDCD1D6
:10361000019B1B78002BD8D113F080FD049B1B78F5
:10362000BB42D6D02346089A2C461D464FF4204371
:10363000C4F20603D655C7E199F8043019067FF5A0
:10364000DDAE049B089A1B7801333F2B86BF002117
:103650000B46D9B2D35CDBB289F80730049B1970F2
:10366000CCE64FF48073E4E64FF4807255E72A7994
:1036700013067FF537AF049B1A78089B01323F2A67
:1036800086BF00200246D0B29A5CD2B2EA71049B97
:10369000187027E74FF48073AFE799F804301906E4
:1036A00093D5049B089A1B7801333F2B86BF0021DA
:1036B0000B46D9B2D35CDBB289F80730049B197092
:1036C00083E7DAF8A82143F6A063C2F20003002AD8
:1036D0007EF485AFA9E4D6F864319DF80C80802291
:1036E00086F83A20C9F30746002B00F02F833146B5
:1036F00040463A469847FEF77DBF02F10C06F1B20C
:1037000001297EF6AAAE02F0FB01F9293EF4A5AE2E
:10371000EF2A35D802F0F001802932D101063EF5BA
:103720009CAE01218BF84F208BF85030CBF858100D
:10373000F6B2012E7EF695AE02F0FB03F92B3EF4B5
:1037400090AEEF2A33D802F0F003B02B3BD040F21A
:10375000F483D02B04D0E02B35D0C02B7EF481AE87
:103760000223CBF854300121DBF8583043F6A05047
:103770008B42C2F2000032D201338365FEF7E2BC15
:10378000114601F0DF0EBEF1900FC7D001F0BF0E61
:10379000BEF1A00FC2D001F0EF01C029BED05AB2D5
:1037A000002ABEF65EAE1A4603F10C06C0E7F62A02
:1037B00000F0D88300F2CF83F12AD1D040F21D84EB
:1037C000F22A40F0E4830323CBF854300221DBF8E3
:1037D000583043F6A0508B42C2F20000CCD3EF2AFF
:1037E00094BF02F0F003134602F00F02501C9BF846
:1037F00050108BF86500002201268BF866308BF89C
:1038000067108BF86820CBF85820CBF854208BF841
:10381000E960F7E25B69002B7FF4F9A8FEF7C1BC11
:10382000C02B7FF4CFAADBF81030002B3FF4CAAADC
:103830009847FFF7C7BAB06C96F8672096F868709B
:103840000368120102F0700207F00F071B681743AC
:103850000E9A934240F049830F9A126852055DD543
:103860000C9B1B680BB101221A70079B1E78013656
:103870003F2E2B4688BF4FF000084FF420492546C5
:1038800094BF5FFA86F84646C4F206091C46049BBC
:103890001B78B3422CD1EFF31383002B40F09E80B2
:1038A000EFF31083002B40F09980EFF3058100299E
:1038B00000F0A9800F2905D94EF2F033CEF20003B3
:1038C0000B441B78EFF3118111B18B4228BF0B46DB
:1038D000402B40F28380B3F5807FD8D1019B1B78C9
:1038E000002BD4D113F01AFC049B1B78B342D2D026
:1038F00008990D982346F1228A552C4601211D4630
:103900004FF420430170C4F206030799BC2281F8EA
:103910000080DA70DBF8480003681B680E9A934257
:1039200040F0DF820F9B1B6858057EF50BAC0C9BAB
:103930001B680BB101221A70079B1E7801363F2EBF
:103940002B4688BF4FF000084FF42049254694BF0E
:103950005FFA86F84646C4F206091C46049B1B78AB
:10396000B34228D1EFF31383002B4FD1EFF3108331
:10397000002B4BD1EFF3058100295BD00F2905D92E
:103980004EF2F033CEF200030B441B78EFF31181BB
:1039900011B18B4228BF0B46402B37D9B3F5807F3E
:1039A000DCD1019B1B78002BD8D113F0B7FB049B13
:1039B0001B78B342D6D0089A234697552C461D460D
:1039C0004FF42043C4F206030D98012101700799BA
:1039D000BC2281F80080DA70FEF7B4BB99F804309D
:1039E0001B067FF554AF049B089A1B7801333F2BCD
:1039F00086BF00210B46D9B2D35CDBB289F8073011
:103A0000049B197043E74FF480735BE799F8043027
:103A10001906A3D5049B089A1B7801333F2B86BF58
:103A200000210B46D9B2D35CDBB289F80730049B86
:103A3000197093E74FF48073A8E7FC2900F2D58250
:103A4000FA2902D2F8297EF47DAB01F10803DBB23A
:103A5000072B3EF677AB012202FA03F313F0DD0FDA
:103A60003EF470AB43F6E850C2F200000DF01CFECD
:103A7000FEF768BBF0297EF465ABB6F86730802BA3
:103A800028BF8023002B3EF45DAB68334FF4204702
:103A90003344DDF810900A9306F16808C4F2060773
:103AA000DBF848000E9A036818F8011F1B68934260
:103AB00071D10F9B1B685E0553D50C9B1B680BB126
:103AC00001221A70079B03911E7801363F2E8CBF8E
:103AD0000023F3B22A4688BF1E461D4611465346B0
:103AE000A24699F80020B2422CD1EFF31382002AAB
:103AF0003CD1EFF31082002A38D1EFF30580002883
:103B000046D00F2805D94EF2F032CEF20002024420
:103B10001278EFF3118010B1824228BF0246402A8A
:103B200024D9B2F5807FDCD1019A1278002AD8D14D
:103B30002191209313F0F2FA99F800202199209B0B
:103B4000B242D2D00A4654469A462B461546089AA7
:103B5000039991550D99012008700799BC220B70AB
:103B6000FA700A9B98459BD1FEF7ECBA3A79100699
:103B7000B7D599F80020089C01323F2A86BF002063
:103B80000246D0B2A25CD2B2FA7189F80000A8E76E
:103B90004FF48072BDE798470A9B984580D1FEF7A5
:103BA000D1BADAF89C2143F6A063C2F20003002ADE
:103BB0007EF415ADFFF739BAB1F5917FFEF4A9AFE8
:103BC000072F3FF407AACFB2C1F30720FEF7C3BF08
:103BD000002206F13D009847D6F8803100220121ED
:103BE000FEF79ABFDAF8A42143F6A063C2F20003FD
:103BF000002A7EF4F4ACFFF718BA48F24402C4F28B
:103C000004024EF201030021C4F20703C2F228218C
:103C1000116000221A702B78802BFCD0FEF770BC4C
:103C20000FF060F9FEF763BCB0F86011B1F5917F59
:103C3000BEF45FAF4B1C0A4699B2FEF753BF48F281
:103C40004402C4F204024EF201030021C4F207034D
:103C5000C2F22821116000221A702B78802BFCD030
:103C6000FEF76BBEB6F86031B3F5917FBEF401ABE1
:103C70005A1C92B23344B2F5917FA6F8602183F8C2
:103C80003D80C9F307473EF4F4AA531C9BB252444B
:103C9000B3F5917F4FEA1969AAF8603182F83D7057
:103CA0003EF4E7AA5A1C92B2FEF7D6BF4FF48073D7
:103CB000FFF759B94EF20103C4F2070360221A70EC
:103CC0002B78802BFCD148F24403C4F20403002279
:103CD000C0F206221A60FEF728BCDAF8982143F6F3
:103CE000A063C2F20003002A7EF479ACFFF79DB90D
:103CF00043F6DD600022C2F2000098470021012354
:103D0000FEF750BBB1F5917FBEF4B3AAFEF748BBF6
:103D1000FFB2C9F30746FEF76DBCDBF83830002B65
:103D20007FF44FA8FFF74EB8DBF83C30002B7FF450
:103D300048A8FFF747B8DBF84030002B7FF441A8D4
:103D4000FFF740B801212120FEF7EFBC1F46FEF728
:103D500051BC0D2F12D10D2B7EF48BAAD6F87831E1
:103D60009DF80C80D02286F83A20002B7FF4F4AA2C
:103D70004FEA1967C9F30746FEF73CBC0E2B7EF4E9
:103D800078AAD6F87C31E02286F83A209BB14FEA37
:103D900019464FEA594106F07F029DF80C8001F464
:103DA0007E511143A1F5005140469847F6B24FEAC3
:103DB0001967FEF71FBC9DF80C804FEA1967C9F31D
:103DC0000746FEF717BCDBF80830002B7FF45EA82F
:103DD000FEF7F8BFF3219847DBF84800026806F0C9
:103DE0007F01D36C9847FEF7ADB9002211468BF8DE
:103DF00066308BF8E9E08BF867208BF868208BF849
:103E000065201046902B3FF408A80022FEF7C0BFA3
:103E10006346FEF77BBF41469047DBF84800189A9F
:103E2000D0F800E0DEF848309342C7F3C6113FF403
:103E3000A9AB9847FEF786B99847DBF84800D0F859
:103E400000E0DEF84830FFF797BB9847B06CD0F839
:103E500000E0FFF71ABB002206F13D00984701275A
:103E60000020D6F8803101463A46FEF76EBEB16DAD
:103E7000FF2311B30820FFF701BA0D2A09D10D2B3A
:103E80007EF48FA9009B9B6A002B7FF4ACA9FEF700
:103E900088B90E2B7EF485A9009BDB6A002B3EF4CB
:103EA00080A9720C02F47E52C6F306411143C0B2DF
:103EB000A1F500519847FEF774B94FF0FF30FEF7B7
:103EC000C5BADBF81830002B3EF47CAFD20102F407
:103ED0007E5201F07F011143A1F500519847FEF792
:103EE00071BF39469847FEF72DB99847B06C036803
:103EF0001B6813E5DBF80C30002B7EF4C7AFFEF730
:103F000061BFDBF81430002B7FF492ACFEF75ABF90
:103F1000DBF82C30002B7EF454AFFEF753BFDBF8F8
:103F20002430002B3EF44EAFD20102F47E5201F059
:103F30007F0010439847FEF745BF902B3FF443ACFA
:103F4000A02B3FF440AC802B7EF48BAA0323CBF84C
:103F5000543002213BE4FC2A5DD8FA2A02D2F82A26
:103F60007EF47FAA002001268BF8662013460146C6
:103F70008BF865008BF867008BF86800CBF8580069
:103F8000CBF8540002468BF8E960FEF701BFF32A34
:103F90003FF4E6ABFEF765BADBF83430002B7EF475
:103FA00010AFFEF70FBFB1F5917F3EF4FDAD0EEB04
:103FB0000107831C310C072A87F8581099B27EF448
:103FC000F3ADB1F5917F4FEA16663EF4EDAD714465
:103FD000033081F8586081B2FEF7E6BDDBF8283087
:103FE000002B7EF428AFFEF7EDBEFE29FEF4AAA852
:103FF0002BE531469847FEF7A5B8F02A7EF431AAA2
:1040000080210023CBF854108BF869208BF84D30B9
:104010007F21FFF7A9BBFE2AA4D2FEF722BA00BF78
:104020002DE9F04F40F64C01342649F23405C4F234
:104030000405C4F2FE31C4F2FE3649F63003002214
:10404000C1F6FF7340F203144AF24C002DED028BCF
:10405000C4F2040086F880222C6081F8802259691D
:10406000046083F8382083F8392083F85C2083F8D3
:104070005D2083F85E2083F85F200C68486825681F
:104080005A6628439A6620601869827093F8612006
:104090000C680A444EF6D020157A527BC0F20E000E
:1040A00000EBC50512026D6802F4E06242F06402A2
:1040B0002A6093F862200A4493B0957CD27D00EB8D
:1040C000C5001202406802F4E06242F0640202603D
:1040D00020684A68104205D01A692C2151701A696B
:1040E000042191711A69202151711B694DF2044517
:1040F000C1F6FF7580229A702B7B6B720022012B18
:10410000AA7184BF0822AA7132200FF075FD4DF20A
:104110000440697BC1F6FF700DF0D4FE4FF47A7055
:104120000FF06AFD4DF20440C1F6FF7030210DF032
:10413000C9FE41F6B0644DF20440C1F6FF70302173
:10414000C0F204040DF07AFE2346013BFDD14DF28E
:104150000440C1F6FF7030210DF0B4FE4DF2044072
:10416000C1F6FF7030210DF069FE013CFDD14DF22A
:104170000440C1F6FF7030210DF0A4FE4DF2044062
:10418000C1F6FF7030210DF059FE42F22833013B99
:10419000FDD14DF20440C1F6FF7020210DF092FEDA
:1041A0004DF20440C1F6FF7020210DF047FEA979C1
:1041B0004DF2044041F02001C1F6FF7000220DF0E5
:1041C0009DFE04234DF20440EB7100220C21C1F648
:1041D000FF700DF093FE4DF20440C1F6FF700DF03C
:1041E00005FF02244DF20440C1F6FF7000220621B3
:1041F0002C720DF083FE4DF204402146C1F6FF7093
:1042000000220DF07BFE4DF2C043C0F20103013BE2
:10421000FDD1EB794DF2044003F0FE0343F00801B9
:10422000EB71C1F6FF7000220DF068FEEB794DF2E4
:10423000044003F0FD03002243F00801EB71C1F6D6
:10424000FF700DF05BFE08234DF204406B730021FC
:10425000C1F6FF700DF036FE4DF20440C1F6FF705E
:104260000DF0C4FE4DF204400022C1F6FF700121A2
:104270000DF098FE4EF230414DF20440C0F20E01B6
:10428000C1F6FF7004F0A8FA4DF204400122C1F615
:10429000FF7000210DF086FE4EF240414DF20440C9
:1042A000C0F20E01C1F6FF704DF27C494DF61415B7
:1042B000C1F6FF7504F090FAC1F6FF794FF47A70F9
:1042C0000FF09AFC4DF240584946284612F0B0FED5
:1042D000C1F6FF784DF2C86341461E46284612F0EB
:1042E000A7FE4DF204673346C1F6FF73C1F6FF77B0
:1042F0001E46394628464DF28C7B12F099FEC1F6D7
:10430000FF7B314628464DF6500AC1F6FF7A0096EB
:1043100012F08EFE5946284612F08AFE5146284673
:1043200012F086FE4DF668102946C1F6FF7085F83A
:1043300052400DF075FD45F209021046C0F2010031
:1043400045F29102154601902846019DC9F8085092
:104350004FF0010589F8C15088F8C15087F8C15065
:10436000C0F20100009D02904FF0010985F8C19054
:104370004DF60036029DC8F80C50C1F6FF76009D40
:104380008BF8C1904DF2792C4BF2191E4BF2E15291
:104390004BF21D534DF67811C0F2000CC0F2000E26
:1043A000C0F20002C0F200033046C1F6FF71C7F848
:1043B00010C0C5F814E0CBF81820CAF81C308AF8F1
:1043C000C19012F035FE4DF63C213046C1F6FF712A
:1043D00012F02EFE4DF664331D464DF654304EF26B
:1043E00048274DF62843C1F6FF773146C1F6FF75E1
:1043F000C1F6FF73C1F6FF7086F852401E460DF0FD
:104400000FFD4DF6EC43294638460093069512F011
:104410000FFE009B02964DF6B052C1F6FF73314677
:10442000384616461D4612F003FE3246C1F6FF72AC
:1044300016464DF67462294638460095154612F028
:10444000F7FD2A46C1F6FF721546314638464DF64D
:10445000387BC1F6FF7B03964DF6FC7A12F0E8FD3F
:1044600029463846C1F6FF7A04954EF2C00912F08B
:10447000DFFD5946384612F0DBFDC1F6FF795146A3
:1044800038464EF2841812F0D3FDC1F6FF78494643
:10449000384612F0CDFD4146384612F0C9FD4EF2C5
:1044A0009C204EF234433946C1F6FF73C1F6FF70CB
:1044B00087F8524005930DF0B3FC44F68D71084621
:1044C00044F611710D46C0F2010007904CF6DD6113
:1044D00028460A46C0F20100089010464CF6555294
:1044E000029DC0F2000201924FF0010285F8C12046
:1044F000009D8BF8C12085F8C120039D8AF8C1205A
:104500004DF2F51785F8C1203E46049D89F8C1207B
:10451000C0F2000009903046069E85F8C120079D34
:104520003562029D86F8C1202E46089D7562009D69
:1045300088F8C1202E46099DB562039DC0F2000097
:104540000A902E460A9DF5624CF6596C049D05981A
:10455000C0F2000C4CF6D15E4DF265174DF2E5034A
:104560004EF2AC21C5F830C0C0F2000EC0F200031C
:10457000019ACBF834E0C0F20007C1F6FF71C9F828
:104580003C20C8F84030CAF8387012F051FD059D43
:104590004EF270312846C1F6FF7112F049FD4EF21D
:1045A00088402946C1F6FF704EF22068C1F6FF78B8
:1045B00085F852400DF034FC4EF298414046C1F669
:1045C000FF7112F035FD4EF25C514046C1F6FF71AD
:1045D00012F02EFD4EF274604146C1F6FF704EF6A9
:1045E0000C07C1F6FF7788F852400DF019FC4EF227
:1045F00084613846C1F6FF7112F01AFD4EF248711F
:104600003846C1F6FF7112F013FD4EF660003946D0
:10461000C1F6FF704EF6F816C1F6FF7687F85240E5
:104620000DF0FEFB4EF670013046C1F6FF7112F040
:10463000FFFC4EF634113046C1F6FF7112F0F8FC63
:104640004EF64C203146C1F6FF704EF6E437C1F607
:10465000FF7786F852400DF0E3FB4EF65C213846BA
:10466000C1F6FF7112F0E4FC4EF620313846C1F677
:10467000FF7112F0DDFC4EF638403946C1F6FF708E
:104680004EF6D056C1F6FF7687F852400DF0C8FBC3
:104690004EF648413046C1F6FF7112F0C9FC4EF6A5
:1046A0000C513046C1F6FF7112F0C2FC4EF6246088
:1046B0003146C1F6FF704EF6BC77C1F6FF7786F83B
:1046C00052400DF0ADFB4EF634613846C1F6FF7135
:1046D00012F0AEFC4EF6F8613846C1F6FF7112F0EA
:1046E000A7FC4FF210003946C1F6FF704FF2A81632
:1046F000C1F6FF7687F852400DF092FB4FF2200191
:104700003046C1F6FF7112F093FC4FF2E4013046DF
:10471000C1F6FF7112F08CFC4FF2FC103146C1F66D
:10472000FF704FF29437C1F6FF7786F852400DF0D4
:1047300077FB4FF20C213846C1F6FF7112F078FC7E
:104740004FF2D0213846C1F6FF7112F071FC4FF2E2
:10475000F8324FF2E8304FF2BC43C1F6FF733946EE
:10476000C1F6FF72C1F6FF7087F8524000930192C4
:1047700040F248360DF054FB019A0F92C2F2000647
:104780001146304612F054FC009B0E934FF2805BB2
:104790001946C1F6FF7B30464FF2446A12F048FCDE
:1047A000C1F6FF7A5946304612F042FC4FF20879C2
:1047B0005146304612F03CFCC1F6FF794FF69003AB
:1047C0004FF2CC78C1F6FF7849461D46304612F0CC
:1047D0002FFCC1F6FF754FF65413414630462F4665
:1047E0001D4612F025FC4FF6182239463046009738
:1047F000174612F01DFC3A46C1F6FF721746C1F685
:10480000FF754FF6DC22294630460195154612F019
:104810000FFC2A46C1F6FF7239463046154602970C
:1048200012F006FC4FF6644E294630460395754655
:104830004FF6A03712F0FCFB2946C1F6FF774FF682
:10484000285EC1F6FF710D4630463946049777461B
:1048500012F0EEFB39464FF6EC5EC1F6FF710F46E3
:10486000304629460595754612F0E2FB29464FF67B
:10487000B06EC1F6FF710D46304639460697774651
:1048800012F0D6FB39464FF6747EC1F6FF710F4623
:10489000304629460795754612F0CAFB294640F274
:1048A000380EC1F6FF710D463046394608977746F7
:1048B00012F0BEFB394640F2FC0EC2F200010F4678
:1048C000304629460995754612F0B2FB294640F25A
:1048D000C01EC2F200010D46304639460B9777469E
:1048E00012F0A6FB394640F2842EC2F200010F46B8
:1048F000304629460C95754612F09AFB2946C2F2BD
:1049000000010D46304639460D9712F091FB2946BD
:1049100030460A9512F08CFB40F29C303146C2F2D0
:10492000000086F852400DF07BFA0F9A4FF0010319
:1049300082F8C1300E9B4FF0010583F8C1508BF80F
:10494000C1508AF8C15089F8C15088F8C150009D03
:10495000AE464FF001058EF8C150019DAE464FF0B6
:1049600001058EF8C150029DAE464FF001058EF84C
:10497000C150039DAE464FF001058EF8C150049D15
:10498000AE464FF001058EF8C150059DAE464FF082
:1049900001058EF8C150069DAE464FF001058EF818
:1049A000C150079DAE464FF001058EF8C150089DDD
:1049B000AE464FF001058EF8C1504CF6D941099D25
:1049C000C0F20001AE4651644CF65D464DF2610006
:1049D0004CF6DD714CF6E132C0F20006C0F2000088
:1049E0004FF00105C0F20001C0F200028EF8C15084
:1049F0009E64CBF84C00CAF850104CF6ED26C9F86E
:104A00005420009DC0F20006EE654CF65970019DE1
:104A1000C0F2000028664CF6712E029DC0F2000E16
:104A2000C5F864E04CF6F51C039DC0F2000CC5F817
:104A300068C04CF6791A049DC0F2000AC5F86CA053
:104A40004CF6FD02059DC0F200022A674CF6693360
:104A5000069D4CF68109C0F20003C0F20009C8F8B7
:104A60005830C5F874904BF2A148079DC0F2000879
:104A7000C5F878804BF2254B089DC0F2000BC5F8B5
:104A80007CB04BF2A936099D4BF22D33C0F20006E3
:104A9000C0F200030093C5F880600B9D009EC5F82E
:104AA00084604FF001024BF2B12085F8C1204BF237
:104AB00029230C9D0D9EC0F2000001904FF00102D1
:104AC000184685F8C120C0F200004FF001020E9098
:104AD00086F8C1200A9A4FF0010E82F8C1E02A46FA
:104AE00040F23457019DC2F88850C2F200070A9A7A
:104AF0000E9DC6F88C504BF2A11340F2AC31C0F2BF
:104B00000003C2F200013846C2F8903012F090FA69
:104B100040F270413846C2F2000112F089FA40F2C8
:104B200088503946C2F2000040F22078C2F20008F4
:104B300087F852400DF074F940F298514046C2F2A5
:104B4000000112F075FA40F25C614046C2F20001C9
:104B500012F06EFA40F274704146C2F2000040F664
:104B60000C16C2F2000688F852400DF059F940F2D6
:104B700084713046C2F2000112F05AFA40F6480140
:104B80003046C2F2000112F053FA40F6601031468E
:104B9000C2F2000040F6F827C2F2000786F8524041
:104BA0000DF03EF940F670113846C2F2000112F0E5
:104BB0003FFA40F634213846C2F2000112F038FACA
:104BC00040F64C303946C2F2000040F6E446C2F2EC
:104BD000000687F852400DF023F940F65C3130466C
:104BE000C2F2000112F024FA40F620413046C2F22F
:104BF000000112F01DFA40F638503146C2F20000B2
:104C000040F6D067C2F2000786F852400DF008F96E
:104C100040F648513846C2F2000112F009FA40F657
:104C20000C613846C2F2000112F002FA40F624701C
:104C30003946C2F2000041F2BC06C2F2000687F813
:104C400052400DF0EDF840F634713046C2F20001EA
:104C500012F0EEF940F6F8713046C2F2000112F09F
:104C6000E7F941F210103146C2F2000041F2A827E4
:104C7000C2F2000786F852400DF0D2F841F220113E
:104C80003846C2F2000112F0D3F941F2E41138467D
:104C9000C2F2000112F0CCF941F2FC203946C2F216
:104CA000000041F29446C2F2000687F852400DF02F
:104CB000B7F841F20C313046C2F2000112F0B8F9F7
:104CC00041F2D0313046C2F2000112F0B1F941F2A6
:104CD000E8403146C2F2000041F28067C2F20007AC
:104CE00086F852400DF09CF841F2F8413846C2F285
:104CF000000112F09DF941F2BC513846C2F20001A8
:104D000012F096F941F2D4603946C2F2000041F641
:104D10006C06C2F2000687F852400DF081F841F2AD
:104D2000E4613046C2F2000112F082F941F2A8714A
:104D30003046C2F2000112F07BF941F6C000314664
:104D4000C2F2000041F65827C2F2000786F852402E
:104D50000DF066F841F6D0013846C2F2000112F0BB
:104D600067F941F694113846C2F2000112F060F979
:104D700041F6AC203946C2F2000041F64446C2F288
:104D8000000687F852400DF04BF841F6BC21304642
:104D9000C2F2000112F04CF941F680313046C2F205
:104DA000000112F045F941F698403146C2F2000088
:104DB00041F63067C2F2000786F852400DF030F835
:104DC00041F6A8413846C2F2000112F031F941F62D
:104DD0006C513846C2F2000112F02AF941F68460A3
:104DE0003946C2F2000042F21C06C2F2000687F801
:104DF00052400DF015F841F694613046C2F20001C0
:104E000012F016F941F658713046C2F2000112F064
:104E10000FF942F270003146C2F2000042F2082758
:104E2000C2F2000786F852400CF0FAFF42F280010D
:104E30003846C2F2000112F0FBF842F24411384643
:104E4000C2F2000112F0F4F842F25C203946C2F2DC
:104E5000000042F2F436C2F2000687F852400CF02D
:104E6000DFFF42F26C213046C2F2000112F0E0F89E
:104E700042F230313046C2F2000112F0D9F842F26B
:104E800048403146C2F2000042F2E057C2F2000749
:104E900086F852400CF0C4FF42F258413846C2F244
:104EA000000112F0C5F842F21C513846C2F200016E
:104EB00012F0BEF842F234603946C2F2000042F20B
:104EC000CC76C2F2000687F852400CF0A9FF42F2FD
:104ED00044613046C2F2000112F0AAF842F20871B1
:104EE0003046C2F2000112F0A3F842F6200031462B
:104EF000C2F2000042F6B817C2F2000786F852402C
:104F00000CF08EFF42F630013846C2F2000112F07A
:104F10008FF842F6F4013846C2F2000112F088F828
:104F200042F60C203946C2F2000042F6A436C2F224
:104F3000000687F852400CF073FF42F61C21304601
:104F4000C2F2000112F074F842F6E0213046C2F2DB
:104F5000000112F06DF842F6F8303146C2F200005E
:104F600086F8524043F68C470CF05AFF43F6043360
:104F7000C2F20003C2F200074BF27152C0F200020B
:104F800019464FF00105384683F8C150C3F8A420F4
:104F900012F04EF843F6C8313846C2F2000112F062
:104FA00047F842F6084B43F6E04042F61876C2F264
:104FB00000063946C2F2000BC2F2000042F6CC4AAB
:104FC00087F85240C2F2000A0CF02AFF42F69059CC
:104FD0005946304612F02CF8C2F2000930465146CC
:104FE00042F6546812F024F8C2F2000830464946EE
:104FF00012F01EF83046414612F01AF842F66C7074
:105000003146C2F2000043F20417C2F2000786F8EC
:1050100052400CF005FF4BF219064BF2990E4AF67E
:10502000A1724AF6197342F67C71C0F2000EC0F20A
:105030000002C0F20003C0F20006C2F200013846CE
:10504000CBF894E0C9F89C20C8F8A0308BF8C15088
:105050008AF8C15089F8C15088F8C150CAF89860E0
:1050600011F0E6FF43F24001C2F20001384611F0B0
:10507000DFFF43F258103946C2F2000043F2F02538
:10508000C2F2000587F852400CF0CAFE43F26811E4
:105090002846C2F2000111F0CBFF43F22C21284632
:1050A000C2F2000111F0C4FF43F244302946C2F2BB
:1050B000000043F2DC46C2F2000685F852400CF0D4
:1050C000AFFE43F254313046C2F2000111F0B0FF9E
:1050D00043F218413046C2F2000111F0A9FF43F239
:1050E00030503146C2F2000043F2C865C2F20005FA
:1050F00086F852400CF094FE43F240512846C2F22A
:10510000000111F095FF43F204612846C2F200014C
:1051100011F08EFF43F21C702946C2F2000043F6E4
:10512000B406C2F2000685F852400CF079FE43F254
:105130002C71C2F20001304611F07AFF43F2F07197
:10514000C2F20001304611F073FF43F608103146F9
:10515000C2F2000043F6A025C2F2000586F85240D4
:105160000CF05EFE43F618112846C2F2000111F061
:105170005FFF43F6DC112846C2F2000111F058FF30
:1051800043F6F4202946C2F2000085F852400CF0A4
:1051900047FE4DF66810C1F6FF7005F045FC4DF670
:1051A0005430C1F6FF7005F03FFC4EF29C20C1F672
:1051B000FF7005F039FC40F29C30C2F2000005F0AF
:1051C00033FC4EF28840C1F6FF7005F02DFC4EF224
:1051D0007460C1F6FF7005F027FC4EF66000C1F662
:1051E000FF7005F021FC4EF64C20C1F6FF7005F073
:1051F0001BFC4EF63840C1F6FF7005F015FC4EF66C
:105200002460C1F6FF7005F00FFC4FF21000C1F6EC
:10521000FF7005F009FC4FF2FC10C1F6FF7005F0BD
:1052200003FC4FF2E830C1F6FF7005F0FDFB40F2E1
:105230009C30C2F2000005F0F7FB40F28850C2F249
:10524000000005F0F1FB40F27470C2F2000005F0BE
:10525000EBFB40F66010C2F2000005F0E5FB40F603
:105260004C30C2F2000005F0DFFB40F63850C2F2CD
:10527000000005F0D9FB40F62470C2F2000005F0F2
:10528000D3FB41F21010C2F2000005F0CDFB41F259
:10529000FC20C2F2000005F0C7FB41F2E840C2F278
:1052A000000005F0C1FB41F2D460C2F2000005F03D
:1052B000BBFB41F6C000C2F2000005F0B5FB41F6B1
:1052C000AC20C2F2000005F0AFFB41F69840C2F2FC
:1052D000000005F0A9FB41F68460C2F2000005F071
:1052E000A3FB42F27000C2F2000005F09DFB42F207
:1052F0005C20C2F2000005F097FB42F24840C2F287
:10530000000005F091FB42F23460C2F2000005F0AB
:105310008BFB42F62000C2F2000005F085FB42F64E
:105320000C20C2F2000005F07FFB42F6F830C2F21A
:10533000000005F079FB43F6E040C2F2000005F002
:1053400073FB42F66C70C2F2000005F06DFB43F295
:105350005810C2F2000005F067FB43F24430C2F27D
:10536000000005F061FB43F23050C2F2000005F08E
:105370005BFB43F21C70C2F2000005F055FB43F6E4
:105380000810C2F2000005F04FFB43F6F420C2F211
:10539000000005F049FB05F011FB43F6F043C2F2B3
:1053A0000003002593F8AD2053F8224020680CF04C
:1053B0001DFE637B04EB83035A6892F8513092F828
:1053C000500008E0834282F8513011D052F8231087
:1053D00091F8C11061B9591C8342CBB2F2D30023BA
:1053E00082F8515052F8231091F8C1100029F2D0E0
:1053F00020684BF2C0150CF0F9FDC1F6FF75204690
:1054000003F052FE05F038F92B22FF21284613F055
:1054100007FE4DF254400023C1F6FF702B7011F0CF
:10542000BBFD4DF26440C1F6FF7011F0B5FD0123E4
:10543000C4F202031B78D80740F122874FF0A05333
:1054400049F2D0281A784DF21443C1F6FF73C1F621
:10545000FF780027D2B2632188F8002099611F7776
:105460005F6172B68A42A8BF0A469200DA6062B6ED
:10547000052698F8002083F83C705F63EA629E631B
:1054800072B6DF6262B64EF25440C0F20E002F6375
:1054900005F07CFA4EF29840C0F20E0005F076FA64
:1054A0004EF2C840C0F20E0005F070FA4EF2F8401D
:1054B000C0F20E0012F014FC4EF224400A213A46CB
:1054C000C0F20C0012F016FC4EF20C50C0F20E00AE
:1054D00005F05CFA05F006F94EF21450C0F20E0029
:1054E00005F054FA40F6E4401AF056F9044645F245
:1054F000A65242F24B4340F20009C4F22C72C3F2AE
:10550000BE73C0F202098260E3603020C4F80090EC
:105510001AF042F9B6EE008A03466360204683ED36
:10552000008A0BF0B1FE6368204683ED018A0BF020
:10553000ABFE6368204683ED028A0BF0A5FE63682C
:10554000204683ED038A0BF09FFE6368204683EDBF
:10555000048A0BF099FE636846F26662C3F626720F
:105560005A6120460BF090FE63684FF07A529A61C0
:1055700020460BF089FE6368204683ED078A0BF016
:1055800083FE63684FF0010B84F810B0204683ED72
:10559000098A0BF079FE636848F20612C3F61562B9
:1055A0009A6220460BF070FE63684FF0000A2046B6
:1055B000C3F82CA00BF068FE04F6DC4245F26551FE
:1055C000C3F6046109F10C031160C4F8803C242384
:1055D00063612723A3612B2323652D236365302378
:1055E000C4F88C303323C4F890303723C4F8C83063
:1055F0003923C4F8CC303C23C4F804313F23C4F829
:1056000008314323C4F840314523C4F844314823CA
:10561000C4F87C314B23C4F880314F23C4F8B8312F
:105620005123C4F8BC315423C4F8F4315723C4F8CF
:10563000F8315B23C4F830325D23C4F83432602380
:10564000C4F86C3240F2E733C4F8703242F21C13F3
:10565000236241F23013636242F21D13236343F667
:105660007873636341F22733A36343F6797363640A
:1056700048F20573A36441F6FE03E761E36448F270
:105680000673A3654AF2A813E36540F662732366C6
:105690004AF2A913E3664BF2C023236740F2616329
:1056A00063674BF2C123C4F8803043F222324FF6D5
:1056B000BB636BF31F42C4F8843041F6C24141F230
:1056C0007D436BF31F41C4F88830C4F8AC204FF61B
:1056D000BC6340F69B0248F62307C4F894306BF392
:1056E0001F47C4F8A810C4F8B02041F6C14E43F2D9
:1056F000233348F624014CF249626BF31F4E6BF3DF
:105700001F436BF31F416BF31F42C4F8C0704FF48B
:10571000C757C4F898E0C4F8BC30C4F8C470C4F8E3
:10572000D010C4F8D4204CF24A6342F6D4024FF2AF
:10573000AD274FF2AE2E43F2F1216BF31F436BF313
:105740001F476BF31F4EC0F20201C4F8D82043F28A
:10575000F222C0F20202C4F8E430C4F8E870C4F8DF
:10576000F8E0C4F8FC1041F2614E40F61B4145F2EE
:105770001F5345F22057C0F20203C0F20207C4F8DB
:10578000ECE0C4F80011C4F80C214AF2334E4AF29E
:1057900034414FF2DE02C0F2020EC0F20201C0F24A
:1057A0000202C4F81031C4F8207141F2BC0340F683
:1057B000793740F64C7CC4F81431C4F824E1C4F8BD
:1057C0009C704FF2DF03C4F828C141F6367EC4F85E
:1057D0003C71C4F83411C4F8382141F6377745F2EA
:1057E000737145F27472C0F20203C0F2030EC0F28C
:1057F0000307C0F20301C0F20302C4F84831C4F841
:105800004CE1C4F85C7141F27C2EC4F86011C4F81C
:10581000702141F27D2149F249134CF6CB0740F645
:105820004742C0F20303C4F850E1C0F20307C4F8D2
:105830006411C0F2040249F24A1E4CF6CC01C0F2D7
:10584000030EC0F20301C4F87431C4F8887140F645
:10585000ED0341F20207C4F89C2141F20302C4F8AF
:105860007831C4F884E1C4F88C71C4F89811C4F894
:10587000A02140F6484344F68F6E44F6906747F601
:10588000903147F69132C0F20403C0F2040EC0F228
:105890000407C0F20401C0F20402C4F8AC31C4F839
:1058A000B0E1C4F8C07140F6196EC4F8C411C4F870
:1058B000D42140F68E114CF2F64340F6D81745F24B
:1058C000D92266F31F4766F31F42C0F20403C4F8EF
:1058D000B4E1C4F8C8114CF2F74E40F6D91166F3A2
:1058E0001F41C0F2040EC4F8D831C4F8EC7141F67F
:1058F000860340F6EB07C4F8002240F68122C4F884
:10590000DC31C4F8E8E1C4F8F071C4F8FC1145F2E8
:10591000DA23C4F8042249F26B4E49F26C474DF683
:10592000AD2C4DF6AE214DF6AE2266F31F4366F365
:105930001F4E66F31F4766F31F4166F31F4266F36F
:105940001F4C41F21216C4F81032C4F814E29D2321
:10595000C4F8186243F21D2E41F26946C0F20603F4
:10596000C0F2060EC4F82472C4F82C6245F2173750
:1059700047F20826C0F20607C0F20606C4F838123D
:10598000C4F84C229C2143F21E22C4F86032C4F8B1
:1059900064E245F2163341F2AA1EC0F20601C0F2DB
:1059A0000603C0F2060247F2A400C4F868E2C4F895
:1059B0009C7240F6790E40F6FB27C4F8A06240F6D0
:1059C0000216C4F83C12C4F85012C4F87832C4F875
:1059D0008C32C3F67D70C4F828C2C4F8A4E2C4F8BF
:1059E0004072C4F85472C4F87422C4F88822C4F80F
:1059F0007C62C4F89062234604F51C61C3F8D0A20F
:105A0000C3F8D402343399424FF00002F6D104F6C1
:105A1000C8410020C4F220300860002304F5496129
:105A200004F69847C4F87C3CC4F88C3C04F54B6001
:105A300004F6944304F6AC463A600A604FF07E5197
:105A400002603260204619600BF01EFC4BF220030E
:105A5000C1F6FF731C6004F03FFA0123C4F2020395
:105A60001B78D90740F114844FF0A052012312781B
:105A700088F80020C4F202031B78DA0740F104849E
:105A80000122C1F2004249F2A42343F6A054C2F21B
:105A90000004C1F6FF7312781A7002F0CDF8A06C02
:105AA000036847F61221DB69984743F2F15143F24C
:105AB00085420326C0F20101C0F2010243F23D30EB
:105AC00084F8646061602260C0F2010043F2D52373
:105AD00043F25D264DF6FD514DF6A952E060C0F24D
:105AE0000103C0F20106C0F20001C0F200024DF64F
:105AF0004D506361A6612161E261C0F200004DF684
:105B0000D1434DF675464DF625414DF6D53220620E
:105B1000C0F20003C0F20006C0F20001C0F20002B1
:105B20004DF68530A360A662E1622263C0F20000F8
:105B30004DF635334DF6E5264DF695214DF64522C9
:105B4000C0F20001C0F200026063C0F20003C0F2C4
:105B500000064EF22450A363E66300234FF6FF765F
:105B600021646264C0F20E0084F84C3084F84E3038
:105B700084F84D30A365636584F8E93084F86630B5
:105B800084F8653084F8673084F86830E665266606
:105B900004F0FCFE4DF21802C4F204024FF214139A
:105BA000C4F20F034FF4807111601A684FF20411B0
:105BB000C4F20F0142F0400240241A600A200C6037
:105BC0000EF01AF84FF45842C4F200024FF480432A
:105BD0001168C4F2060341F04051116019784FF486
:105BE000A042C4F2060241F002011970117848F295
:105BF0000403C4F2040341F0800111701A6842F0FA
:105C000002021A601A6847F20801C4F2040122F085
:105C100001021A600B6848F23002C4F2040243F435
:105C200000030B60116843F2040742F23806C4F225
:105C30000A0641F00E0142F2340442F23410C4F27A
:105C40000A0742F2A0031160C4F20A0384224FF053
:105C50004041C4F20A04C4F20A003A6031604FF4D1
:105C60004042012643F24101226006601A46196053
:105C70001368002BFCDA4FF40053C4F20A0300222D
:105C80001A600A200DF0B8FF4FF48A53C4F20A03D9
:105C900019461A6842F002021A600B689B07FCD48E
:105CA00042F63004C2F2010444F28050C2F2000015
:105CB00044F284514BF2F412C1F6FF722368066875
:105CC0002260C2F2000102F12C046B6341F6FC7306
:105CD000046002F5A67702F18C0402F1CC00C2F256
:105CE000010302F586722E660E68C5F880210F60EA
:105CF000C5F8C060C5F80041C5F8400103F1800156
:105D0000012243F8042F8B424FF00105F9D141F2F3
:105D100048204FF480720021C2F2010013F080F994
:105D200042F62803C2F2010341F2900C41F2A81E90
:105D30000024C4F20A0CC4F20A0E1C7041F248128C
:105D4000032341F2541041F24C11CCF80050C4F23C
:105D50000A02CEF80030C4F20A00C4F20A0142F28C
:105D60000003C2F2010341F258164FF48A5714603F
:105D7000C4F20A060360C4F20A070C6048F6153E36
:105D800041F28411C4F20A01C0F2080E3460C7F86F
:105D900000E00F6848F2006347F480570F60C1F6D7
:105DA000FF7346F6E901C0F201014EF208173668AA
:105DB0000068C3F8B411CEF2000704234FF000517D
:105DC000C0F2003339601360136843F012031360AC
:105DD000166843F6A063C2F200034DF6B91146F40B
:105DE0004026C0F200014EF205501660C0F20000DD
:105DF000C3F868114EF221274EF29D164EF2514122
:105E00004EF28D22C3F87001C0F20007C0F2000606
:105E1000C0F20001C0F200024EF28D00C3F87871AA
:105E2000C3F87C61C3F87411C3F88421C0F2000088
:105E30004EF225174EF201064DF6A9714DF6557238
:105E4000C3F88801C0F20007C0F20006C0F20001EA
:105E5000C0F200024DF60170C3F86C71C3F8906196
:105E6000C3F89411C3F89821C0F200004EF2516EAD
:105E70004DF6AD674DF665164DF611114DF6BD02A6
:105E8000C3F89C01C0F2000EC0F20001C0F2000293
:105E9000C0F20007C0F200064EF23C50C3F864E1C5
:105EA000C0F20E00C3F8A071C3F8A461C3F8A81132
:105EB000C3F8AC214BF2380604F068FDC1F6FF765A
:105EC0004DF6310EC0F2000E4BF23402C6F800E07F
:105ED000C1F6FF724DF2C16EC0F2000E4BF24000EF
:105EE000C2F800E0C1F6FF704DF2755EC0F2000E20
:105EF0004BF24801C0F800E0C1F6FF714DF24D4E83
:105F0000C0F2000E4BF24C03C1F800E0C1F6FF7383
:105F10004DF2C93EC0F2000E4BF24407C3F800E058
:105F2000C1F6FF774DF2B94EC0F2000E4BF29C164F
:105F3000C7F800E0C1F6FF7642F2595EC0F2010EEA
:105F40004BF25002C6F800E0C1F6FF7242F24D4E2D
:105F5000C0F2010E4BF23C00C2F800E0C1F6FF7047
:105F600042F2E54EC0F2010E4BF25401C0F800E0DF
:105F7000C1F6FF7142F2C13EC0F2010E4BF258036E
:105F8000C1F800E0C1F6FF7342F2693EC0F2010EB3
:105F90004BF25C07C3F800E0C1F6FF7742F2153E12
:105FA000C0F2010E4BF26006C7F800E0C1F6FF76C2
:105FB00042F2C127C0F201074BF264024BF26800C3
:105FC0003760C1F6FF72C1F6FF7042F26D2642F2F1
:105FD0001927C0F20106C0F201074BF26C014BF227
:105FE0007003C1F6FF71C1F6FF731660076042F2DD
:105FF000C51642F271124EF25C50C0F20102C0F2BC
:106000000106C0F20E001A600E6004F0BFFC4EF2F2
:106010008813CEF200031D6072B642F2E84742F2E6
:10602000EC43C2F20103C2F2010740F2002642F241
:1060300078402146C1F6FF76C2F2010070221E6050
:106040003C8012F0EDFF42F278402346C2F201009C
:106050005C0903F01F0150F8242005FA01F1013317
:106060000A43802B40F82420F2D140F20022C1F6EE
:10607000FF72002353800133802B02F58272F9D125
:1060800062B640F63070C2F201000AF0D9FD4FF45A
:10609000407211460E2004F0E7FD0E2004F0D6FCFD
:1060A00010F00C0F04D00C2200210E2004F0DCFDB7
:1060B00040F63074C2F201044FF6FF7243F63C41E1
:1060C000102004F0D1FDE288242122F010022046A5
:1060D00010F0E2FB44F240022221204610F0DCFBEB
:1060E000E288242122F48072204610F0D5FB41F68C
:1060F0001F7241F61D512E2004F0B6FD20460122EC
:106100004FF4807110F0C8FB20B1204670220A21A4
:1061100010F0C2FB032202214FF4847004F0A4FDAE
:10612000012211464FF4927004F09EFD01221146A7
:106130004FF4827004F098FD4EF27850C0F20E00D9
:1061400004F024FC42F2744042F2EA41C2F201003F
:1061500042F27642C2F20102C2F2010142F2F0437F
:106160004EF20814C2F20103008809881080CEF2B2
:10617000000401254EF294501980C0F20E002560F3
:1061800011F0AEFD00220A21802011F0B3FD4EF285
:10619000AC50C0F20E0011F0A3FD00220A2140F61F
:1061A000553011F0A7FD4EF2C050C0F20E0004F0C1
:1061B000EDFB40F60853C2F201034BF2803200249B
:1061C000C1F6FF724FF400694FF4806721469C844A
:1061D0001A62A3F826901F8510464FF4805212F0E1
:1061E0001FFF40F63453C2F201034CF28036C1F671
:1061F000FF762146A3F826909C841F851E623046B8
:106200004FF4805212F00CFF40F66053C2F20103CB
:1062100040F6584140F6904247F64846C2F2010126
:10622000C2F2010265F31F464FF480351C62DE6145
:106230005C869C865D6298F8000015629461D4616A
:106240008C61CC610D6211F05BFF4EF2C450C0F264
:106250000E0004F09BFB04F045FA11F093FE4DF2A2
:106260007442C1F6FF7240F6487312681192C2F28E
:106270000103119A1A6013B0BDEC028BBDE8F08FD8
:106280000CF030FEFFF7DAB80CF02CFEFFF7F8BB8D
:106290000CF028FEFFF7E8BB2DE9F04F4DF28036F9
:1062A000C1F6FF76304642F20303C3F6000349F21B
:1062B000A02246F6650189B040F8043BC1F6FF72A2
:1062C000C0F2010112F072FE49F2A02246F6650109
:1062D000C1F6FF72C0F2010106F10C0012F066FE79
:1062E00049F2A02246F66501C1F6FF72C0F2010133
:1062F00006F1140012F05AFE49F2A02246F665019A
:10630000C1F6FF72C0F2010106F11C0012F04EFE50
:1063100049F2A02246F66501C1F6FF72C0F2010102
:1063200006F1240012F042FE49F2A02246F6650171
:10633000C1F6FF72C0F2010106F12C0012F036FE28
:1063400049F2A02246F66501C1F6FF72C0F20101D2
:1063500006F1340012F02AFE49F2A02246F6650149
:10636000C1F6FF72C0F2010106F13C0012F01EFE00
:1063700049F2A02246F66501C1F6FF72C0F20101A2
:1063800006F1440012F012FE49F2A02246F6650121
:10639000C1F6FF72C0F2010106F14C0012F006FED8
:1063A00049F2A02246F66501C1F6FF72C0F2010172
:1063B00006F1540012F0FAFD49F2A02246F66501FA
:1063C000C1F6FF72C0F2010106F15C0012F0EEFDB1
:1063D00049F2A02246F66501C1F6FF72C0F2010142
:1063E00006F1640012F0E2FD49F2A02246F66501D2
:1063F000C1F6FF72C0F2010106F16C0012F0D6FD89
:1064000049F2A02246F66501C1F6FF72C0F2010111
:1064100006F1740012F0CAFD49F2A02246F66501A9
:10642000C1F6FF72C0F2010106F17C004EF2D857AE
:106430000024C0F20E0712F0B9FD10250CF052FD39
:106440000223272286F890304FF0604886F8892092
:1064500003211A4686F88F50C6F884706FF06045A5
:1064600006F1940086F8884086F88E4086F89140C0
:1064700002F09EFD1D221C21C6F8A880C6F8AC5073
:1064800006F1B40086F8B04002F092FDD6F8F43080
:10649000079334230799C6F8C8801422C4F2FE3348
:1064A000C6F8D410C6F8D820C6F8CC5086F8D0402C
:1064B000C6F8DC4093F80052D6F8F430069340F664
:1064C0004C03069986F8E0500420C4F2FE33C6F867
:1064D000E82086F8E100C6F8E410C6F8EC4093F82E
:1064E0000032D6F8F42005924FF01E0E86F8F1E047
:1064F000059D86F8F030224607F11003012106F1D0
:10650000FC00C6F8F85011F017FF012207F11C0338
:10651000114606F5E07011F00FFF012207F1280384
:10652000114606F5217011F007FF012207F1300333
:10653000114606F5527011F0FFFE012207F13C03EF
:10654000114606F20C4011F0F7FE012207F1440358
:10655000114606F59A6006F1840911F0EDFE07F187
:106560004C032246012106F5BF6086F8E44586F813
:10657000E54586F8E74586F8F44586F8F545C6F81A
:10658000E89511F0D9FE49F2A421C1F6FF7106F297
:10659000BC6006F00DF807F158032246012106F20F
:1065A000E470C6F8D49786F8D04786F8D14786F8C5
:1065B000D34786F8E04786F8E14711F0BDFE012297
:1065C00007F16003114606F6A80011F0B5FE01229E
:1065D00007F16803114606F66C1011F0ADFE0122BA
:1065E00007F17403114606F5236011F0A5FE0122A0
:1065F00007F17C03114606F6F42011F09DFE0122FE
:1066000007F18C03114606F6B83011F095FE012211
:1066100007F19803114606F67C4011F08DFE012229
:1066200007F1A003114606F5546011F085FE012222
:1066300007F1A803114606F6046011F07DFE07F18C
:10664000B8032246012106F62C704EF27845C6F8B2
:106650001C9F86F8184F86F8194F86F81B4F86F84E
:10666000284F86F8294F11F067FE49F2AC21C1F698
:10667000FF75C1F6FF7106F57F6005F099FF07F120
:10668000C003224605F120000121C5F810902C73AB
:106690006C73EC732C776C7711F04EFE49F2AD21E0
:1066A00005F1E400C1F6FF7105F082FF07F1C803B0
:1066B000224605F503700121C5F8FC9185F8F841E3
:1066C00085F8F94185F8FB4185F8084285F80942CB
:1066D00011F032FE49F2AE2105F53470C1F6FF71BA
:1066E00005F066FF07F1D403224605F57E7001210F
:1066F000C5F8E89385F8E44385F8E54385F8E74372
:1067000085F8F44385F8F54311F016FE49F2AF2100
:1067100005F2BC40C1F6FF7105F04AFF07F1DC034A
:10672000224605F2E4500121C5F8D49585F8D045FC
:1067300085F8D14585F8D34585F8E04585F8E145EC
:1067400011F0FAFD49F2B02105F5D560C1F6FF71EF
:1067500005F058FF07F1E403224605F5FA60012130
:10676000C5F8C09785F8BC4785F8BD4785F8BF4791
:1067700085F8CC4785F8CD4711F0DEFD49F2B1210F
:1067800005F69400C1F6FF7105F03CFF07F1F00338
:10679000224605F6BC100121C5F8AC9985F8A84938
:1067A00085F8A94985F8AB4985F8B84985F8B9490C
:1067B00011F0C2FD45F2E11105F52860C0F20101BA
:1067C00005F04AFF07F1F803224605F6A83001213B
:1067D000C5F8989B85F8944B85F8954B85F8974BB1
:1067E00085F8A44B85F8A54B11F0A6FD49F2B3211D
:1067F00005F66C40C1F6FF7105F0DAFE07F580730F
:10680000224605F694500121C5F8849D85F8804DF7
:1068100085F8814D85F8834D85F8904D85F8914D2B
:1068200011F08AFD49F2B42105F65860C1F6FF71F6
:1068300005F0BEFE4FF2705A07F5887305F57860D3
:1068400022460121C1F6FF7AC5F8709F85F86C4F8A
:1068500085F86D4F85F86F4F85F87C4F85F87D4F33
:1068600011F06AFD012207F590731146AAF1B400F8
:1068700011F062FD012207F5987311460AF110002C
:1068800011F05AFD012207F59E7311460AF1D4005A
:1068900011F052FD012207F5A47311460AF5CC70E0
:1068A00011F04AFD012207F5AC7311460AF5177085
:1068B00011F042FD012207F5B27311460AF5487046
:1068C00011F03AFD012207F5BA7311460AF5797005
:1068D00011F032FD012207F5C27311460AF59560E9
:1068E00011F02AFD012207F5C87311460AF26C5017
:1068F00011F022FD012207F5D07311460AF5C6609A
:1069000011F01AFD012207F5D87311460AF2F4605E
:1069100011F012FD012207F5DE7311460AF5F7604A
:1069200011F00AFD012207F5E67311460AF67C0014
:1069300011F002FD012207F5EE7311460AF514600D
:1069400011F0FAFC012207F5F67311460AF604204D
:1069500011F0F2FC012207F5FE7311460AF6C82079
:1069600011F0EAFC012207F5037311460AF68C3098
:1069700011F0E2FC012207F5077311460AF54560A4
:1069800011F0DAFC012207F5097311460AF61450DA
:1069900011F0D2FC07F50C73224601210AF63C6087
:1069A000CAF82C9E8AF8284E8AF8294E8AF82B4E6F
:1069B0008AF8384E8AF8394E11F0BEFC49F2B521FA
:1069C000C1F6FF710AF5706005F0F2FD40F26868EB
:1069D00041F2140341F2150241F21701C2F200081C
:1069E000A8F1D0000AF803400AF8024007F5107336
:1069F00022460AF80140012148F8E09C08F8D44CEE
:106A000008F8D34C11F098FC49F2B621A8F10C001B
:106A1000C1F6FF7105F0CCFD07F51473224608F5A9
:106A20008E700121C8F80C9188F8084188F8094156
:106A300088F80B4188F8184188F8194111F07CFC5E
:106A400049F2B72108F5F070C1F6FF7105F0B0FD0D
:106A500007F51773224608F542700121C8F8F8922D
:106A600088F8F44288F8F54288F8F74288F8044339
:106A700088F8054311F060FC44F6ED6108F5737089
:106A8000C0F2010105F0E8FD07F51A73224608F28D
:106A9000F4400121C8F8E49488F8E04488F8E1441F
:106AA00088F8E34488F8F04488F8F14411F044FC95
:106AB00044F6CD6108F5B760C0F2010105F0CCFDE8
:106AC00007F51E73224608F5DC600121C8F8D09650
:106AD00088F8CC4688F8CD4688F8CF4688F8DC465A
:106AE00088F8DD4611F028FC44F6AD6108F2A47088
:106AF000C0F2010105F0B0FD07F52173224608F64A
:106B0000CC000121C8F8BC9888F8B84888F8B94882
:106B100088F8BB4888F8C84888F8C94811F00CFCC8
:106B200045F2912108F51960C0F2010105F094FDCC
:106B300007F52573224608F6B8200121C8F8A89A5F
:106B400088F8A44A88F8A54A88F8A74A88F8B44A79
:106B500088F8B54A11F0F0FB45F24D2108F67C307B
:106B6000C0F2010105F078FD07F52973224608F609
:106B7000A4400121C8F8949C88F8904C88F8914C66
:106B800088F8934C88F8A04C88F8A14C11F0D4FBFD
:106B900045F2092108F66850C0F2010105F05CFDDC
:106BA00007F52C73224608F569600121C8F8809E1C
:106BB00088F87C4E88F87D4E88F87F4E88F88C4E99
:106BC00088F88D4E41F2607511F0B6FB49F2BE2196
:106BD000C2F2000508F65470C1F6FF7105F0E8FC3A
:106BE00007F530732246A5F17C00012145F88C9C05
:106BF00005F8904C05F88F4C05F88D4C05F8804C45
:106C000005F87F4C11F098FB49F2BF2105F14800CF
:106C1000C1F6FF7105F0CCFC07F53473224605F58B
:106C2000B8700121C5F8609185F85C4185F85D4137
:106C300085F85F4185F86C4185F86D4111F07CFB6A
:106C400049F2C02105F50D70C1F6FF7105F0B0FCE9
:106C500007F53873224605F557700121C5F84C93A6
:106C600085F8484385F8494385F84B4385F85843F0
:106C700085F8594311F060FB49F2C12105F58460A4
:106C8000C1F6FF7105F094FC07F53C73224605F54B
:106C9000A9600121C5F8389585F8344585F8354552
:106CA00085F8374585F8444585F8454511F044FB9E
:106CB00049F2C22105F20C60C1F6FF7105F078FCC3
:106CC00007F54073224605F234700121C5F8249778
:106CD00085F8204785F8214785F8234785F8304710
:106CE00085F8314711F028FB49F2C32105F5FF6013
:106CF000C1F6FF7105F05CFC07F54473224605F50B
:106D000012600121C5F8109985F80C4985F80D49E4
:106D100085F80F4985F81C4985F81D4911F00CFBD1
:106D200049F2C42105F6E410C1F6FF7105F040FCFC
:106D300007F54873224605F60C300121C5F8FC9A88
:106D400085F8F84A85F8F94A85F8FB4A85F8084B32
:106D500085F8094B11F0F0FA49F2C52105F53D60BF
:106D6000C1F6FF7105F024FC07F54C73224605F6C9
:106D7000F8400121C5F8E89C85F8E44C85F8E54C1D
:106D800085F8E74C85F8F44C85F8F54C11F0D4FA09
:106D900049F2C62105F6BC50C1F6FF7105F008FCAA
:106DA00007F55073224605F6E4600121C5F8D49E2C
:106DB00085F8D04E85F8D14E85F8D34E85F8E04E53
:106DC00085F8E14E42F6580811F0B6FA49F2C721AB
:106DD000C2F2000805F6A870C1F6FF7105F012FCBA
:106DE00007F5527322460121A8F1280048F8389C83
:106DF00008F83C4C08F83B4C08F8394C08F82C4C87
:106E000008F82B4C11F098FA49F2C821C1F6FF712D
:106E100008F19C0005F0F6FB07F5557322460121A9
:106E200008F5E270C8F8B49188F8B04188F8B1412B
:106E300088F8B34188F8C04188F8C14111F07CFA64
:106E400049F2A421C1F6FF7108F5227005F0B0FBEC
:106E500007F558732246012108F56C70C8F8A09315
:106E600088F89C4388F89D4388F89F4388F8AC4392
:106E700088F8AD4311F060FA012207F55B73114603
:106E800008F2744011F058FA012207F55F731146B9
:106E900008F5A76011F050FA012207F56373114657
:106EA00008F2FC5011F048FA07F5677322460121F9
:106EB00008F22470C8F8149788F8104788F811472A
:106EC00088F8134788F8204788F8214711F034FAEA
:106ED00049F2C921C1F6FF7108F5FD6005F068FBB4
:106EE00007F56A732246012108F51160C8F8009978
:106EF00088F8FC4888F8FD4888F8FF4888F80C496D
:106F000088F80D4911F018FA45F2DD21C0F20101AF
:106F100008F6D41005F0A0FB07F56E732246012198
:106F200008F6FC20C8F8EC9A88F8E84A88F8E94A9C
:106F300088F8EB4A88F8F84A88F8F94A11F0FCF921
:106F400044F66561C0F2010108F53C6005F084FB80
:106F500007F572732246012108F6E840C8F8D89C6C
:106F600088F8D44C88F8D54C88F8D74C88F8E44C8D
:106F700088F8E54C11F0E0F949F2CC21C1F6FF7137
:106F800008F6AC5005F014FB43F6501507F5767380
:106F90002246214608F6D460C2F20005C8F8C49E15
:106FA00088F8C04E88F8C14E88F8C34E88F8D04E95
:106FB00088F8D14E11F0C0F907F57A732146012205
:106FC00008F6987011F0B8F907F57C732246012194
:106FD000A5F1380045F8489C05F84C4C05F84B4C99
:106FE00005F8494C05F83C4C05F83B4C11F0A4F968
:106FF00049F2D021C1F6FF7105F18C0005F0D8FAF5
:1070000007F580632246012105F5DA70C5F8A491E1
:1070100085F8A04185F8A14185F8A34185F8B041E4
:1070200085F8B14111F088F944F62161C0F20101FF
:1070300005F51E7005F010FB95F8B43485F8B544DD
:10704000012249F2D42E43F0010362F34703C1F653
:10705000FF7E4FF6FF772146802205F2B94085F882
:10706000B64485F8B74485F8B84485F8394585F8BD
:10707000B434C5F898E4C5F8AC74C5F8B074C5F874
:10708000909385F88C4385F88D4385F88F4385F878
:107090009C4385F89D4385F84C4485F84D4485F81C
:1070A0009C4485F89D4485F89E44C5F8A444C5F8E1
:1070B000A84411F0B5FF49F2A02247F68171C1F64C
:1070C000FF72C0F2010105F58A60C5F85044C5F8A9
:1070D0005444C5F85844C5F85C44C5F86044C5F844
:1070E0006444C5F86844C5F86C44C5F87044C5F8F4
:1070F0007444C5F87844C5F87C44C5F88044C5F8A4
:107100008444C5F88844C5F88C44C5F89044C5F853
:10711000944411F04BFF4EF6EC13C0F20E0305F64B
:10712000282005F6682105F6A822C5F85035C5F8CF
:10713000640505F6E8234020C5F86815C5F86C25F8
:107140005021C5F8743505F5EE62D5F8303CA5F848
:107150007A0505F5FA6005F5E267A5F87C15C5F82E
:10716000103705F5036105F50763C5F8D027C5F8A5
:10717000300C05F50F62D5F8340CC5F87077C5F8FA
:107180003008C5F87018C5F8B03805F51B61C5F8AA
:10719000302905F50B6CD5F8382CC5F8341C05F5ED
:1071A000136705F5176005F51F63C5F8F029C5F8E5
:1071B000B446C5F8B846C5F8BC46C5F8C046C5F8DB
:1071C000C446C5F8C846C5F8CC46C5F8D046C5F88B
:1071D000F0C8C5F87079C5F8B009C5F8383CC5F8ED
:1071E000D446D5F83C2CC5F8D84605F5AA61C5F8B3
:1071F000DC46C5F8E046C5F8E446C5F8E846C5F8FB
:10720000EC46C5F8F046C5F8F446C5F8F846C5F8AA
:10721000FC46C5F80047A5F87E45A5F88045C5F8A9
:107220005C45C5F86045C5F85845C5F8544512B9E0
:1072300000F0E3BC1A465368002BFBD1516044F2C6
:107240009058C2F2000800224EF6EC191746C0F220
:107250000E091146404609F11C04C5F8509501F08D
:10726000F7FE3A46394608F1A00085F8DC7CC5F8FF
:10727000404CC5F8D87C85F8DD7C01F0E9FE08F5C6
:10728000AC7208F5A070012185F87C7D09F1280B0E
:10729000C5F8E04CC5F8787D85F87D7D4FF4004A4F
:1072A00001F0D6FE08F5BE7247F6FF73012108F51E
:1072B000B270C5F880BDA5F89E3D0193A5F8A0ADBC
:1072C00040F2F04401F0C4FE019BA5F8C23D08F570
:1072D000C470C2F20104C5F8A4BDA5F8C4AD05F0A0
:1072E00017FA4AF6B81004F5ED6BC2F2000005F08B
:1072F0000FFA04F5F2625846042101F0A9FE4FF49A
:10730000803A09F1340504F5F96204F5F4600421CA
:10731000C4F86857C4F880A7C4F884A7C4F888A73D
:10732000C4F88CA701F094FE04F2F47204F5FB603B
:107330000121C4F8A057C4F8B8A709F14005C4F862
:10734000BCA7C4F8C0A7C4F8C4A701F081FE04F626
:10735000140204F5FF600121C4F8F0A7C4F8D8575F
:1073600001F076FE04F5036204F618000221C4F869
:1073700010A8C4F8F85704F5076A01F069FE09F18E
:107380004C0504F65C0204F644000221C4F81858C7
:1073900001F05EFE3A4639465046C4F8445801F0C2
:1073A00057FE09F158024FF0804308F5A07104F62A
:1073B000A800C4F89838C4F8AC18C4F8A888C4F871
:1073C0007028C4F88878C4F88C78C4F89078C4F829
:1073D0009478C4F89C78A4F8A078A4F8A278A4F8CB
:1073E000A47884F8B07884F8B178C4F8B47884F8D4
:1073F000B87805F05BF949F2A02248F25D71C1F658
:10740000FF72C0F2000104F6A80011F0CFFD08F5EC
:10741000B27304F6BC00C4F8C03808F1A003C4F885
:10742000BC3884F8C47884F8C578C4F8C87884F87F
:10743000CC7805F03BF949F2A02248F25D71C1F623
:10744000FF72C0F2000104F6BC0011F0AFFD08F5B8
:10745000C47304F50D60C4F8D438C4F8D08884F837
:10746000D87884F8D978C4F8DC7884F8E07805F026
:107470001DF949F2A02248F25D71C1F6FF72C0F217
:10748000000104F50D6011F091FD08F1A003C4F8AE
:10749000E4384AF6B813C2F2000304F6E400C4F874
:1074A000E83884F8EC7884F8ED78C4F8F07884F85B
:1074B000F47805F0FBF849F2A02248F25D71C1F6BC
:1074C000FF72C0F2000104F6E40011F06FFD04F653
:1074D000F800A0F1E003C4F8FC38C4F8F88884F898
:1074E000007984F80179C4F8047984F8087905F002
:1074F000DDF849F2A02248F25D71C1F6FF72C0F2D8
:10750000000104F6F80011F051FD04F60C10A0F192
:10751000C803C4F8103908F1A003C4F80C3984F882
:10752000147984F81579C4F8187984F81C7905F071
:10753000BDF849F2A02248F25D71C1F6FF72C0F2B7
:10754000000104F60C1011F031FD04F51260012564
:10755000A0F58473C4F82439C4F820A984F82879E4
:10756000C4F82C7984F8307984F8295905F09EF80C
:1075700049F2A02248F25D71C1F6FF72C0F200012B
:1075800004F5126011F012FD04F63410A0F1F003BE
:10759000C4F83839C4F834A984F83C7984F83D59E2
:1075A000C4F8407984F8447905F080F849F2A022C3
:1075B00048F25D71C1F6FF72C0F2000104F63410AA
:1075C00011F0F4FC04F64810C4F84889C4F84CB92A
:1075D00084F8507984F85179C4F8547984F858794A
:1075E00005F064F849F2A02248F25D71C1F6FF721D
:1075F000C0F2000104F6481011F0D8FC04F65C104B
:1076000008F1A003C4F85C39A0F5DE73C4F8603952
:1076100084F8647984F86579C4F8687984F86C79B9
:1076200005F044F849F2A02248F25D71C1F6FF72FC
:10763000C0F2000104F65C1011F0B8FC04F517600C
:10764000A0F5AC734FF00208C4F87039C4F874B9EF
:1076500084F87879C4F87C7984F8807984F8798919
:1076600005F024F849F2A02248F25D71C1F6FF72DC
:10767000C0F2000104F5176011F098FC04F68410C4
:10768000A0F5A073C4F88439A0F5F273C4F8883962
:1076900084F88C7984F88D89C4F8907984F8947989
:1076A00005F004F849F2A02248F25D71C1F6FF72BC
:1076B000C0F2000104F6841011F078FC44F2187353
:1076C000C2F2000304F69810C4F89839C4F89CB9C3
:1076D00084F8A07984F8A159C4F8A47984F8A87929
:1076E00004F0E4FF49F2A02248F25D71C1F6FF7296
:1076F000C0F2000104F6981011F058FC4AF6B813D5
:1077000004F6AC10C2F20003C4F8AC39A0F5037360
:10771000C4F8B03984F8B47984F8B559C4F8B879A4
:1077200084F8BC7904F0C2FF49F2A02248F25D71EE
:10773000C1F6FF72C0F2000104F6AC1011F036FC85
:1077400004F51C60A0F5F473C4F8C439C4F8C0B9DA
:1077500084F8C87984F8C979C4F8CC7984F8D079E8
:1077600004F0A4FF49F2A02248F25D71C1F6FF7255
:10777000C0F2000104F51C6011F018FC04F6D410EE
:10778000A0F50D73C4F8D439A0F5EE73C4F8D83958
:1077900084F8DC7984F8DD79C4F8E07984F8E47958
:1077A00004F084FF49F2A02248F25D7104F6D4107F
:1077B000C1F6FF72C0F2000111F0F8FB04F520627F
:1077C00004F6E810414601F043FC09F16403C4F8F3
:1077D000E83972B6B4F8083A13EA050200F01282EA
:1077E0009F0740F1C5815D0740F10E82180740F107
:1077F0000D82D90640F10C829A0640F10B825F0699
:1078000040F10A821D0640F10982D80540F1088244
:10781000990540F107825A0540F106821F0540F1A3
:107820000582DD0440F10482980440F1038259048A
:1078300040F19D81DA0B08BF0F2500F0998162B6F7
:1078400000221023F26286F8303048F23C03C4F282
:10785000040348F2400219680020C4F2040241F413
:107860000041C4F80C0AC4F8100A1960116841F00C
:10787000020111601A684FF4704142F00202C4F232
:1078800002011A600B6883427EDB4FF28003C4F270
:1078900002031B68834277DB4FF47142C4F2020299
:1078A0004FF0804313601368002BFCDB4FF204158C
:1078B000C4F202054FF26003C4F202034FF2FE0E5F
:1078C0004FF20400C5F800E0C4F202004FF0000ED1
:1078D000C3F800E04FF2080101230360C4F2020183
:1078E00018464FF20C07C4F20207C0F2007008609D
:1078F0004FF210024FF480303860C4F2020241F6B9
:107900001B7763F31F474FF214054FF2E001176036
:10791000C4F20205C4F202014FF4F852C1F61F721C
:107920004FF284072A60C4F20207C1F800E04FF268
:1079300088054FF28C01C4F20205C4F2020141F63F
:107940001B7C3B6063F31F4CC4F200732B604FF24F
:10795000900E08604FF294074BF208054BF20C00B2
:107960004BF21801C4F2020EC4F20207C4F204057D
:10797000C4F20400C4F204014FF4C063CEF800C0A6
:107980003A602B6003600B604BF20402C4F2040205
:10799000F36A94F8145A4FF4C061116002229A807D
:1079A0009A6048F200404FF22202C4F20202C1F68D
:1079B000FF7018601A6140F20112DA804FF47E42C3
:1079C00096F83010CFF6FF72DA604FF48072DA82E8
:1079D00001F18041DA8306229A8301F50431002205
:1079E0009A829A618D230A700B7040F2F043C2F2C2
:1079F000010375B94EF24041CEF200014EF2081279
:107A0000CEF20002D0250D70012111600A4683F8E4
:107A1000141A48F21B05C4F200054FF4704196F8A1
:107A2000303084F8152AC4F202012B704FF08075B3
:107A30000D605A110125C9F2000592000D6000EB9E
:107A4000830040F6D86702F1604246F2B101C2F20B
:107A5000010702F561424FF00108C0F2010103F095
:107A60001F03C0F8401208FA03F307F13000136057
:107A70000025A0F51073C4F8183AC4F81C7A84F8ED
:107A8000205A84F8215AC4F8245A84F8285A04F059
:107A90000DFE49F2A02248F25D71C1F6FF72C0F2FC
:107AA000000107F1300011F081FA07F14400A0F560
:107AB0000D73C4F82C3A84F8358AC4F8307A84F807
:107AC000345AC4F8385A84F83C5A04F0EFFD49F2AD
:107AD000A02248F25D7107F14400C1F6FF72C0F2C6
:107AE000000111F063FA4EF65C23C0F20E03C4F8F5
:107AF000403A0A2384F8483A72B64EF218034EF61A
:107B00000451CEF20001CEF200031B68D6F8F40057
:107B10000A6862B6520102D5322B88BF4044D6F8BB
:107B2000F4200492049FD6F8F4200392C3F52F3377
:107B300003F21F3346F61741039DD6F8F460029610
:107B4000C1F2C1619B084FF47A7202FB00F2A1FB03
:107B5000031302EB9303029AC4F84C3AC4F8507A28
:107B6000C4F8545AC4F8582A09B0BDE8F08F0E255D
:107B70000122AA401343A4F8083A62B648F240032F
:107B8000E9B2C4F2040386F83010186848F23C02E7
:107B9000C4F2040240F00200186010684FF4004E76
:107BA00040F0020005F10075C4F2000E106005F50A
:107BB000906540F2824048F21A0748F21E02CEF861
:107BC00000006B01C4F20002C4F2000748F218057D
:107BD00048F21F00C4F20005C4F2000039701170B1
:107BE000002229700170F3625A601A609A60DA60AC
:107BF0001A615A619A61DA6127E62B46C3F83C1C88
:107C0000FFF71DBB1546B3E74546B1E70325AFE7D0
:107C10000425ADE70525ABE70625A9E70725A7E776
:107C20000825A5E70925A3E70A25A1E70B259FE776
:107C30000C259DE70D259BE72DE9F04149F2A42590
:107C4000C1F6FF754FF6BC109AB00B21C0F20100CF
:107C50000FF064FB00220A21287810F04BF802F0A4
:107C600041FD0123C4F202032C781B78DE0740F1AA
:107C70009D830123C1F200431B789C422ED0012337
:107C8000C4F202031B78D80740F169830123C1F2D3
:107C900000431B789C4221D04EF20302C4F207023B
:107CA0001378802B00F070830022C4F20202137854
:107CB00013F0700340F051830123C1F2004301220D
:107CC0001C70C4F202021378D907FCD54EF20302ED
:107CD000C4F207021378012B00F044832F78013F90
:107CE00007EB8707FF004FF00108BC1CC4F2020835
:107CF0002A370DF1FF360DE098F80030DB0740F130
:107D0000F58204F1A05301341B78BC42DBB206F8C3
:107D1000013F08D0B4F5805FEED301340023BC42AC
:107D200006F8013FF6D14EF6D044C0F20E040FCC57
:107D30000AAE37460FC70FCC0FC70FCC0FC794E85A
:107D40000F004FF0FF3487E80F0001A911F8013B45
:107D500083EA04021AA802F00F0200EB8202B14289
:107D600052F8402C82EA141484EA131303F00F0330
:107D700000EB830353F8403C83EA14146FEA0404D5
:107D8000E4D14EF610500E21C0F20E000FF0C6FAEC
:107D900000220A2128780FF0ADFF4EF6205008216E
:107DA000C0F20E000FF0BAFA2B78013B03EB83030D
:107DB000D8000022102102300FF09CFF4EF62C500C
:107DC0001421C0F20E000FF0A9FA009F002210212A
:107DD00038460FF08FFF4EF644500521C0F20E00DA
:107DE0000FF09CFA00221021204649F2A4260FF041
:107DF00081FFA742C1F6FF7600F07B824EF6545019
:107E0000C0F20E0002F0C2FD02F066F80123C4F2D7
:107E1000020334781B78D90740F19C820123C1F218
:107E200000431B789C422ED00123C4F202031B782E
:107E3000DA0740F1BE820123C1F200431B789C4265
:107E400021D04EF20302C4F207021378802B00F017
:107E5000C5820022C4F20202137813F0700300D02E
:107E600013700123C1F2004301221C70C4F202020C
:107E70001378DB07FCD54EF20302C4F20702137835
:107E8000012B00F099824EF684500F21C0F20E00B3
:107E90000FF044FA49F2D023C1F6FF73002218789C
:107EA0000A210FF027FF02F01DFC4EF69450072127
:107EB000C0F20E000FF032FA49F2A82400220A2183
:107EC0002878C1F6FF740FF015FF02F00BFC4EF698
:107ED0009C500C21C0F20E000FF020FA002210215D
:107EE00020680FF007FF02F0FDFB4EF6AC500721B3
:107EF000C0F20E000FF012FA00220A2120790FF0D2
:107F0000F9FE02F0EFFB4EF6B4500921C0F20E006C
:107F10000FF004FA00220A2160790FF0EBFE02F064
:107F2000E1FB4EF6C0500A21C0F20E000FF0F6F948
:107F300000220A21A0790FF0DDFE02F0D3FB4EF6FD
:107F4000CC500821C0F20E000FF0E8F900220A21FF
:107F5000E0790FF0CFFE02F0C5FB4EF6D8500821B5
:107F6000C0F20E000FF0DAF994F908000028B6BF4D
:107F70002D22002240420A210FF0BCFE02F0B2FB8B
:107F80004EF6E4500B21C0F20E000FF0C7F994F941
:107F900009000028B6BF2D22002240420A210FF01E
:107FA000A9FE02F09FFB4EF6F0500621C0F20E0033
:107FB0000FF0B4F994F90A000028B6BF2D22002270
:107FC00040420A210FF096FE02F08CFB4EF6F8506C
:107FD0000821C0F20E000FF0A1F900220A21E07A78
:107FE0000FF088FE02F07EFB4EF604601021C0F216
:107FF0000E000FF093F900220A21207B0FF07AFE89
:1080000002F070FB4EF618601721C0F20E000FF060
:1080100085F900220A21607B0FF06CFE02F062FB02
:108020004EF630601321C0F20E000FF077F90022F7
:108030000A21A07B0FF05EFE02F054FB4EF6446076
:108040000A21C0F20E000FF069F900220A21E07B3C
:108050000FF050FE02F046FB4EF650601121C0F2C8
:108060000E000FF05BF900220A21207C0FF042FE87
:1080700002F038FB4EF664601421C0F20E000FF0DF
:108080004DF900220A21607C0FF034FE02F02AFB39
:108090004EF67C601221C0F20E000FF03FF9002274
:1080A0000A21A07C0FF026FE02F01CFB4EF6906029
:1080B0001621C0F20E000FF031F900220A21E07CF7
:1080C0000FF018FE02F00EFB4EF6A8601321C0F26E
:1080D0000E000FF023F900220A21207D0FF00AFE86
:1080E00002F000FB4EF6BC601221C0F20E000FF051
:1080F00015F900220A21607D0FF0FCFD02F0F2FA72
:108100004EF6D0601121C0F20E000FF007F90022E8
:108110000A21A07D0FF0EEFD02F0E4FA4EF6E460D5
:108120001021C0F20E000FF0F9F800220A21E07DC4
:108130000FF0E0FD02F0D6FA4EF6F8600E21C0F224
:108140000E000FF0EBF800220A21207E0FF0D2FD86
:1081500002F0C8FA4EF608701221C0F20E000FF0BD
:10816000DDF800220A21607E0FF0C4FD02F0BAFAA9
:108170004EF61C700E21C0F20E000FF0CFF8002258
:108180000A21A07E0FF0B6FD02F0ACFA4EF62C707C
:108190001221C0F20E000FF0C1F800220A21E07E89
:1081A0000FF0A8FD02F09EFA4EF640700E21C0F2CC
:1081B0000E000FF0B3F800220A21207F0FF09AFD85
:1081C00002F090FA4EF650701021C0F20E000FF03F
:1081D000A5F800220A21607F0FF08CFD02F082FAE0
:1081E0004EF664701121C0F20E000FF097F80022D5
:1081F0000A21A07F0FF07EFD02F074FA4EF678702F
:108200000921C0F20E000FF089F894F91F00002830
:10821000B6BF2D22002240420A210FF06BFD02F072
:1082200061FA4EF684700B21C0F20E000FF076F862
:1082300094F920000028B6BF2D22002240420A21D6
:108240000FF058FD02F04EFA4EF690700A21C0F27F
:108250000E000FF063F800220A2194F821000FF0BD
:1082600049FD02F03FFA4EF69C700E21C0F20E005E
:108270000FF054F800220A2194F822000FF03AFD82
:1082800002F030FA4EF6AC701021C0F20E000FF082
:1082900045F800220A2194F823000FF02BFD02F08C
:1082A00021FA4EF6C0701321C0F20E000FF036F81E
:1082B00000220A2194F824000FF01CFD02F012FAAB
:1082C0004EF6D4700A21C0F20E000FF027F894F990
:1082D00025000028BABF40422D2200220A210FF0BB
:1082E00009FD1AB0BDE8F04102F0FCB90AF0FAFD50
:1082F00007E53778013F07EB8707FF0049F2A7261C
:108300004FF00108BC1CC1F6FF762A37C4F2020800
:108310000CE098F80030D80719D504F1A0530134C7
:108320001B78BC42DBB206F8013F08D0B4F5805F91
:10833000EFD301340023BC4206F8013FF6D14EF6DC
:108340004C500521C0F20E000EF0E8FF9BE50AF04C
:10835000C9FDE2E70AF0C6FD60E51370ACE40AF07F
:10836000C1FD93E44EF20103C4F2070360211970CA
:108370001378802BFCD148F24403C4F2040300229A
:10838000C0F206221A60A9E448F244014EF2010349
:10839000C4F204010020C4F20703C2F22820002620
:1083A00008601E701378802BFCD07DE40AF09AFDE3
:1083B0005FE40AF097FD3EE54EF20103C4F20703C5
:1083C000602119701378802BFCD148F24403C4F269
:1083D00004030022C0F206221A6054E548F2440168
:1083E0004EF20103C4F204010020C4F20703C2F2FA
:1083F0002820002608601E701378802BFCD028E50A
:10840000002070470020704730B442F63D0342F62A
:108410003E04C2F20103C2F201041A782378D2B2F8
:10842000DBB29A422AD001333F2B14D942F2D03129
:1084300042F21043C2F20101C2F201030878196846
:108440000023C0B2237021B1D31A1A2B01DC002300
:108450000B7030BC704742F2D03042F21041C2F291
:108460000100C2F20101C05C0968DDB2C0B2257032
:108470000029EED09A4238BF4032E5E74FF0FF3096
:10848000E7E700BF42F63D0242F63E03C2F20102B8
:10849000C2F2010310781B78C0B2DBB2984238BF39
:1084A0004030C01A704700BF10B5044619B1012909
:1084B00011D0002010BD552220210EF0EDF900282A
:1084C000F7D0E28842F00402204692B22421BDE8AF
:1084D00010400EF0E1B940F273122A210EF0DCF9DF
:1084E0000028E6D08822202120460EF0D5F9002869
:1084F000DFD0E288204622F004022421BDE81040AB
:108500000EF0CAB938B50023C4F2013307EE103AB1
:1085100047F6EE43C3F6FF6307EE903AE0EE077AC4
:108520000546FCEEE77A17EE902AF2B1802A03792D
:108530009ABFC2F1800444EA0424002433B92246DD
:1085400028462221BDE838400EF0A6B9C288002393
:1085500022F01002037124210EF09EF922462846D3
:108560002221BDE838400EF097B90123037147F688
:108570007F7222210EF090F9EA8842F0100228461C
:1085800092B22421BDE838400EF086B90846114663
:108590000EF0C4BE10B50846144611460BF08EF915
:1085A000204610BD48F23403C4F204031B685A0588
:1085B00078D542F25C43C2F201032DE9F0471B6813
:1085C0000BB101221A7042F21448C2F2010842F2C1
:1085D000154598F8004001343F2C88BF4FF0000A41
:1085E00042F218474FF4204694BF5FFA84FA54468B
:1085F0008946C2F20105C2F20107C4F206062B78D1
:10860000A3422AD1EFF31383002B39D1EFF3108368
:10861000002B35D1EFF30582002A40D00F2A05D96F
:108620004EF2F033CEF2000313441B78EFF31182C5
:1086300012B1934228BF1346402B21D9B3F5807F56
:10864000DDD142F64903C2F201031B78002BD6D1DB
:108650000EF064FD2B78A342D4D042F258434FF47D
:108660002042C2F20103C4F2060207F8049001207E
:10867000BC21187088F800A0D1700120BDE8F087F7
:1086800033791B06BBD52B7801333F2B86BF0022E5
:108690001346DAB2FB5CDBB2F3712A70AFE74FF43A
:1086A0008073C3E7012070474FF42853C1F275531C
:1086B00003EB5100B0FBF1F00BF00ABA10B4036801
:1086C00041681A780C78417A037A0C4202EA030274
:1086D0001AD0837A03F003030AB143F0040343F092
:1086E00008039A10082B82722AD8072B22D2032B58
:1086F0002ED011D9042B13D0062B14D1C3685DF8EA
:10870000044B023BC3607047837A03F00303002AE3
:10871000E7D043F00403E4E7012B0BD0022B02D196
:10872000C368013BC3605DF8044B70470D2BF7D065
:108730000E2BF8D1C3685DF8044B0133C36070475A
:108740000C2B05D0F2D8092BD8D00B2BE8D0EAE7B8
:10875000C3685DF8044B0233C3607047037C10B5F7
:108760000446002B31D04368427A5B7A9A422CD877
:1087700072B60268D3683BB3984202D129E09C42AA
:1087800002D0DB68002BFAD16368617A1B6953F869
:10879000210048B10CF05AFA72B66368627A1B691C
:1087A000002143F822102268937A013B93722368D8
:1087B0009A7A02B91A726268937A013B937263687B
:1087C0009A7A22B10023237462B6204610BD1A7231
:1087D000F8E7C368D360D7E770B5044608460D468E
:1087E00011F0AEFE23680246294620465B68BDE8CC
:1087F000704018471D2810B50A4600F0AF8321D9F4
:108800002C2800F054813DD8242800F0B48340F295
:10881000A280282800F0428300F2CE80262800F0B3
:10882000DB8140F2AD8242F2F443C2F2010345F231
:108830007141C0F201012720C3F89C2002F0F4FA34
:10884000012010BD0E2800F0628338D8062800F001
:108850006B8368D90A2800F0D98200F2FB800828CF
:1088600000F06A8140F2528242F2F443C2F2010304
:1088700045F25161C0F2010109205A6202F0D4FAB6
:10888000012010BD342800F0848334D8302800F053
:10889000308300F2CC802E2800F0408140F2E58148
:1088A00042F2F443C2F2010345F2F131C0F2010198
:1088B0002F20C3F8BC2002F0B7FA012010BD152804
:1088C00000F03F8360D9192800F0DE8100F29D801E
:1088D000172800F0748140F2A68242F2F443C2F2FB
:1088E000010345F26151C0F2010118201A6602F03D
:1088F0009BFA012010BD382800F0A38270D83628DA
:1089000000F0278140F2598242F2F443C2F201039F
:1089100045F27131C0F201013720C3F8DC2002F0CA
:1089200083FA012010BD022800F0E38140F2628149
:10893000042800F0378140F2928242F2F443C2F2FE
:10894000010345F29161C0F2010105205A6102F074
:108950006BFA012010BD202800F0218240F27281C4
:10896000222800F0118140F2A78242F2F443C2F2C1
:10897000010345F2B141C0F201012320C3F88C206C
:1089800002F052FA012010BD112800F0978140F248
:108990004581132800F0EB8040F29D8142F2F443C0
:1089A000C2F2010345F2A151C0F2010114201A657F
:1089B00002F03AFA012010BD2A2800F0A18040F20E
:1089C000C28142F2F443C2F2010345F23141C0F2E6
:1089D00001012B20C3F8AC2002F026FA012010BDC3
:1089E0003A287FD0C0F04B823B2840F0468242F2CA
:1089F000F444C2F2010445F23131C0F20101C4F87D
:108A0000EC2002F011FA012010BD1B285DD040F2CD
:108A1000628242F2F443C2F2010345F22151C0F2F4
:108A200001011C201A6702F0FFF9012010BD322855
:108A300022D040F2798142F2F443C2F2010345F2BE
:108A4000B131C0F201013320C3F8CC2002F0ECF9BF
:108A5000012010BD0C281DD040F2848142F2F44365
:108A6000C2F2010345F21161C0F201010D205A6307
:108A700002F0DAF9012010BD42F2F443C2F2010320
:108A800045F2C131C0F20101C3F8C82002F0CCF9AF
:108A9000012010BD42F2F443C2F2010345F221610C
:108AA000C0F201011A6302F0BFF9012010BD42F2C9
:108AB000F443C2F2010345F22141C0F20101C3F8BF
:108AC000B02002F0B1F9012010BD42F2F443C2F22D
:108AD000010345F23151C0F20101DA6602F0A4F956
:108AE000012010BD42F2F443C2F2010345F24131CC
:108AF000C0F20101C3F8E82002F096F9012010BD90
:108B000042F2F443C2F2010345F24141C0F20101D5
:108B1000C3F8A82002F088F9012010BD42F2F44306
:108B2000C2F2010345F20141C0F20101C3F8B820CD
:108B300002F07AF9012010BD42F2F443C2F20103BF
:108B400045F26161C0F201011A6202F06DF9012083
:108B500010BD42F2F443C2F2010345F28131C0F28A
:108B60000101C3F8D82002F05FF9012010BD42F2E4
:108B7000F443C2F2010345F2B151C0F20101DA64DB
:108B800002F052F9012010BD42F2F443C2F2010397
:108B900045F2C141C0F20101C3F8882002F044F956
:108BA000012010BD42F2F443C2F2010345F2A1617B
:108BB000C0F201011A6102F037F9012010BD42F242
:108BC000F443C2F2010345F27151C0F20101DA65CA
:108BD00002F02AF9012010BD42F2F443C2F201036F
:108BE00045F28141C0F20101C3F8982002F01CF95E
:108BF000012010BD002800F0EF80012840F03D81E9
:108C000042F2F443C2F2010345F2D161C0F2010124
:108C100001205A6002F008F9012010BD0F2800F071
:108C2000E880102840F0298142F2F443C2F20103A7
:108C300045F2E151C0F2010110201A6402F0F4F88B
:108C4000012010BD1E282CD01F2840F0168142F2B2
:108C5000F443C2F2010345F2F141C0F201011F20C9
:108C6000DA6702F0E1F8012010BD42F2F443C2F2EB
:108C7000010345F21141C0F201012D20C3F8B420D7
:108C800002F0D2F8012010BD42F2F443C2F2010317
:108C900045F25151C0F201015A6602F0C5F80120B7
:108CA00010BD42F2F443C2F2010345F20151C0F299
:108CB00001019A6702F0B8F8012010BD42F2F443B6
:108CC000C2F2010345F2D151C0F201015A6402F02F
:108CD000ABF8012010BD42F2F443C2F2010345F2A9
:108CE000C151C0F2010112209A6402F09DF80120E6
:108CF00010BD42F2F443C2F2010345F2C161C0F279
:108D000001019A6002F090F8012010BD42F2F44394
:108D1000C2F2010345F27161C0F201010720DA617C
:108D200002F082F8012010BD42F2F443C2F20103C6
:108D300045F2D131C0F201013120C3F8C42002F064
:108D400073F8012010BD42F2F443C2F2010345F270
:108D50005141C0F201012920C3F8A42002F064F8B7
:108D6000012010BD42F2F443C2F2010345F2316129
:108D7000C0F201010B20DA6202F056F8012010BDAA
:108D800042F2F443C2F2010345F29141C0F2010103
:108D90002520C3F8942002F047F8012010BD42F2CC
:108DA000F443C2F2010345F2E141C0F20101C3F80C
:108DB000802002F039F8012010BD42F2F443C2F2E3
:108DC000010345F29131C0F201013520C3F8D420EE
:108DD00002F02AF8012010BD42F2F443C2F201036E
:108DE00045F2E161C0F201011A6002F01DF80120B4
:108DF00010BD42F2F443C2F2010345F2F151C0F258
:108E00000101DA6302F010F8012010BD42F2F443D0
:108E1000C2F2010345F24161C0F201019A6202F01F
:108E200003F8012010BD42F2F443C2F2010345F2FF
:108E30008151C0F2010116209A6501F0F5FF012071
:108E400010BD42F2F443C2F2010345F26131C0F2B7
:108E50000101C3F8E02001F0E7FF012010BD42F25C
:108E6000F443C2F2010345F2B161C0F201010320F3
:108E7000DA6001F0D9FF012010BD002010BD42F2E0
:108E8000F443C2F2010345F25131C0F2010139202D
:108E9000C3F8E42001F0C8FF012010BD42F2F44302
:108EA000C2F2010345F26141C0F20101C3F8A02002
:108EB00001F0BAFF012010BD42F2F443C2F20103F7
:108EC00045F2D141C0F201012120C3F8842001F014
:108ED000ABFF012010BD42F2F443C2F2010345F2A0
:108EE0004151C0F201011A209A6601F09DFF012054
:108EF00010BD42F2F443C2F2010345F2E131C0F287
:108F00000101C3F8C02001F08FFF012010BD42F223
:108F1000F443C2F2010345F20161C0F201019A6318
:108F200001F082FF012010BD42F2F443C2F20103BE
:108F300045F28161C0F201019A6101F075FF0120E3
:108F400010BD42F2F443C2F2010345F29151C0F266
:108F500001015A6501F068FF012010BD42F2F4439F
:108F6000C2F2010345F21151C0F201015A6701F04A
:108F70005BFF012010BD42F2F443C2F2010345F24F
:108F8000A141C0F20101C3F8902001F04DFF012082
:108F900010BD42F2F443C2F2010345F2A131C0F226
:108FA0000101C3F8D02001F03FFF012010BD00BF38
:108FB000F8B53F294EF6D02304461546C0F20E03FD
:108FC0000AD803EBC10253F831605268002740F21F
:108FD000031086F8807210603F2D0AD803EBC5029B
:108FE00053F835005268002740F2031680F880726B
:108FF000166053F8316053F8350006F500772760A6
:1090000000F50077012267604DF2C043002762F34C
:109010001F4322726272E760013BFDD196F8003275
:1090200090F8002203F00103D20744BF43F002038B
:10903000DBB2A37208462146FFF7DCFB2146207411
:109040002846FFF7D7FB237C184420742046F8BD40
:1090500010B44EF6E8740023C0F20E0441720261AF
:1090600004600372C36041B1194600E0026942F82E
:109070002310427A01339A42F8DC42F27043C2F282
:1090800001031A680AB90CE01A465369002BFBD198
:109090005061002343618380C38083725DF8044B79
:1090A00070471860F5E700BF2DE9F04F49F2E4255D
:1090B0009DB0C1F6FF752B7802AF04469BB12A46DE
:1090C000002302F8043B0F21006801F005FA05F1C6
:1090D0000C020E21206801F0FFF905F114020D21A8
:1090E000206801F0F9F9637BD4F8009004EB830465
:1090F0006368BB6393F85220002A40F0AE8393F874
:109100005030FB611846BA6B92F851203A638242A4
:1091100080F0918300247C61B861BA69944280F246
:10912000F1824EF6EC72C0F20E023A610022FA634E
:109130007A6949F630064CF6CD41C1F6FF76CCF699
:10914000CC410132B246B960FA604FF0010B97F89A
:109150003C207869FA6211468218D2B2BA62FA6982
:109160009A4203D2BB6B53F8243019703B69BD6B34
:109170000FCB55F8248007F1440498F8005098F874
:1091800001E084E80F0099F8093099F8052086F885
:109190005EB09D4284BF03F1FF35EDB207F1680375
:1091A00003EB8505520055F8243C86F85DB00EEBC4
:1091B000030464F07F04E4B2B6F85E3086F83B2026
:1091C0002501EDB204F0F0043BB199F80D30022214
:1091D00023438AF83C308AF85D2001200EF0A0FC81
:1091E00099F8053086F85EB0B6F85E2086F85DB076
:1091F0005B0086F83B304AB199F80D3043F0040328
:10920000234302228AF83C308AF85D2001200EF0C8
:1092100087FC3C23013BFDD199F8053086F85EB010
:10922000B6F85E2086F85DB05B0086F83B303AB158
:1092300099F80D301C4302238AF83C408AF85D30CF
:1092400001200EF06DFC40F6B833013BFDD199F8DA
:10925000053086F85EB0B6F85E2086F85DB05B003B
:1092600086F83B303AB199F80D3002222B438AF848
:109270003C308AF85D2001200EF052FC99F8053050
:1092800086F85EB0B6F85E2086F85DB05B0086F8C2
:109290003B304AB199F80D3043F004032B430222CE
:1092A0008AF83C308AF85D2001200EF039FC3C231E
:1092B000013BFDD199F8053086F85EB0B6F85E2026
:1092C00086F85DB05B0086F83B303AB199F80D3016
:1092D0001D4302238AF83C508AF85D3001200EF0CD
:1092E0001FFC40F6B833013BFDD141F6997308F1FC
:1092F000BC02C0F2010308F1BB0508F1A804C7F8DD
:1093000034803B6290467E6215F8012F412A00F0BE
:1093100056815AD8202A00F0828176D8092A00F096
:109320002A8100F2B480012A00F0A081082A14D119
:10933000236893F90020002AC0F2538240F0A682ED
:10934000302387F8653001222121D9F8003007F158
:10935000440001445B684846984704344445D3D1EF
:109360003B6BBA6AD7F834807E6A93421BD198F877
:109370000420022A00F0AF81032A00F09581012A1F
:10938000D9F8003000F082811A6888F804B041F6FC
:109390009973C0F201039A4240F06A8201220F21C0
:1093A000484608F0ABFDFB6AFA681344DCB2FB6B7D
:1093B0000133FB63BB699C4280F2A481BA6B92F8D3
:1093C00051303B6392F85030C1E6D92A53D032D99C
:1093D000F02A00F03A8149D9FB2A00F0A780FC2A44
:1093E00000F0A480FA2AB8D12368002BB5D09847A2
:1093F000D9F800303A6A1B689342014640F0A680D3
:109400000122484608F07AFDA7E73C2A00F0958043
:109410006BD8212A00F0A780322A9ED123681868D1
:109420000FF0EEFA7B6B5B79009302460B464846E1
:1094300009F01AFE91E7D02A00F08B8066D8462A00
:109440007BD0C92A89D12368002B86D0984707F1A1
:10945000680100280CBF3023312301F8033DD9F8FF
:10946000003001225B684846984776E7E82A70D0CA
:10947000E92A7FF472AF2368002B3FF46EAF984760
:10948000002301460A22484609F0AEFD65E7102A8E
:1094900079D0112A7FF461AF23681A88002A3FF43B
:1094A0004FAFBE68A6FB0213DB0803EB8301A2EB00
:1094B0004102303287F86520002B00F0D68121214F
:1094C000A6FB0302D20802EB82000139A3EB4003A2
:1094D000C9B207F168000844303300F8243C134651
:1094E000002AEDD1C1F122022FE73D2A63D03E2AA6
:1094F0007FF433AF2668304611F022F8D9F80030F7
:10950000024631465B684846984726E7D12AB2D0E2
:10951000D82A7FF422AF2368002B3FF41EAF984770
:1095200000280146C0F284810023ABE72368002BAA
:109530003FF413AF98470646DEE72268D9F80030BB
:1095400011781B683A6A93423FF45AAF48469847ED
:1095500003E72368002B3FF400AF9847011EE3DACE
:1095600049422D238EE722680023116848460A22CB
:1095700009F03AFDF1E622680023117848460A22F4
:1095800009F032FDE9E62368B3F90020002AC0F2B1
:10959000F3803FF4D5AEBB68A3FB0213DB0803EBFB
:1095A0008301A2EB4102303287F86520002B00F0E6
:1095B0005C810026F0E023681E6830469CE7226844
:1095C0003A60104610F0BCFF38643B6C386CC7F84A
:1095D00004D0073323F00703ADEB030D002802A9E5
:1095E0003A680BDD0020034603F1010E3E6CD35CAC
:1095F0000B545FFA8EF3B3421846F5DB3B6C3960CF
:109600000022CA54084610F09BFFD9F80030396890
:109610005B68024648469847D7F804D09DE6236821
:109620001B68002B72DB3FF48BAEBA68A2FB0321F0
:10963000C90801EB8102A3EB4203303387F86530A0
:10964000002900F01281002670E02368002B3FF40F
:1096500084AE984710EE100A0FF0D2F902260246A7
:109660000B460096484609F0FFFC76E623681B7817
:1096700007F16801002B0CBF3023312301F8033DB3
:10968000D9F8003048465B68984766E641F699711C
:109690001B68C0F201018B4248464FF00F0140F0B9
:1096A000F38008F02BFC7EE698F8022098F803106F
:1096B000484608F077FCD9F8002041F69973126803
:1096C000C0F201039A4240F0DB8001220D2148469E
:1096D00008F014FC67E698F8011098F800200139AA
:1096E000C9B2484608F05EFCD9F8002041F69973EB
:1096F0001268C0F201039A4240F0BE8001220E219E
:109700004846CEE76C37BD46BDE8F08FB9685B428E
:10971000A1FB0301C90801EB8100A3EB4003303337
:1097200087F86530002900F0C6802D262120D7F863
:1097300008C000E01846ACFB0132D20802EB820EF2
:10974000431EA1EB4E01DBB207F1680E9E4430319F
:109750000EF8241C1146002AECD1002E00F0A9803E
:109760000238C0B20146C0F1220207F16803184472
:109770002D2300F8243CE8E5BB685242A3FB02130A
:10978000DB0803EB8301A2EB4102303287F865204E
:10979000002B00F08A802D262120D7F808C000E099
:1097A0001046ACFB0321C90801EB810E421EA3EB5E
:1097B0004E03D2B207F1680E964430330EF8243CC3
:1097C0000B460029ECD1002E79D0831EDBB219465E
:1097D000C3F1220207F1680003442D2003F8240C92
:1097E000B3E5BB685242A3FB0213DB0803EB830122
:1097F000A2EB4102303287F86520002B55D02D2690
:109800002120D7F808C000E01046ACFB0321C908AE
:1098100001EB810E421EA3EB4E03D2B207F1680E9C
:10982000964430330EF8243C0B460029ECD1CAE7AD
:1098300041422D2326E60132121AD2B201461044CB
:1098400098427A61B86114467FF767AC5A1AD2B26F
:109850007A6114468A18BA615FE493F850309A42EC
:1098600028BF1A46FA6110464DE4012221216CE519
:109870000F214846904796E50E214846904792E5CD
:109880000D21484690478EE598478CE5BB68A3FBC1
:109890000213DB0803EB8301A2EB4102303287F8AD
:1098A0006520002BE1D00026AAE720210B460222EA
:1098B00090E7194616E611461046022255E7114672
:1098C000C2F1220241E500BF70B5064649F2A82563
:1098D0004EF6FC702DED028B0E21C0F20E00C1F68B
:1098E000FF750DF01BFD00220A2130460EF002FA32
:1098F00000F0F8FE95F91F3007EE106A07EE903A77
:109900000023C4F2482306EE103AF8EEE77AB8EEE8
:10991000477A002377EE867A37EE067AC4F2C823B8
:1099200006EE903A77EEA77A37EE077AC7EEA68A68
:1099300040F63073C2F201035B7AC7EE267AB7EEC7
:10994000008A78EEC88A37EEC88A002B62D10023DD
:10995000C4F2402307EE103A47F6EE43C3F6FF6326
:1099600007EE903A0023E8EE877ACCF23C2306EE2D
:10997000903AF4EEE67AF1EE10FA47D4F4EEC77AB4
:10998000F1EE10FAC8BF5F245FDD4FF48B7001F079
:109990005DF820F07F0240F630702243C2F20100F1
:1099A0004FF48B710CF078FF0023C4F2402307EED4
:1099B000103A47F6EE43C3F6FF6307EE903A0023F2
:1099C000E8EE077ACCF23C2306EE903AF4EEE67A23
:1099D000F1EE10FA1CD4F4EEC77AF1EE10FAC8BF1B
:1099E0005F2426DD4FF48F7001F030F820F07F0205
:1099F00040F630702243C2F201004FF48F710CF038
:109A00004BFFBDEC028B85F8206070BD0024BCE7E5
:109A10000024E7E74FF4847001F018F800F0030029
:109A2000022894D0032202214FF4847001F01CF923
:109A30008DE70023C4F23C2307EE103A77EE877AD5
:109A4000FCEEE77A17EE904ACCE70023C4F23C2301
:109A500007EE103A77EE877AFCEEE77A17EE904A37
:109A600093E700BF70B5064649F2A8254FF20C00F7
:109A70002DED028B0C21C0F20E00C1F6FF750DF02A
:109A80004DFC00220A2130460EF034F900F02AFE87
:109A900095F9203007EE106A07EE903A0023C4F2E1
:109AA000482306EE103AF8EEE77AB8EE477A00233C
:109AB00077EE867A37EE067AC4F2C82306EE903A3D
:109AC00077EEA77A37EE077A87EEA68A40F63073EC
:109AD000C2F201035B7AC7EE267AF7EE008A38EE0F
:109AE000688A77EEE88A002B61D10023C4F2402314
:109AF00007EE103A47F6EE43C3F6FF6307EE903ADF
:109B00000023E8EE877ACCF23C2306EE903AF4EE9E
:109B1000E67AF1EE10FA46D4F4EEC77AF1EE10FAD6
:109B2000C8BF5F245EDD4FF48B7000F08FFF20F024
:109B30007F0240F630702243C2F201004FF48B7175
:109B40000CF0AAFE0023C4F2402307EE103A47F6B9
:109B5000EE43C3F6FF6307EE903A0023E8EE077A80
:109B6000CCF23C2306EE903AF4EEE67AF1EE10FAEF
:109B70001BD4F4EEC77AF1EE10FAC8BF5F2425DDDE
:109B80004FF48F7000F062FF20F07F0240F63070DB
:109B90002243C2F201004FF48F710CF07DFEBDEC48
:109BA000028BEE7770BD0024BDE70024E8E74FF498
:109BB000847000F04BFF00F00300022895D00322D0
:109BC00002214FF4847001F04FF88EE70023C4F2B5
:109BD0003C2307EE103A77EE877AFCEEE77A17EE31
:109BE000904ACDE70023C4F23C2307EE103A77EE0B
:109BF000877AFCEEE77A17EE904A94E7F0B50746CD
:109C000049F2A8264FF21C0083B0C1F6FF7614215A
:109C1000C0F20E000DF082FB00220A2138460EF041
:109C200069F800F05FFD737F06EE107A07EE903A58
:109C30000023C4F2C62305EE903AF8EE464AF8EE49
:109C4000677A002387EEA56A4FF48370C4EEA57A85
:109C500007EE103A0023C4F27C2305EE103A47F6D3
:109C6000EE43C3F6FF6336EE076A37EE877A07EEF8
:109C7000903AE6EE057AFCEEE77ACDED017A9DF8B2
:109C800004303F2B9CBFC3F13F031D024FF0000384
:109C9000C4F2FE2306EE903A47F6EE43C3F6FF63A6
:109CA00007EE903AE7EE267A88BF0025FCEEE77AC9
:109CB000CDED017A9DF804307F2B94BFC3F17F0472
:109CC000002400F0C3FE20F47D5245EA040322F094
:109CD0003F0240F630701A434FF48371C2F2010024
:109CE0000CF0DAFDB77703B0F0BD00BFF0B5074662
:109CF0004FF2340083B01221C0F20E000DF00EFBC3
:109D000000220A2138460DF0F5FF00F0EBFC00239D
:109D1000C4F2C62305EE103A002307EE103A07EE10
:109D2000907A0023C4F27C2349F2A82604EE903AEC
:109D3000C1F6FF76F8EE677A47F6EE43C3F6FF63A7
:109D400087EE856A4FF4837006EE903AB37F05EE96
:109D5000903AF8EE655A36EE076AC5EE857AE6EE79
:109D6000246A37EE877AFCEEE67ACDED017A9DF82B
:109D700004303F2B9CBFC3F13F031D024FF0000393
:109D8000C4F2FE2306EE903A47F6EE43C3F6FF63B5
:109D900007EE903AE7EE267A88BF0025FCEEE77AD8
:109DA000CDED017A9DF804307F2B94BFC3F17F0481
:109DB000002400F04BFE20F47D5245EA040322F01B
:109DC0003F0240F630701A434FF48371C2F2010033
:109DD0000CF062FD777703B0F0BD00BF10B504460C
:109DE0004FF248001121C0F20E000DF097FA002248
:109DF0000A2120460DF07EFF00F074FC07EE904A29
:109E00000023C4F2C62306EE103AF8EE675A002388
:109E1000C5EE867A40F6584240F69041C2F2010201
:109E2000C2F2010106EE903A4FF47E43C4F2FF63A2
:109E300007EE103A77EEA67A4FF48033F4EEC77A45
:109E4000F1EE10FA93618B612BDC4FF47E43CCF280
:109E5000FF6307EE103AF4EEC77AF1EE10FA2BD456
:109E6000B0EE677ABEEEC87A17EE103A4FF47E4035
:109E7000C4F2FF6007EE100AF4EEC77AF1EE10FAB2
:109E8000D36124DC4FF47E43CCF2FF6307EE103A3B
:109E9000F4EEC77AF1EE10FA12D50023C8F20103EE
:109EA00003E00023C7F6FF73D36149F2A822C1F68D
:109EB000FF72CB61147610BD0023C8F20103D5E711
:109EC000B0EE677ABEEEC87A17EE103AEDE70023DF
:109ED000C7F6FF73E9E700BF2DE9F04149F2A82476
:109EE0002DED048BC1F6FF7400232779C4F2C6233D
:109EF0004FF2F47008EE903AC0F20100002308EE31
:109F0000103A0DF0EDFE384600F04EFD07EE907A67
:109F1000B8EE677A4BF22005C7EE287AC1F6FF75D6
:109F200028684368B2EE049A77EE887AC3ED007A27
:109F300007F0AAF9667927714FF60000C0F2010018
:109F40000DF0CEFE304600F02FFD07EE906AB8EE21
:109F5000677A2868C7EE287A436877EE887AC3ED77
:109F6000017A07F091F9A77966714FF61000C0F2F7
:109F700001000DF0B5FE384600F016FD07EE907AB0
:109F8000B8EE677A2868C7EE287A436877EE887A51
:109F9000C3ED027A07F078F9E679A7714FF6200051
:109FA000C0F201000DF09CFE304600F0FDFC07EE13
:109FB000906AB8EE677A2868C7EE287A436837EE69
:109FC000888A83ED038A07F05FF994F90870E671D7
:109FD0004FF62C00C0F201000DF082FE002FB5BF3D
:109FE0002D220022784238460A210DF083FE00F02F
:109FF00079FB07EE907A0023C4F2C623B8EEE76A35
:10A0000006EE903AC6EE267A0023286807EE103A4C
:10A01000436877EE877AC3ED077A07F035F994F94C
:10A020000A6027724FF64800C0F201000DF058FE9A
:10A03000002EB4BF2D2200224FF00A013046B8BFD7
:10A0400070420DF057FE00F04DFB07EE906A0023C2
:10A05000C4F24823F8EEE77A07EE103A0023C4F280
:10A06000C82306EE903A37EE877A0023C7EE267AA9
:10A07000286808EE103A0023C4F2C62308EE903A8E
:10A0800077EE887A4368C3ED097A07F0FDF894F813
:10A090000B80A6724FF65400C0F201000DF020FEB6
:10A0A000404600F081FC07EE908AB8EE677A286897
:10A0B000C7EE287A436877EE887AC3ED0A7A07F00C
:10A0C000E3F8277B84F80B804FF66000C0F20100B4
:10A0D0000DF006FE384600F067FC07EE907AB8EE09
:10A0E000677A2868C7EE287A436877EE887AC3EDE6
:10A0F000067A07F0C9F8667B27734FF67400C0F242
:10A1000001000DF0EDFD304600F04EFC07EE906AC8
:10A11000B8EE677A2868C7EE287A436877EE887ABF
:10A12000C3ED057A07F0B0F8A77B66734FF68C0095
:10A13000C0F201000DF0D4FD384600F035FC07EE0A
:10A14000907AB8EE677A2868C7EE287A436877EE87
:10A15000887AC3ED047A07F097F8E67BA7734FF689
:10A16000A000C0F201000DF0BBFD304600F01CFC69
:10A1700007EE906AB8EE677A2868C7EE287A4368D7
:10A1800077EE887AC3ED0B7A07F07EF8207CE673D1
:10A190000EF014FA607C0EF0CDF9A07C0EF086F97A
:10A1A000E77C4FF6B000C0F201000DF099FD384693
:10A1B00000F0FAFB637DA27C617C207C01EE103A0A
:10A1C000237D00EE903A07EE907AB8EE411AF8EE51
:10A1D000600AB8EE670A81EE091AC0EE890A00F03B
:10A1E0005BFD267DE7744FF6C400C0F201000DF060
:10A1F00077FD304600F0D8FB637DA27C617C207C3B
:10A2000007EE906A01EE103AE37CF8EE670A00EE82
:10A21000103AB8EE411AC0EE890A81EE091AB8EE7A
:10A22000400A00F039FD677D26754FF6D800C0F270
:10A2300001000DF055FD384600F0B6FB237DA27CF1
:10A24000617C207C07EE907A00EE903AE37CB8EED9
:10A25000671A00EE103AF8EE600A81EE091AC0EEB5
:10A26000890AB8EE400A00F017FDA67D67754FF623
:10A27000E800C0F201000DF033FD304600F094FB21
:10A2800007EE906AF8EE676AB7EE007AC6EEA87A33
:10A2900077EE887AF4EEC77AF1EE10FA40F3D780C1
:10A2A00044F21872C2F2000245F2606147F6705340
:10A2B00053524AF6B81245F26061C2F20002E07DE4
:10A2C0005352A6750EF066F80023207E08EE103A71
:10A2D000FFF784FD677E4FF60010C0F201000DF01D
:10A2E000FFFC384600F060FBA67E67764FF6301024
:10A2F000C0F201000DF0F4FC304600F055FBE77EA3
:10A30000A6764FF61810C0F201000DF0E9FC3846B1
:10A3100000F04AFB267FE7764FF64410C0F20100BA
:10A320000DF0DEFC304600F03FFB607F2677FFF744
:10A33000DDFCA07FFFF762FCE07FFFF793FB94F862
:10A340002000FFF7C1FA94F821604FF65810C0F2D0
:10A3500001000DF0C5FC304600F026FB07EE906AC8
:10A360000023C4F2C62306EE903AB8EE676A4CF6B4
:10A37000CD43C6EE267AC3F64C6394F8228084F867
:10A3800021604FF66810C0F2010007EE103A77EE38
:10A39000887A2B6867EE877A03F6DC43C3ED007A90
:10A3A0000DF09EFC404600F0FFFA94F8237084F80C
:10A3B00022804FF67C10C0F201000DF091FC38466F
:10A3C00000F0F2FA94F8246084F823704FF69010AD
:10A3D000C0F201000DF084FC304600F0E5FA286878
:10A3E00047F2A4050674C3F67D75F0EE487A84F84A
:10A3F0002460034600F51C61C3EDB47AC3F8D4525F
:10A4000034338B424FF00002F6D1BDEC048B00F6E2
:10A41000C8410024C4F220340C60002300F69847A1
:10A4200000F5496600F54B6500F6AC4400F6944132
:10A43000C0F87C3CC0F88C3C4FF07E533A603260F0
:10A440002A6022600B60BDE8F04106F01DBFF4EE0B
:10A45000C87AF1EE10FA36D445F62943C4F20F63F8
:10A4600007EE103A27EE877ABDEEC77A17EE103A5C
:10A4700003F5B34319331BB244F21872B7EE007AF6
:10A48000C2F2000245F26061F4EEC77AF1EE10FA12
:10A4900053521BDCF5EEC07AF1EE10FA10D445F6FB
:10A4A0002943C4F20F6307EE103A67EE877AFDEE98
:10A4B000E77A17EE903A03F5B34319331BB2F8E687
:10A4C00045F69913F5E645F69913D5E747F6705327
:10A4D000EFE600BFFFFFFFFF2DE9F04F01F007019E
:10A4E000C900914683B041F040010022054649F67B
:10A4F000300B07F003FD41F6997A09F10703C1F625
:10A50000FF7B09F1FF370193C0F2010A0124A3E0A8
:10A5100068798BF85E40BBF85E308BF85D4001F0E7
:10A52000F009400009018BF83B00CEB249F0010868
:10A530005BB1697B49F63003C1F6FF73022048EA3C
:10A54000010183F83C1083F85D0001200DF0E8FA6A
:10A5500069798BF85E40BBF85E008BF85D4049007E
:10A560008BF83B1048B1697B41F0050149EA0102D3
:10A5700002218BF83C208BF85D1001200DF0D0FA01
:10A580003C22013AFDD16A798BF85E40BBF85E103F
:10A590008BF85D4052008BF83B2039B16A7B022179
:10A5A00048EA02088BF83C808BF85D1001200DF022
:10A5B000B7FA40F6B832013AFDD16A798BF85E40BD
:10A5C000BBF85E108BF85D4052008BF83B2041B128
:10A5D0006A7B42F00102324302218BF83C208BF867
:10A5E0005D1001200DF09CFA6A798BF85E40BBF893
:10A5F0005E108BF85D4052008BF83B2041B16A7BC6
:10A6000042F00502324302218BF83C208BF85D10AA
:10A6100001200DF085FA3C22013AFDD16A798BF8D0
:10A620005E40BBF85E108BF85D4052008BF83B201B
:10A6300041B1697B41F001010E4302228BF83C607D
:10A640008BF85D2001200DF06BFA40F6B832013A2C
:10A65000FDD1019BBB420BD02A6817F8011F12687D
:10A6600052453FF455AF28469047019BBB42F3D17A
:10A6700003B0BDE8F08F00BF10B543F6F043C2F25F
:10A68000000393F8AD2053F82240206807F0AEFC99
:10A690002046BDE81040FEF707BD00BF38B543F6C1
:10A6A000F045C2F2000595F8AC1069B12C688442FF
:10A6B0000CD02A46002303E052F8044F844206D00F
:10A6C0000133DBB28B42F7D1002038BD002385F87F
:10A6D000AD30206807F08AFC2046FEF7E5FC01203B
:10A6E00038BD00BF00B54FF25C03C0F20E0383B06B
:10A6F0001B88ADF80430022101A80CF00FFE03B056
:10A700005DF804FB72B640F64C73C2F201039A780E
:10A71000012A23D01CD3022A07D0032A24D140F2D5
:10A7200078020421C1F6FF7204E040F27002C1F623
:10A73000FF7205219970018812F0080F14BFC82319
:10A740008823083043EA01435060136062B67047C3
:10A7500040F270020321C1F6FF72EBE740F278028B
:10A760000221C1F6FF72E5E71A6922B11A6B506047
:10A77000186362B670471861FAE700BF72B640F618
:10A780004C73C2F20103DA78012A23D01CD3022AC7
:10A7900007D0032A24D140F298020421C1F6FF72A7
:10A7A00004E040F29002C1F6FF720521D9700188E1
:10A7B00012F0080F14BFC8238823083043EA01436E
:10A7C0005060136062B6704740F290020321C1F6F8
:10A7D000FF72EBE740F298020221C1F6FF72E5E753
:10A7E0005A6922B15A6B5060586362B6704758611B
:10A7F000FAE700BF72B640F64C73C2F201031B6960
:10A8000033B100205B680130002BFBD162B670478A
:10A810001846FBE799B3012938B540D04378044680
:10A8200000781B0643EA004040F470408D1E40F063
:10A8300004000CF05BFE022D04F1020315D905346F
:10A8400014F8023C14F8032C14F8010C1B0443EA1E
:10A85000022343F0040343EA0060033D0CF046FE8C
:10A86000022D234604F10304EAD8022D22D0012D43
:10A870000BD04FF20570BDE838400CF037BE4FF2F8
:10A880000600C0F2F7000CF031BE1878000240F468
:10A89000770040F00600BDE838400CF027BE037892
:10A8A0004FF207001B04CFF200701843BDE8384098
:10A8B0000CF01CBE5A781878130443EA002040F0CC
:10A8C000774040F00700BDE838400CF00FBE00BFF5
:10A8D00099B3012938B540D04378044600781B0667
:10A8E00043EA004040F470408D1E40F004000DF03B
:10A8F000ABF9022D04F1020315D9053414F8023C1A
:10A9000014F8032C14F8010C1B0443EA022343F04F
:10A91000040343EA0060033D0DF096F9022D23463F
:10A9200004F10304EAD8022D22D0012D0BD04FF2FE
:10A930000570BDE838400DF087B94FF20600C0F24F
:10A94000F7000DF081B91878000240F4770040F06C
:10A950000600BDE838400DF077B903784FF20700E4
:10A960001B04CFF200701843BDE838400DF06CB9FD
:10A970005A781878130443EA002040F0774040F0FA
:10A980000700BDE838400DF05FB900BF10B50446C0
:10A990000FF0D6FD014620460CF0C0FC0446FFF740
:10A9A000A1FE204410BD00BF10B500220A210DF009
:10A9B000A1F90446FFF796FE204410BD70B443F69B
:10A9C000F043C2F2000393F8AD2053F82260337BCA
:10A9D000CBB100252846022406EB8502516891F888
:10A9E000502062B1002351F823201471D070907070
:10A9F000013391F85020DBB29A42F4D8337B013511
:10AA0000EDB29D42E8D3012070BC7047002810B51C
:10AA1000BABF40422D2200220A210DF06BF90446F4
:10AA2000FFF760FE204410BD43F6F043C2F200037E
:10AA300093F8AC202A2A06D8511C43F8220083F848
:10AA4000AC10012070470020704700BFF0B540F601
:10AA5000307549F63004C1F6FF74C2F201050122D7
:10AA60002B7A84F85E20B4F85E1084F85D20934061
:10AA700089B084F83B3039B1020A032384F83D00E1
:10AA800084F83C2084F85D3000200DF049F810B1C6
:10AA9000002009B0F0BD23692E7A84F83800122214
:10AAA00084F83900DA702269937849F6300503F0AA
:10AAB000200303F0FF07C1F6FF75002B00F0A7800D
:10AAC000B42393704DF27442C1F6FF72216913688A
:10AAD0000793079D06E013680693069B5B1B042BF8
:10AAE00000F29080CB7803F0200303F0FF00002BEE
:10AAF000F1D0730043F00103DBB20B7113680593CF
:10AB0000059D216905E013680493049B5B1B052BDD
:10AB100078D8CB7803F0020303F0FF00002BF2D0CB
:10AB20000223CB702169C87849F6300310F0110F69
:10AB3000C1F6FF7340F08180A020887019690B79FD
:10AB400013680393039D05E013680293029B5B1B4C
:10AB5000052B67D8CB7803F0020303F0FF00002B2E
:10AB6000F2D00223CB702069C178C9B249F6300314
:10AB7000CE06C1F6FF738BD48D0689D5A8218170CE
:10AB800019690879156801951876019805E0136828
:10AB90000093009B1B1A052B52D8CB7803F00203BD
:10ABA00003F0FF05002BF2D00225CD702169CB7890
:10ABB000DBB249F63002D806C1F6FF7248D49B06D4
:10ABC0007FF566AFB0238B7013691979517600BF9A
:10ABD00000BF00BF8021997092F8383082F8395058
:10ABE000012B26D8D1180133087ED9B202294FEAA9
:10ABF000002382F838101CD0507E82F83850184359
:10AC000009B0F0BD8870236980229A7040E70CF08B
:10AC100003FD00283FF43CAF2B6985F85F70B0223C
:10AC20009A704FE78870236980229A7084F83900FF
:10AC30002EE74FF0FF3009B0F0BD80238B7027E77F
:10AC40008D70226980210123917084F839301FE7CB
:10AC500010204FF49673C870013BFDD112699378B0
:10AC600003F0F703937013E770B50D4614460646DC
:10AC7000FFF7ECFE20EA040040EA050440F63070DD
:10AC800031462246C2F201000BF006FE002814BF36
:10AC90002046002070BD00BFF3EE047A80EE277AD4
:10ACA0002DE9704F054614460E4604F00104640178
:10ACB0002DED048B17EE100A82B0B0EE609AF0EE24
:10ACC000418A0DF09DFE9FED508A41EC110B9FEDE6
:10ACD0004C0B12F0A5FCC9EE087A5BEC10ABF1EE60
:10ACE000677A17EE900A0DF08BFE9FED450B41EC55
:10ACF000110B12F095FCC8EE887A59EC108BF1EE2E
:10AD0000677A17EE900A0DF07BFE9FED3D0B41EC4C
:10AD1000110B12F085FC45F61C234FF02042C3F6C0
:10AD2000E473504659468DED000B0DF00DFF0023E6
:10AD3000C4F2E00300220DF007FF0EF017F9C2B2D3
:10AD400040F630704FF49371C2F201000BF0A4FD95
:10AD5000002142464B460020C3F6F0710DF0F0FC96
:10AD60000023C4F2201300220DF0EEFE0EF0FEF8D8
:10AD7000C2B240F630704FF49471C2F201000BF091
:10AD80008BFD9DED000B002153EC102B0020C3F632
:10AD9000F0710DF0D5FC0023C4F2601300220DF019
:10ADA000D3FE0EF0E3F8C2B240F630704FF4957166
:10ADB000C2F201000BF070FD4FF49270FFF746FEF7
:10ADC000022D06F0030144EA012128BF022520F4E8
:10ADD0004C5020F0200041EA0534044340F6307026
:10ADE0002246C2F201004FF492710BF055FD00B102
:10ADF000A0B202B0BDEC048BBDE8708FAFF3008051
:10AE0000000000000000244000555749002810B5FC
:10AE1000BABF40422D2200220A210CF06BFF0446EB
:10AE2000FFF760FC204410BDF0B44EF6D024C0F211
:10AE30000E0404EBC0035A68136813F4E06301D1F5
:10AE40003F2856D948F20063C1F6FF7349F27127D3
:10AE5000C1F6FF7749F24126C1F6FF76C3F82C719F
:10AE600002F1404749F2112549F2E11449F2B110CB
:10AE7000C3F83061A7F59226C1F6FF75C1F6FF74DD
:10AE8000C1F6FF707C2EC3F83451C3F83841C3F8C3
:10AE90003C0129D9A7F594237C2B10D9A7F596233B
:10AEA0007C2B33D9A7F598237C2B2AD9A7F59A2791
:10AEB0007C2F17D849F20034C1F6FF7403E049F241
:10AEC000DC34C1F6FF7472B6136823F4702343F0C8
:10AED0008570C2F3840540F48030136044F8251077
:10AEE000106062B6F0BC704749F23C44C1F6FF7492
:10AEF000E9E754F830404FF4807084F880321060F5
:10AF0000A0E749F26C34C1F6FF74DCE749F2AC34D7
:10AF1000C1F6FF74D7E700BF4FF2600070B5C0F212
:10AF20000E00FFF733FD43F21C70C2F20000FFF782
:10AF3000B5FB49F2A822C1F6FF724BF2EC11C1F643
:10AF4000FF7192F824204E684A604BF2C0104DF217
:10AF50001443C1F6FF733021C1F6FF7000250124B0
:10AF60008A42467183F83C505C63996316DC9AB15F
:10AF7000920072B6DA6262B643F6F043C2F20003A0
:10AF800093F8AD2053F82240206807F02FF82046B0
:10AF9000BDE87040FEF788B80422EAE7C022E8E77F
:10AFA0004FF27C0010B5C0F20E00FFF7EFFC43F249
:10AFB0003050C2F20000FFF771FB4BF2EC11C1F60A
:10AFC000FF7149F2A8224BF2C010C1F6FF70C1F622
:10AFD000FF724DF21443C1F6FF734C68447192F84E
:10AFE00023204A60002001249C6383F83C005863BE
:10AFF00072B69200DA6262B643F6F043C2F2000320
:10B0000093F8AD2053F82240206806F0EFFF204669
:10B01000BDE81040FEF748B84FF2A00010B5C0F2EE
:10B020000E00FFF7B3FC43F24430C2F20000FFF71A
:10B0300035FB4BF2EC11C1F6FF7149F2A8224BF23D
:10B04000C010C1F6FF70C1F6FF724DF21443C1F695
:10B05000FF734C68447192F822204A60002010244B
:10B060009C6383F83C00586372B6A242A8BF224694
:10B070009200DA6262B643F6F043C2F2000393F83C
:10B08000AD2053F82240206806F0B0FF2046BDE80E
:10B090001040FEF709B800BF4FF2C00010B5C0F273
:10B0A0000E00FFF773FC43F25810C2F20000FFF7E6
:10B0B000F5FA4BF2EC11C1F6FF7149F2A8224BF2FE
:10B0C000C010C1F6FF70C1F6FF724DF21443C1F615
:10B0D000FF734C68447192F821204A600020632479
:10B0E0009C6383F83C00586372B6A242A8BF224614
:10B0F0009200DA6262B643F6F043C2F2000393F8BC
:10B10000AD2053F82240206806F070FF2046BDE8CD
:10B110001040FDF7C9BF00BF4FF2DC0070B5C0F2B0
:10B120000E00FFF733FC42F6F830C2F20000FFF7E2
:10B13000B5FA49F2A422C1F6FF724BF2EC11C1F646
:10B14000FF7112784E684A604BF2C0104DF2144302
:10B15000C1F6FF736321C1F6FF70002501248A4206
:10B16000067083F83C505C63996316DC9AB19200D8
:10B1700072B6DA6262B643F6F043C2F2000393F8A5
:10B18000AD2053F82240206806F030FF2046BDE88D
:10B190007040FDF789BF0422EAE74FF4C672E7E783
:10B1A0004FF2FC0070B5C0F20E00FFF7EFFB42F665
:10B1B0000C20C2F20000FFF771FA49F2A823C1F691
:10B1C000FF734BF2EC11C1F6FF7193F920304E681A
:10B1D0004B604BF2C0104DF21442C1F6FF726FF09B
:10B1E0003101C1F6FF70002532248B42C670B8BF12
:10B1F0000B46516382F83C50946372B6A342A8BFD9
:10B2000023469B00D36262B643F6F043C2F20003CA
:10B2100093F8AD2053F82240206806F0E7FE204660
:10B22000BDE87040FDF740BF4FF2181070B5C0F296
:10B230000E00FFF7ABFB42F62000C2F20000FFF762
:10B240002DFA49F2A823C1F6FF734BF2EC11C1F6B7
:10B25000FF7193F91F304E684B604BF2C0104DF2F6
:10B260001442C1F6FF726FF03101C1F6FF70002584
:10B2700032248B42C670B8BF0B46516382F83C50F3
:10B28000946372B6A342A8BF23469B00D36262B602
:10B2900043F6F043C2F2000393F8AD2053F8224086
:10B2A000206806F0A3FE2046BDE87040FDF7FCBE16
:10B2B0004FF2341010B5C0F20E00FFF767FB42F2F8
:10B2C0003460C2F20000FFF7E9F94BF2EC11C1F66D
:10B2D000FF7149F2A8224BF2C010C1F6FF70C1F60F
:10B2E000FF724DF21443C1F6FF734C68C470927F35
:10B2F0004A60002063249C6383F83C00586372B664
:10B30000A242A8BF22469200DA6262B643F6F04338
:10B31000C2F2000393F8AD2053F82240206806F0F3
:10B3200065FE2046BDE81040FDF7BEBE4FF2581046
:10B3300010B5C0F20E00FFF729FB42F24840C2F2FE
:10B340000000FFF7ABF94BF2EC11C1F6FF7149F2C7
:10B35000A8224BF2C010C1F6FF70C1F6FF724DF289
:10B360001443C1F6FF734C68C470527F4A600020DA
:10B3700063249C6383F83C00586372B6A242A8BF62
:10B3800022469200DA6262B643F6F043C2F200034C
:10B3900093F8AD2053F82240206806F027FE20469F
:10B3A000BDE81040FDF780BE4FF2781010B5C0F236
:10B3B0000E00FFF7EBFA42F25C20C2F20000FFF74A
:10B3C0006DF94BF2EC11C1F6FF7149F2A8224BF274
:10B3D000C010C1F6FF70C1F6FF724DF21443C1F602
:10B3E000FF734C68C470127F4A60002063249C6322
:10B3F00083F83C00586372B6A242A8BF224692006E
:10B40000DA6262B643F6F043C2F2000393F8AD206D
:10B4100053F82240206806F0E9FD2046BDE81040C0
:10B42000FDF742BE4FF2981010B5C0F20E00FFF7C4
:10B43000ADFA42F27000C2F20000FFF72FF94BF2B2
:10B44000EC11C1F6FF7149F2A8224BF2C010C1F60F
:10B45000FF70C1F6FF724DF21443C1F6FF734C68E2
:10B46000C470D27E4A60002064249C6383F83C0050
:10B47000586372B6A242A8BF22469200DA6262B650
:10B4800043F6F043C2F2000393F8AD2053F8224094
:10B49000206806F0ABFD2046BDE81040FDF704BE75
:10B4A0004FF2BC1010B5C0F20E00FFF76FFA41F674
:10B4B0008460C2F20000FFF7F1F84BF2EC11C1F624
:10B4C000FF7149F2A8224BF2C010C1F6FF70C1F61D
:10B4D000FF724DF21443C1F6FF734C68C470927E44
:10B4E0004A60002014249C6383F83C00586372B6C1
:10B4F000A242A8BF22469200DA6262B643F6F04347
:10B50000C2F2000393F8AD2053F82240206806F001
:10B510006DFD2046BDE81040FDF7C6BD4FF2DC10C2
:10B5200010B51621C0F20E000BF0F8FEFFF7DAF8A6
:10B5300043F60810C2F20000FFF7B0F843F6F043FC
:10B54000C2F200034BF2EC1193F8AD00C1F6FF71AB
:10B550004BF2C012C1F6FF7253F820404B681370D3
:10B56000206806F043FD2046BDE81040FDF79CBD75
:10B570004FF2F41010B52021C0F20E000BF0CEFEF9
:10B58000FFF7B0F843F6E040C2F20000FFF786F89C
:10B590004BF21C02C1F6FF724BF2EC11C1F6FF71C7
:10B5A0004DF21443C1F6FF7312784A600120002166
:10B5B000986383F83C10596372B69200DA6262B6FF
:10B5C00043F6F043C2F2000393F8AD2053F8224053
:10B5D000206806F00BFD2046BDE81040FDF764BD75
:10B5E000F8B54BF2C0164FF21820C1F6FF762921AC
:10B5F000C0F20E000BF092FE96F905000028BABFCB
:10B6000040422D2200220A2143F6F0450CF072FB45
:10B61000C2F20005FFF766F842F66C70C2F2000055
:10B62000FFF73CF895F8AD3055F823E09EF80C3064
:10B63000D3B10027384602240EEB8702516891F8F7
:10B6400050206AB1002351F823201471D0709070FB
:10B65000013391F85020DBB29A42F4D89EF80C30B6
:10B660000137FFB29F42E7D34BF2EC11C1F6FF71F5
:10B6700096F905204B683370002A4BF2C013C1F6CF
:10B68000FF731DDB4DF21443C1F6FF73032400204A
:10B69000A2424A609C6383F83C005863D4BF920086
:10B6A0000C2272B6DA6262B695F8AD3055F82340D6
:10B6B000206806F09BFC2046BDE8F840FDF7F4BC8E
:10B6C0004DF21442C1F6FF7200240320906382F809
:10B6D0003C4054635C714C6072B6D46262B695F8BB
:10B6E000AD3055F82360306806F080FC737B06EBC4
:10B6F00083035A6892F8513092F8500008E098425B
:10B7000082F851300CD052F8231091F8C11039B999
:10B71000591C9842CBB2F2D8002382F85140F2E78C
:10B72000306806F063FC3046FDF7BEFCBCE700BFA6
:10B73000F8B504464DF23440C1F6FF7009F0D8FF69
:10B740004BF2C017C1F6FF77385540F29C30C2F279
:10B750000000FEF7A3FF43F6F043C2F2000393F8A4
:10B76000AD2053F82260337BCBB10025284602245C
:10B7700006EB8502516891F8502062B1002351F820
:10B7800023201471D0709070013391F85020DBB2F7
:10B790009A42F4D8337B0135EDB29D42E8D34BF2A7
:10B7A000EC114DF21442C1F6FF7297F90330C1F665
:10B7B000FF71002013244B60946323EAE37382F843
:10B7C0003C00506372B6A342A8BF23469B00D362DD
:10B7D00062B6F8BDF8B504464DF23440C1F6FF70CC
:10B7E00009F086FF4BF2C017C1F6FF7738554EF2CD
:10B7F0009C20C1F6FF70FEF751FF43F6F043C2F202
:10B80000000393F8AD2053F82260337BCBB10025C1
:10B810002846022406EB8502516891F8502062B157
:10B82000002351F823201471D0709070013391F8E7
:10B830005020DBB29A42F4D8337B0135EDB29D4201
:10B84000E8D34BF2EC114DF21442C1F6FF7297F9B6
:10B850000230C1F6FF71002008244B60946323EA94
:10B86000E37382F83C00506372B6A342A8BF23463C
:10B870009B00D36262B6F8BDF8B504464DF2344081
:10B88000C1F6FF7009F034FF4BF2C017C1F6FF7725
:10B8900038554DF66810C1F6FF70FEF7FFFE43F60F
:10B8A000F043C2F2000393F8AD2053F82260337BDB
:10B8B000CBB100252846022406EB8502516891F899
:10B8C000502062B1002351F823201471D070907081
:10B8D000013391F85020DBB29A42F4D8337B013522
:10B8E000EDB29D42E8D34BF2EC114DF21442C1F699
:10B8F000FF7297F90030C1F6FF71002005244B60FC
:10B90000946323EAE37382F83C00506372B6A34267
:10B91000A8BF23469B00D36262B6F8BD70B54DF256
:10B920003444C1F6FF740646204609F0E1FE4BF2AE
:10B93000C015C1F6FF75A85542F66C70C2F2000042
:10B94000FEF7ACFEFFF73AF84BF2EC12A4F1200040
:10B9500095F90530C1F6FF7200210324536084631A
:10B9600023EAE37380F83C10416372B6A342A8BF98
:10B9700023469B00C36262B670BD00BF2DE9F04153
:10B98000091A002643F6F0444FB2B046C2F2000452
:10B9900087EAE772F3B2A2EBE772934244DA94F8D3
:10B9A000AD3054F82350002F28681DDA06F01EFB36
:10B9B0006B7B05EB83035B6893F8501093F85100A1
:10B9C000421C8842D2B204D2914283F8512002D163
:10B9D00022E083F8518093F8512053F8222092F806
:10B9E000C120002AEAD017E006F000FB6B7B05EBD4
:10B9F00083035B6893F851104A1ED2B221B993F8C1
:10BA0000502083F8512007E083F8512053F822207A
:10BA100092F8C120002AEDD0286806F0E7FA2846FF
:10BA2000FDF742FB0136B3E7BDE8F081013BDBB235
:10BA30000F2B1BD82DE9F04145B2002D01DBBDE8ED
:10BA4000F081E02813D9F728F9D900F10803DAB218
:10BA50000123934013F0DD0FF1D0014643F6E85087
:10BA6000C2F20000BDE8F04105F01EBE704743F68B
:10BA7000A058C2F200081646D8F848E0DEF80020C8
:10BA800048F2A5571268C0F200072B43BA42044699
:10BA900001F07F05D8B222D107F098FFD8F848000E
:10BAA00003681B68BB4217D1284607F08FFF04F0DC
:10BAB000EF00C028C3D0D8F8482013681B68BB42E9
:10BAC00006F07F0003D1BDE8F04107F07FBF0146DB
:10BAD000BDE8F0411046184729469847E7E7014678
:10BAE00070469047DAE700BF72B641F20003C2F237
:10BAF0000103586850B101885A8C10B4521A446836
:10BB00005C605A8462B65DF8044B704762B6704759
:10BB100072B641F20003C2F20103186950B1018804
:10BB20001A8D10B4521A44681C611A8562B65DF809
:10BB3000044B704762B67047C368BBB110B401E0F4
:10BB4000DB688BB11A7A002AFAD15A68587A1269DE
:10BB500052F82040002CF3D142F820100A7801322C
:10BB60000A70DB68002BEDD15DF8044B704700BF15
:10BB7000F0B44FF44044C4F202044FF0004623688E
:10BB8000FE2743F4806323602246E6622346676310
:10BB900035464C1C01F20127D16A0029FCDA1968EC
:10BBA00014F8016C41F480611960DD625E63D16A52
:10BBB0000029FCDA196814F8026B41F48061A7428D
:10BBC0001960DD625E63E7D14FF44041C4F20201C7
:10BBD000CA6A4FF44043002AC4F20203F8DA1A6832
:10BBE0004FF0004542F48062FF241A601946DD627E
:10BBF0005C63CA6A4FF44043002AC4F20203F8DAD5
:10BC00001A684FF0004542F48062FF241A6019461A
:10BC1000DD625C63CA6A4FF44043002AC4F2020347
:10BC2000F8DA1A684FF0004542F48062FF241A6087
:10BC30001946DD625C63CA6A4FF44043002AC4F2CD
:10BC40000203F8DA9B6BDBB203F01F024370A2F130
:10BC50000500B0FA80F04009F0BC70472DE9F04FC4
:10BC60008468066A83B0002C55D000230134019308
:10BC7000F368591C8846A3B3A045274638BF022461
:10BC800041F2000A49F2B44B38BF27468C42814644
:10BC9000C2F2010AC1F6FF7B4FF0000521D896F8E9
:10BCA0002030F069102BDBF8003022D000EBD410EC
:10BCB000984222D104F07F030AEB83031B6B23F02D
:10BCC000704393B101342746F3680135AB4208D97C
:10BCD000A04538BF022403F1010138BF27468C423A
:10BCE000DDD9002003B0BDE8F08FBC4217D001348D
:10BCF000EAE700EB1420984208D0002106F098F9FA
:10BD00000028EED096F82030102BD3D1E3B20AEB06
:10BD100043031B8ED5E7012334680193A8E7012F65
:10BD2000DFD9F36801339F42DBD86FF070423946A8
:10BD3000304606F095F90028D3D0D9F8081059B14B
:10BD40000129CED9F36801339942CAD83A46304620
:10BD500006F086F90028C4D0019BC9F808700BB121
:10BD60007B1C3360D9F81C305BB999F80530C9F8F1
:10BD70001C7063F07F03012089F8053003B0BDE833
:10BD8000F08F012003B0BDE8F08F00BF38B5026925
:10BD9000D478E4B2E106054628D51023D3706306B3
:10BDA00023D504F0040404F0FF03002C62D041F218
:10BDB0000003C2F20103696E002283F8302285F885
:10BDC0005D2000296ED0884795F85D30002B69D042
:10BDD0002B69D0229A702B6995F83B201A712B6938
:10BDE000012285F85C200222DA7038BD04F040039D
:10BDF00003F0FF00002BD4D19379DBB203F0600194
:10BE0000602956D0937803F0100303F0FF01B3B11B
:10BE100014F001043FD195F85C3095F85D1099421B
:10BE200053D9591C2B4485F85C1093F83B3013719F
:10BE30002B69D0229A702B690222DA70D5E785F837
:10BE40006010937943F0200393712B6995F83910B2
:10BE50001A791F29D2B2C6D841F20000C2F20100FD
:10BE600090F830020028BED06818013185F83910EA
:10BE70000276B8E72A6985F83930C02393702B69B8
:10BE800041F20002C2F201021979012182F8301256
:10BE90000222DA70A9E7C02393702B691A79022273
:10BEA000DA70A2E70122002385F85D2085F83B3097
:10BEB0008EE703F0DF039371AB6E23B185F8380092
:10BEC00095F8390098472A699CE71471B0E700BFDC
:10BED0002DE9F04F44F28454C2F200042268002A93
:10BEE00066D013682360002B00F09A8041F20005B1
:10BEF000C2F201058B46B5F8466219682160002E32
:10BF000052D148F280141360C8F2000441F2402C70
:10BF1000C2F2010C2CF47F614FF4207921F00F0163
:10BF20004FF0010EC0F20809C2F804E001F5805A92
:10BF3000C2F80890C2F80CC001F5005901F5405C48
:10BF400001F58041C2F810A0C2F81490C2F818C0E0
:10BF5000D161C3F804E0D5F84412D5F840820568F1
:10BF60009D629C6099634FF0000C4FF48059C3F8B8
:10BF700034804FF4005A4FF440554FF48044006829
:10BF8000C3F80CC0C3F83CC0C3F81090C3F82CB081
:10BF9000C3F814A01E639D611146DC61C3F800E084
:10BFA000BDE8F04F09F04EBF29B911601A60236057
:10BFB0000020BDE8F08F95F940820F6827604FEAB6
:10BFC000064C6FEA08044CF0004C4FEAD878E40FB6
:10BFD0002BF47F6E4CF0800C2EF00F0E4CEA082CE8
:10BFE0004FF001092402C1F804900EF58058C1F801
:10BFF00008C00EF500590EF5405C44F080240EF5A3
:10C00000804EC1F80CB044F08004C1F81080C1F833
:10C010001490C1F818C0C1F81CE011600B6075E7FE
:10C0200013602260C4E700BF2DE9F04F44F2805452
:10C03000C2F2000489B0D4F800A00594BAF1000F50
:10C0400074D0264644F28454C2F200042746079472
:10C050003D68DAF80040346006952E46002D00F069
:10C06000748288461D46039233680291814601908E
:10C0700060220021402450463B600CF0D1FF224654
:10C08000002130460CF0CCFF43460122EDB2032BD9
:10C0900032604146B460CAF810608AF83550CAF878
:10C0A0003090CAF814208AF8348000F0A280039BF4
:10C0B0004BB1019B5A680AB96FE21A46936B002B89
:10C0C000FBD1C2F838A0029B002B33D1019B9AF818
:10C0D00037001D7D039F9AF83630012D8CBF00215B
:10C0E0000121C9064FF48042019E747D44F07044E2
:10C0F00044EA0724129F44EA07442143114341EADA
:10C100000532CAF80420B27DF17D120442EAC15220
:10C1100042F08042134343EA0023CAF80830029BEE
:10C1200033F0020310D0029B032B1FD0504609B0FE
:10C13000BDE8F08F019B9AF837001D7D039F9AF8A8
:10C14000363000221146CFE741F25812C4F20A02FB
:10C150001368002B00F00B821A68CAF800205046C2
:10C160004AF002021A6009B0BDE8F08FBAF8420046
:10C17000BAF840101F28D9D842F20005C2F20105D2
:10C180004AF0020655F82020D4074FEA800729D448
:10C1900002F00604022C22F01F0308D1E1E19A45C7
:10C1A00017D01A68D20708D41B6823F01F03B3F80E
:10C1B00040209142F3D99A450BD01A6832F01F0201
:10C1C00005D1C9E1126832F01F0200F0C581924525
:10C1D000F8D108441F28A9D855F82020D4074FEAE1
:10C1E0008007D5D508441F28CAF80020EE51F3D99E
:10C1F0009CE701991298097D42F6AB23C0F2010336
:10C2000003FB00F302294FEA134300F00881AAF868
:10C210004020002D40F0C48184334FEA5318022798
:10C2200000224FF0FF3341F2000C99469646C2F2CD
:10C23000010CCDF810A0934651E0824580F0898032
:10C24000A04238BF2046984228BF18460CEB050391
:10C2500038BFF14693F8491293F84D32414438BF44
:10C260004FF0000B8A453B446DD3544566D29A4546
:10C27000514638BF1946884298BF01460CEB05006D
:10C28000424490F84E0284BFF1464FF0010B9442B5
:10C2900038444DD39C4246D98442224638BF024698
:10C2A0006544914298BF0A46464495F84F1284BFB0
:10C2B000F1464FF0020BB342394430D3834229D9BF
:10C2C0008B4238BF0B469A4288BFF1460EF1010EF1
:10C2D00094BF13464FF0030BBEF1200F3ED04FEA40
:10C2E000CE050CEB050494F8480294F84A2294F821
:10C2F0004B6294F84C4200EB0801D01981423C4457
:10C3000006EB070A99D9514523D9A14238BF2146E6
:10C31000084698E78842034638BF0B46D3E7B04249
:10C32000F8D23346CCE783421A4638BF0246B7E715
:10C330009342F8D2824238BF0246B1E79C4221467E
:10C3400038BF194697E78C42F8D2994238BF194650
:10C3500091E75445204638BF504674E7BB2BDDF8C3
:10C3600010A05E464CD85FFA88F8FFB201231FFA8E
:10C3700089F4B9F11F0F8AF84A808AF84B70AAF83D
:10C3800048B0AAF84430AAF8464098BF584622D888
:10C3900000EBC9030CEB0305991C95F84822614496
:10C3A000424485F8482291F84852DA1C62443D44E0
:10C3B00081F8485292F8481204336344394482F8B1
:10C3C000481293F8482209F101093A44B9F1200FC3
:10C3D00083F84822DCD101231C20B340B040DBB2FB
:10C3E000C0B2AAF842408AF836308AF83700039A79
:10C3F000002A7FF45EAE019917460D7D114673E663
:10C40000079A06981368059C036023681060002053
:10C41000CAF80030C4F800A009B0BDE8F08F41F2BE
:10C420004720C2F201005733AAF840205B0900F50B
:10C430008074002110F8012F1A44914238BF114630
:10C440008442F7D1BB29DBD841F2000CC2F2010CC7
:10C450000CF51274614201F00301B1F5807FDBB28B
:10C460004FF001004FF0000228BF4FF480718AF8AE
:10C470004A30AAF84400AAF84620002900F0958026
:10C480009CF8482281421A448CF8482200F08D80A2
:10C490009CF8492202291A448CF8492200F0858030
:10C4A0009CF84A221A448CF84A220322002663F39D
:10C4B000070663F30F26C1F1FC0563F31746AD08C9
:10C4C0000C4463F31F66013506F07F39C1F5807BAC
:10C4D0004FEA850EA4F10408002758F8041F01F064
:10C4E0007F307140484401F0803101374140AF4214
:10C4F00044F8041BF1D3DE4572441DD0944441F24C
:10C5000000009CF8481219448CF84812511CB1F5EF
:10C51000807FC2F201000FD00144023291F84842FC
:10C52000B2F5807F1C4481F8484205D0024492F85D
:10C5300048120B4482F848320020FF238AF8363034
:10C54000AAF842008AF8370051E7059BCAF8004074
:10C550002846C3F800A0EAE51A68CAF800201E6061
:10C5600037E6B3F84040A1427FF619AE3AE6DAF872
:10C5700004104FF48A534AF00200C4F20A0341F453
:10C580000041CAF80410CAF80000C2F800A01A68F6
:10C5900042F0200250461A60C9E5C3F804A092E5B3
:10C5A00066335F094FF002083AE60A467EE700BFAD
:10C5B000F8B50446002301250570457005718370A8
:10C5C000C37080F8C130C0F8A830C0F8AC30C0F8F3
:10C5D000B030C0F8B430C0F8B8300E46C4F8BC3043
:10C5E000194684F8C030A02208300CF019FD022250
:10C5F0000923A5716271C4F8A86084F8BC30204694
:10C60000F8BD00BFF8B5044600230125057045704C
:10C6100005718370C37080F8C130C0F8A830C0F8CD
:10C62000AC30C0F8B030C0F8B430C0F8B8300E4606
:10C63000C4F8BC30194684F8C030A02208300CF091
:10C64000EFFC02220823A5716271C4F8A86084F887
:10C65000BC302046F8BD00BFF8B5044600230125D4
:10C660000570457005718370C37080F8C130C0F8E3
:10C67000A830C0F8AC30C0F8B030C0F8B430C0F862
:10C68000B8300E46C4F8BC30194684F8C030A02239
:10C6900008300CF0C5FC0222FB23A5716271C4F8BE
:10C6A000A86084F8BC302046F8BD00BF4368427AD9
:10C6B0005B7A9A421FD830B472B60468E3682BB331
:10C6C000DA6832B119688C4216D01346DA68002A4B
:10C6D000F8D1D8600023C360A37A0133A372026843
:10C6E0004168012313728A7A1A448A72426813726B
:10C6F000037462B630BC70475D6841688D42E4D116
:10C70000198903899942F4D01346DFE7E060E1E735
:10C71000F8B500F1180204460121FCF799FC204607
:10C720004FF24C23C0F20E0340F81C3B40F6B80217
:10C7300000210CF075FC04F6D40040F648120021EC
:10C740000CF06EFC04F5905040F6FA1200211C30FB
:10C750000CF066FC04F5E05040F6982200211630FB
:10C760000CF05EFC04F51A5040F61C3200212E300D
:10C770000CF056FC04F5475040F6A63200210A3072
:10C780000CF04EFC04F5755040F62A420021303082
:10C790000CF046FC04F5934040F6A24200211A300A
:10C7A0000CF03EFC45F23E6745F23C63002545F245
:10C7B000406645F2426245F24460E55245F2466108
:10C7C000E55345F2486345F24A67A553A55245F241
:10C7D0004C66255245F24E6245F250606552E55274
:10C7E00045F25261E55345F2546345F25667A5534D
:10C7F000A55245F25866255245F25A6245F25C60F0
:10C800006552E55245F25E61E55345F2606341F6DB
:10C810009917A553A55246F26766275246F6843209
:10C8200004F5AC4066526230E25229464FF48B6206
:10C830000CF0F6FB04F5B540294640F272323A306E
:10C840000CF0EEFB04F5BC40294640F2AA222C3045
:10C850000CF0E6FB04F5C14029464FF4E172563076
:10C860000CF0DEFB46F2982046F29A2146F29C221A
:10C8700046F29E23255265522046A552E552F8BD48
:10C880004FF2502010B5C0F20E00FEF77FF841F6CF
:10C890009840C2F20000FDF701FF4BF2EC11C1F627
:10C8A000FF7149F2A8224BF2C010C1F6FF70C1F629
:10C8B000FF724DF21443C1F6FF734C68C470527E90
:10C8C0004A60002014249C6383F83C00586372B6CD
:10C8D000A242A8BF22469200DA6262B643F6F04353
:10C8E000C2F2000393F8AD2053F82240206805F00F
:10C8F0007DFB2046BDE81040FCF7D6BB4FF274200C
:10C9000010B5C0F20E00FEF741F841F6AC20C2F2BD
:10C910000000FDF7C3FE4BF2EC11C1F6FF7149F2C6
:10C92000A8224BF2C010C1F6FF70C1F6FF724DF2A3
:10C930001443C1F6FF734C68C470127E4A60002035
:10C9400063249C6383F83C00586372B6A242A8BF7C
:10C9500022469200DA6262B643F6F043C2F2000366
:10C9600093F8AD2053F82240206805F03FFB2046A5
:10C97000BDE81040FCF798BB4FF2942010B5C0F210
:10C980000E00FEF703F841F6C000C2F20000FDF70A
:10C9900085FE4BF2EC11C1F6FF7149F2A8224BF271
:10C9A000C010C1F6FF70C1F6FF724DF21443C1F61C
:10C9B000FF734C68C470D27D4A60002063249C637E
:10C9C00083F83C00586372B6A242A8BF2246920088
:10C9D000DA6262B643F6F043C2F2000393F8AD2088
:10C9E00053F82240206805F001FB2046BDE81040C6
:10C9F000FCF75ABB4FF2B82010B5C0F20E00FDF79D
:10CA0000C5FF41F2D460C2F20000FDF747FE4BF2D1
:10CA1000EC11C1F6FF7149F2A8224BF2C010C1F629
:10CA2000FF70C1F6FF724DF21443C1F6FF734C68FC
:10CA3000C470927D4A60002063249C6383F83C00AC
:10CA4000586372B6A242A8BF22469200DA6262B66A
:10CA500043F6F043C2F2000393F8AD2053F82240AE
:10CA6000206805F0C3FA2046BDE81040FCF71CBB67
:10CA70004FF2DC2010B5C0F20E00FDF787FF41F247
:10CA8000E840C2F20000FDF709FE4BF2EC11C1F6DE
:10CA9000FF7149F2A8224BF2C010C1F6FF70C1F637
:10CAA000FF724DF21443C1F6FF734C68C470527D9F
:10CAB0004A60002063249C6383F83C00586372B68C
:10CAC000A242A8BF22469200DA6262B643F6F04361
:10CAD000C2F2000393F8AD2053F82240206805F01D
:10CAE00085FA2046BDE81040FCF7DEBA4FF2FC2084
:10CAF00010B5C0F20E00FDF749FF41F21010C2F26E
:10CB00000000FDF7CBFD4BF2EC11C1F6FF7149F2CD
:10CB1000A8224BF2C010C1F6FF70C1F6FF724DF2B1
:10CB20001443C1F6FF734C68C470D27C4A60002085
:10CB300060249C6383F83C00586372B6A242A8BF8D
:10CB400022469200DA6262B643F6F043C2F2000374
:10CB500093F8AD2053F82240206805F047FA2046AC
:10CB6000BDE81040FCF7A0BA4FF2203010B5C0F27B
:10CB70000E00FDF70BFF40F62470C2F20000FDF737
:10CB80008DFD4BF2EC11C1F6FF7149F2A8224BF278
:10CB9000C010C1F6FF70C1F6FF724DF21443C1F62A
:10CBA000FF734C68C470927C4A60002001249C632F
:10CBB00083F83C00586372B69200DA6262B643F6BC
:10CBC000F043C2F2000393F8AD2053F822402068EE
:10CBD00005F00CFA2046BDE81040FCF765BA00BF2E
:10CBE0004FF2403010B5C0F20E00FDF7CFFE40F618
:10CBF0003850C2F20000FDF751FD4BF2EC11C1F6C6
:10CC0000FF7149F2A8224BF2C010C1F6FF70C1F6C5
:10CC1000FF724DF21443C1F6FF734C68C470527C2E
:10CC20004A60002003249C6383F83C00586372B67A
:10CC3000A242A8BF22469200DA6262B643F6F043EF
:10CC4000C2F2000393F8AD2053F82240206805F0AB
:10CC5000CDF92046BDE81040FCF726BA4FF260300F
:10CC600010B5C0F20E00FDF791FE40F27470C2F2F2
:10CC70000000FDF713FD4BF2EC11C1F6FF7149F214
:10CC8000A8224BF2C010C1F6FF70C1F6FF724DF240
:10CC90001443C1F6FF734C68C470927B4A60002055
:10CCA00063249C6383F83C00586372B6A242A8BF19
:10CCB00022469200DA6262B643F6F043C2F2000303
:10CCC00093F8AD2053F82240206805F08FF92046F4
:10CCD000BDE81040FCF7E8B94FF2843010B5C0F25F
:10CCE0000E00FDF753FE40F28850C2F20000FDF73F
:10CCF000D5FC4BF2EC11C1F6FF7149F2A8224BF2C0
:10CD0000C010C1F6FF70C1F6FF724DF21443C1F6B8
:10CD1000FF734C68C470527B4A60002063249C639C
:10CD200083F83C00586372B6A242A8BF2246920024
:10CD3000DA6262B643F6F043C2F2000393F8AD2024
:10CD400053F82240206805F051F92046BDE8104014
:10CD5000FCF7AAB94FF2AC3010B5C0F20E00FDF7E7
:10CD600015FE4FF2FC10C1F6FF70FDF797FC4BF279
:10CD7000EC11C1F6FF7149F2A8224BF2C010C1F6C6
:10CD8000FF70C1F6FF724DF21443C1F6FF734C6899
:10CD90008470D27A4A60002063249C6383F83C004C
:10CDA000586372B6A242A8BF22469200DA6262B607
:10CDB00043F6F043C2F2000393F8AD2053F822404B
:10CDC000206805F013F92046BDE81040FCF76CB967
:10CDD0004FF2C83070B5C0F20E00FDF7D7FD4EF629
:10CDE0002460C1F6FF70FDF759FC49F2A823C1F693
:10CDF000FF734BF2EC11C1F6FF7193F909304E68E5
:10CE00004B604BF2C0104DF21442C1F6FF726FF04E
:10CE10001701C1F6FF70002518248B428670B8BF39
:10CE20000B46516382F83C50946372B6A342A8BF8C
:10CE300023469B00D36262B643F6F043C2F200037E
:10CE400093F8AD2053F82240206805F0CFF8204633
:10CE5000BDE87040FCF728B94FF2E43038B5C0F2B5
:10CE60000E00FDF793FD4EF63840C1F6FF70FDF75A
:10CE700015FC49F2A823C1F6FF734BF2EC11C1F681
:10CE8000FF714BF2C0104DF21442C1F6FF7293F9DC
:10CE900008304D684B60C1F6FF700021632423EA1F
:10CEA000E3738570946382F83C10516372B6A342B9
:10CEB000A8BF23469B00D36262B643F6F043C2F29A
:10CEC000000393F8AD2053F82240206805F08EF857
:10CED0002046BDE83840FCF7E7B800BF4FF20040FD
:10CEE00010B5C0F20E00FDF751FD4EF66000C1F620
:10CEF000FF70FDF7D3FB4BF2EC11C1F6FF7149F265
:10CF0000A8224BF2C010C1F6FF70C1F6FF724DF2BD
:10CF10001443C1F6FF734C68847092794A60002014
:10CF200063249C6383F83C00586372B6A242A8BF96
:10CF300022469200DA6262B643F6F043C2F2000380
:10CF400093F8AD2053F82240206805F04FF82046B2
:10CF5000BDE81040FCF7A8B84FF21C4010B51D21E9
:10CF6000C0F20E000AF0DAF9FDF7BCFB41F2FC203A
:10CF7000C2F20000FDF792FB4BF2EC11C1F6FF711B
:10CF800049F2A8224BF2C010C1F6FF70C1F6FF7241
:10CF90004DF21443C1F6FF734C68C470127D4A60B1
:10CFA000002063249C6383F83C00586372B6A2425D
:10CFB000A8BF22469200DA6262B643F6F043C2F29C
:10CFC000000393F8AD2053F82240206805F00EF8D6
:10CFD0002046BDE81040FCF767B800BF4FF23C4068
:10CFE00010B51B21C0F20E000AF098F9FDF77AFB8C
:10CFF00040F64C30C2F20000FDF750FB4BF2EC1152
:10D00000C1F6FF7149F2A8224BF2C010C1F6FF70C1
:10D01000C1F6FF724DF21443C1F6FF734C68C47041
:10D02000127C4A60002002249C6383F83C00586311
:10D0300072B6A242A8BF2246A240DA6262B643F6A6
:10D04000F043C2F2000393F8AD2053F82240206869
:10D0500004F0CCFF2046BDE81040FCF725B800BF27
:10D060004FF2584010B51B21C0F20E000AF056F9DD
:10D07000FDF738FB40F66010C2F20000FDF70EFB32
:10D080004BF2EC11C1F6FF7149F2A8224BF2C0102D
:10D09000C1F6FF70C1F6FF724DF21443C1F6FF7383
:10D0A0004C68C470D27B4A60002063249C6383F880
:10D0B0003C00586372B6A242A8BF22469200DA62D0
:10D0C00062B643F6F043C2F2000393F8AD2053F882
:10D0D0002240206804F08AFF2046BDE81040FBF79C
:10D0E000E3BF00BF4FF2744010B52021C0F20E0024
:10D0F0000AF014F94FF2E830C1F6FF70FDF7CEFAEE
:10D100004BF2EC11C1F6FF7149F2A8224BF2C010AC
:10D11000C1F6FF70C1F6FF724DF21443C1F6FF7302
:10D120004C688470127B4A60002063249C6383F8FF
:10D130003C00586372B6A242A8BF22469200DA624F
:10D1400062B643F6F043C2F2000393F8AD2053F801
:10D150002240206804F04AFF2046BDE81040FBF75B
:10D16000A3BF00BF4FF2984070B51621C0F20E0069
:10D170000AF0D4F8FDF7B6FA4FF21000C1F6FF70CE
:10D18000FDF78CFA49F2A823C1F6FF734BF2EC11BC
:10D19000C1F6FF7193F90A304E684B604BF2C01034
:10D1A0004DF21442C1F6FF726FF03101C1F6FF700B
:10D1B000002532248B428670B8BF0B46516382F83B
:10D1C0003C50946372B6A342A8BF23469B00D3622F
:10D1D00062B643F6F043C2F2000393F8AD2053F871
:10D1E0002240206804F002FF2046BDE87040FBF7B3
:10D1F0005BBF00BF4FF2B04010B51821C0F20E0067
:10D200000AF08CF8FDF76EFA4EF64C20C1F6FF706E
:10D21000FDF744FA4BF2EC11C1F6FF7149F2A82276
:10D220004BF2C010C1F6FF70C1F6FF724DF214430D
:10D23000C1F6FF734C688470D2794A600020632481
:10D240009C6383F83C00586372B6A242A8BF224692
:10D250009200DA6262B643F6F043C2F2000393F83A
:10D26000AD2053F82240206804F0C0FE2046BDE8FF
:10D270001040FBF719BF00BFF8B54BF2C0164FF2D4
:10D28000CC40C1F6FF762921C0F20E000AF046F824
:10D2900096F903000028BABF40422D2200220A213D
:10D2A00043F6F0450AF026FDC2F20005FDF71AFA32
:10D2B00040F29C30C2F20000FDF7F0F995F8AD3075
:10D2C00055F823E09EF80C30D3B1002738460224ED
:10D2D0000EEB8702516891F850206AB1002351F893
:10D2E00023201471D0709070013391F85020DBB27C
:10D2F0009A42F4D89EF80C300137FFB29F42E7D330
:10D300004BF2EC11C1F6FF7196F903204B683370B4
:10D31000002A4BF2C013C1F6FF731DDB4DF214431C
:10D32000C1F6FF7313240020A2424A609C6383F875
:10D330003C005863D4BF92004C2272B6DA6262B6E7
:10D3400095F8AD3055F82340206804F04FFE204694
:10D35000BDE8F840FBF7A8BE4DF21442C1F6FF72DB
:10D3600000241320906382F83C405463DC704C60CE
:10D3700072B6D46262B695F8AD3055F82360306865
:10D3800004F034FE737B06EB83035A6892F8513045
:10D3900092F8500008E0984282F851300CD052F8D0
:10D3A000231091F8C11039B9591C9842CBB2F2D868
:10D3B000002382F85140F2E7306804F017FE30464F
:10D3C000FBF772FEBCE700BF38B505464FF2F840E8
:10D3D0000C46C0F20E000D2109F0A0FF49F2A8236F
:10D3E000C1F6FF7393F823305BB304F50051C1F32A
:10D3F000C6122B4601F07F01E020FEF717FB04F375
:10D400000D044FF2085004F50054C0F20E00013D27
:10D410000AF066FC2D02200400F4FE0005F470659D
:10D42000054345F46040640440F00E0004F0FE44FF
:10D4300020430AF009FC4FF21850C0F20E000AF027
:10D440004FFCBDE83840FDF74DB900BF38B5054683
:10D450004FF230500C46C0F20E000D2109F05EFF75
:10D4600049F2A823C1F6FF7393F82330FBB121469C
:10D470002B460022D020FEF7D9FA4FF20850C0F216
:10D480000E0024040AF02CFC04F4FE04681E44F48C
:10D490005044000244F00D0400F4706020430AF090
:10D4A000D3FB4FF21850C0F20E000AF019FCBDE891
:10D4B0003840FDF717B900BFF8B549F2A825C1F605
:10D4C000FF750C4695F82230064623B1984202D0EB
:10D4D0000AF02CFDC0B149F2A423C1F6FF731C7001
:10D4E000FAF7AAFB43F6F043C2F200034DF600320E
:10D4F00093F8AD1053F821707B7B07EB8303C1F6E3
:10D50000FF725B6893422DD04FF24050C0F20E0084
:10D510000D2109F003FF95F82330FBB12146334676
:10D520000022C020FEF782FA4FF20850C0F20E002F
:10D5300024040AF0D5FB04F4FE04701E44F44044B5
:10D54000000244F00C0400F4706020430AF07CFBFD
:10D550004FF21850C0F20E000AF0C2FBBDE8F840CE
:10D56000FDF7C0B8386804F041FD3846FBF79CFD74
:10D57000CAE700BF2DE9F04149F2A826C1F6FF76BF
:10D580000C4696F8223015460746B3B3984234D07D
:10D590000AF0CCFC88BB4FF25050C0F20E000D21B7
:10D5A00009F0BCFE96F823301BB32A4621463B46C1
:10D5B000B020FEF73BFA2D064FF20850C0F20E00E5
:10D5C00005F0FE450AF08CFB45F430452404781E36
:10D5D00045F00B0504F4FE0400022C4300F47060D7
:10D5E00020430AF031FB4FF21850C0F20E000AF04F
:10D5F00077FBBDE8F041FDF775B85C2CCBD00CD8BB
:10D600000A2C29D05B2C50D105EB850000EB800063
:10D61000C0F34710FCF7E2FBBDE75D2C33D05E2C76
:10D6200043D107EE905A0023C4F2FE2306EE903A4F
:10D63000B8EE676A0023C6EE267A07EE103A4BF280
:10D640002003C1F6FF7377EE877A18684368C3ED4D
:10D650000A7A03F019FE9EE707EE905A0023C4F2FF
:10D66000FE2306EE903AB8EE676A0023C6EE267AED
:10D6700007EE103A77EE877AFDEEE77A17EE903AEA
:10D6800086F8253087E705EB850808EB88084FF614
:10D690004410C8F34718C0F201000AF021FB4046CD
:10D6A000FDF782F986F81C8075E74BF22003C1F67E
:10D6B000FF732A461868036821465B6898476AE743
:10D6C0002DE9F04F49F2A826C1F6FF7687B096F80B
:10D6D0002230029104920390D3B3984238D00AF0DA
:10D6E00025FCA8BB4FF26050C0F20E00122109F0D9
:10D6F00015FE96F8233033B3039E049D029C3346F7
:10D700002A4621468020FEF791F94FF20850C0F2D8
:10D710000E000AF0E5FA2B0603F0FE4343F4004343
:10D720002204701E02F4FE0243F0080300021343B9
:10D7300000F4706018430AF087FA4FF21850C0F2F4
:10D740000E000AF0CDFA07B0BDE8F04FFCF7CABFF3
:10D750004BF22003C1F6FF7396F909A0D3F800B08D
:10D76000029B9BF81020DBF804809A44002AB9D071
:10D7700005965C4600258027464604E00135AA420E
:10D7800004F134040FDDD4F8EC329A45F6D1DBF81D
:10D790008C3C53B1C4F8EC729BF810200135AA42BE
:10D7A00004F13404EFDC059E9CE7DBF80C0080F00C
:10D7B00000400BF025F9CDE9000150460BF00EF9C1
:10D7C00047F6E1234FF08042C3F684730BF0BCF9B7
:10D7D00000230022C4F218030AF0B4FF736807EEB6
:10D7E000103AF1EE047A67EE277A804617EE900A37
:10D7F00089460BF005F902460B46404649460AF0B9
:10D800009FFF41EC100B0FF087FEDDE9000153ECA8
:10D81000102B0BF099F941EC100B0FF07DFE51EC41
:10D82000100B0BF041F9C4F8D4029BF81020A5E7C7
:10D83000F8B549F2A825C1F6FF750E4695F82230D5
:10D840001446074623B1984202D00AF06FFB18B184
:10D850002146304603F0B2FF4FF27450C0F20E0082
:10D86000112109F05BFD95F823301BB322463146A8
:10D870003B469020FEF7DAF824064FF20850C0F23B
:10D880000E0004F0FE440AF02BFA44F4104436046F
:10D89000781E44F0090406F4FE060002344300F446
:10D8A000706020430AF0D0F94FF21850C0F20E0019
:10D8B0000AF016FABDE8F840FCF714BF4FF28850A2
:10D8C00008B5C0F20E001B2109F028FD49F2A8237B
:10D8D000C1F6FF7393F82330B3B143F6E850FF214C
:10D8E000C2F2000003F0E0FE4FF20850C0F20E005A
:10D8F0000AF0F6F94FF60F7009F0F8FD4FF2A45058
:10D90000C0F20E000AF0ECF9BDE80840FCF7EABEF0
:10D910004FF2B45008B5C0F20E001D2109F0FEFC14
:10D9200049F2A823C1F6FF7393F82330B3B143F64D
:10D93000E850FE21C2F2000003F0B6FE4FF208509C
:10D94000C0F20E000AF0CCF94FF60F6009F0CEFDE0
:10D950004FF2A450C0F20E000AF0C2F9BDE8084030
:10D96000FCF7C0BE4FF2D45008B5C0F20E0014212F
:10D9700009F0D4FC49F2A823C1F6FF7393F82330D1
:10D98000B3B143F6E850FC21C2F2000003F08CFE74
:10D990004FF20850C0F20E000AF0A2F94FF60F4005
:10D9A00009F0A4FD4FF2A450C0F20E000AF098F95D
:10D9B000BDE80840FCF796BEF8B549F2A825C1F6C7
:10D9C000FF750E4695F822301446074623B198425B
:10D9D00002D00AF0ABFA18B12146304603F0EEFE51
:10D9E0004FF2EC50C0F20E00162109F097FC95F8AA
:10D9F00023301BB3224631463B469020FEF716F8F3
:10DA000024064FF20850C0F20E0004F0FE440AF063
:10DA100067F944F410443604781E44F0090406F40F
:10DA2000FE060002344300F47060204309F05EFDFE
:10DA30004FF2A450C0F20E000AF052F9BDE8F840CF
:10DA4000FCF750BE4FF2046008B5C0F20E0016217C
:10DA500009F064FC49F2A823C1F6FF7393F8233060
:10DA60009BB14FF60F700AF0EFF84FF21850C0F26A
:10DA70000E000AF035F94FF60F7009F037FD4FF23E
:10DA8000A450C0F20E000AF02BF9BDE80840FCF7E4
:10DA900029BE00BF4FF21C6008B5C0F20E0018216D
:10DAA00009F03CFC49F2A823C1F6FF7393F8233038
:10DAB0009BB14FF60F600AF0C7F84FF21850C0F252
:10DAC0000E000AF00DF94FF60F6009F00FFD4FF24E
:10DAD000A450C0F20E000AF003F9BDE80840FCF7BC
:10DAE00001BE00BF4FF2386008B5C0F20E000F2132
:10DAF00009F014FC49F2A823C1F6FF7393F8233010
:10DB00009BB14FF60F400AF09FF84FF21850C0F249
:10DB10000E000AF0E5F84FF60F4009F0E7FC4FF26F
:10DB2000A450C0F20E000AF0DBF8BDE80840FCF794
:10DB3000D9BD00BF4FF2486008B5C0F20E001321F6
:10DB400009F0ECFB49F2A823C1F6FF7393F82330E8
:10DB50009BB14FF60F300AF077F84FF21850C0F231
:10DB60000E000AF0BDF84FF60F3009F0BFFC4FF27F
:10DB7000A450C0F20E000AF0B3F8BDE80840FCF76C
:10DB8000B1BD00BF4FF25C6008B5C0F20E001021BD
:10DB900009F0C4FB49F2A823C1F6FF7393F82330C0
:10DBA0009BB14FF60F200AF04FF84FF21850C0F219
:10DBB0000E000AF095F84FF60F2009F097FC4FF28F
:10DBC000A450C0F20E000AF08BF8BDE80840FCF744
:10DBD00089BD00BF4FF2706008B5C0F20E00102181
:10DBE00009F09CFB49F2A823C1F6FF7393F8233098
:10DBF0009BB14FF60F000AF027F84FF21850C0F211
:10DC00000E000AF06DF84FF60F0009F06FFC4FF2AE
:10DC1000A450C0F20E000AF063F8BDE80840FCF71B
:10DC200061BD00BF4FF2846008B5C0F20E0016213E
:10DC300009F074FB49F2A823C1F6FF7393F823306F
:10DC40009BB14FF20F6009F0FFFF4FF21850C0F286
:10DC50000E000AF045F84FF20F6009F047FC4FF252
:10DC6000A450C0F20E000AF03BF8BDE80840FCF7F3
:10DC700039BD00BF10B504464FF29C60C0F20E00E3
:10DC8000152109F04BFB49F2A823C1F6FF7393F865
:10DC90002330C3B1240404F4FE0444F4734444F078
:10DCA0000204204609F0D0FF4FF21850C0F20E00D7
:10DCB0000AF016F8204609F019FC4FF2A450C0F201
:10DCC0000E000AF00DF8BDE81040FCF70BBD00BFD8
:10DCD00070B506464FF2B4600C46C0F20E00122139
:10DCE000154609F01BFB49F2A823C1F6FF7393F810
:10DCF00023301BB9BDE87040FCF7F4BC6B1E1B025F
:10DD0000240404F4FE0403F47063234343F45043F7
:10DD1000340143F00D03E4B21C43204609F094FFA4
:10DD20004FF21850C0F20E0009F0DAFF4EB14FF278
:10DD3000A450C0F20E0009F0D3FFBDE87040FCF71C
:10DD4000D1BC204609F0D2FBF1E700BF38B504464C
:10DD50004FF2C860C0F20E001F2109F0DFFA49F24D
:10DD6000A823C1F6FF7393F82330CBB104F00F045E
:10DD70004FF202152404C0F210052543284609F08D
:10DD800063FF4FF21850C0F20E0009F0A9FF2846B9
:10DD900009F0ACFB4FF2A450C0F20E0009F0A0FF56
:10DDA000BDE83840FCF79EBC38B504464FF2E86049
:10DDB0000D46C0F20E00102109F0B0FA49F2A82376
:10DDC000C1F6FF7393F823309BB129462046FCF738
:10DDD0007FFD4FF21850C0F20E0009F081FF20467F
:10DDE0002946FCF717FD4FF2A450C0F20E0009F0CF
:10DDF00077FFBDE83840FCF775BC00BF70B549F24D
:10DE0000A826C1F6FF760D4696F82230044623B1C7
:10DE1000984202D00AF08AF8C0B149F2A423C1F6B0
:10DE2000FF731D70F9F708FF43F6F043C2F20003D9
:10DE30004DF6003293F8AD1053F82130597B03EBC7
:10DE40008103C1F6FF725B6893422BD04FF2FC60F6
:10DE5000C0F20E000D2109F061FA96F82330EBB103
:10DE60002D0405F4FE05013C45F44045240245F02F
:10DE70000C0504F470642C43204609F0E5FE4FF2D3
:10DE80001850C0F20E0009F02BFF204609F02EFBBF
:10DE90004FF2A450C0F20E0009F022FFBDE870401E
:10DEA000FCF720BCFCF7E8FBD0E700BF4FF20C709A
:10DEB00008B5C0F20E00182109F030FA49F2A82383
:10DEC000C1F6FF7393F82330B3B143F6E850FB215A
:10DED000C2F2000003F0E8FB4FF20850C0F20E005F
:10DEE00009F0FEFE4FF60F3009F000FB4FF2A45090
:10DEF000C0F20E0009F0F4FEBDE80840FCF7F2BBEA
:10DF00004FF2287008B5C0F20E00152109F006FA8C
:10DF100049F2A823C1F6FF7393F82330B3B143F657
:10DF2000E850FA21C2F2000003F0BEFB4FF20850A5
:10DF3000C0F20E0009F0D4FE4FF60F2009F0D6FA19
:10DF40004FF2A450C0F20E0009F0CAFEBDE808402E
:10DF5000FCF7C8BB4FF2407008B5C0F20E001521A7
:10DF600009F0DCF949F2A823C1F6FF7393F82330D6
:10DF7000B3B143F6E850F821C2F2000003F094FB7D
:10DF80004FF20850C0F20E0009F0AAFE4FF60F0043
:10DF900009F0ACFA4FF2A450C0F20E0009F0A0FE56
:10DFA000BDE80840FCF79EBB4FF2587008B5C0F2C0
:10DFB0000E001B2109F0B2F949F2A823C1F6FF7344
:10DFC00093F82330C3B143F6A053C2F20003F62105
:10DFD000986C0368DB6C98474FF20850C0F20E0053
:10DFE00009F07EFE4FF20F6009F080FA4FF2A45064
:10DFF000C0F20E0009F074FEBDE80840FCF772BBE9
:10E0000038B504464FF27470C0F20E001A2109F0C0
:10E0100085F949F2A823C1F6FF7393F823301BB9A1
:10E02000BDE83840FCF75EBB43F6A055C2F20005E0
:10E0300048F2A553A86C02681268C0F200039A4225
:10E0400021D1F32005F0C2FCA86C036804F07F0125
:10E05000DB6C98474FF20850C0F20E0009F040FE0A
:10E06000200400F4FE0040F4734040F0020009F088
:10E070003DFA4FF2A450C0F20E0009F031FEBDE8A7
:10E080003840FCF72FBBF3219047DDE770B504461D
:10E090004FF29070C0F20E00242109F03FF949F2CE
:10E0A000A823C1F6FF7393F823301BB9BDE8704075
:10E0B000FCF718BB43F6A056C2F2000648F2A5557D
:10E0C000B06C03681B68C0F20005AB4224D1F1209C
:10E0D00005F07CFCB06C03681B68AB421FD1204686
:10E0E00005F074FC4FF20850C0F20E0009F0F8FD84
:10E0F00004F00F044FF202102404C0F21000204379
:10E1000009F0F4F94FF2A450C0F20E0009F0E8FD56
:10E11000BDE87040FCF7E6BAF1219847DAE72146FE
:10E120009847DFE770B506464FF2B8700C46C0F26C
:10E130000E001721154609F0F1F849F2A823C1F69F
:10E14000FF7393F823301BB9BDE87040FCF7CABADF
:10E15000A02033462A462146FDF768FC4FF2D070D6
:10E16000C0F20E0009F0BCFD4EB14FF2A450C0F257
:10E170000E0009F0B5FDBDE87040FCF7B3BA681EAB
:10E180000002240404F4FE0400F47060204340F410
:10E19000504040F00D0009F0A9F9E6E738B5054612
:10E1A0004FF2DC700C46C0F20E00122109F0B6F8F6
:10E1B00049F2A823C1F6FF7393F8233063B304F543
:10E1C0000051C1F3C6122B4601F07F01E020FDF79C
:10E1D0002DFC04F30D044FF208500F2104F50054F8
:10E1E000C0F20E00013D09F099F82D02200400F460
:10E1F000FE0005F47065054345F46040640440F09A
:10E200000E0004F0FE44204309F070F94FF2A450D0
:10E21000C0F20E0009F064FDBDE83840FCF762BAB8
:10E2200038B505464FF2F0700C46C0F20E001221D0
:10E2300009F074F849F2A823C1F6FF7393F823306C
:10E24000FBB121462B460022D020FDF7EFFB4FF219
:10E250000850C0F20E00240409F042FD04F4FE044C
:10E26000681E44F45044000244F00D0400F4706051
:10E27000204309F03BF94FF2A450C0F20E0009F020
:10E280002FFDBDE83840FCF72DBA00BF2DE9F04F57
:10E2900087B005904FF604000491C0F20E001521DE
:10E2A00009F03CF849F2A823C1F6FF7393F8233034
:10E2B00023B907B0BDE8F04FFCF714BA43F6A05BF2
:10E2C000C2F2000BF021DBF848000368DB6C9847D2
:10E2D000049B002B00F0B8801A4648F23403C4F2C5
:10E2E0000403DBF848000093059B056848F2A55A33
:10E2F0004FF420461F461344C0F2000AC4F206063B
:10E3000099462B6817F8011B534540F09580009BF8
:10E310001B685C0560D542F25C43C2F201031B68D6
:10E320000BB10120187042F21443C2F2010342F211
:10E3300015451C7801343F2C88BF002042F2184854
:10E3400094BFE0B20446C2F20105C2F201082A7885
:10E35000A24233D1EFF31382002A57D1EFF3108298
:10E36000002A53D1EFF3058EBEF1000F61D0BEF14C
:10E370000F0F05D94EF2F032CEF20002724412783D
:10E38000EFF3118EBEF1000F02D0724528BF724626
:10E39000402A3BD9B2F5807FD9D142F64902C2F278
:10E3A00001021278002AD2D103930291019008F061
:10E3B000B5FE2A7801A8A2420BC8CBD042F258453C
:10E3C000C2F2010508F804100124BC212C70187059
:10E3D000F170DBF848000568B94592D1EB6CF72184
:10E3E00098474FF20850C0F20E0009F079FC0499EA
:10E3F0000598FCF70FFA4FF2A450C0F20E0009F096
:10E400006FFC07B0BDE8F04FFCF76CB9327912062B
:10E410009DD52A7801323F2A86BF4FF0000E724602
:10E420005FFA82FE18F80220D2B2F27185F800E09D
:10E430008DE74FF48072A3E79847DBF84800B945B1
:10E4400005687FF45EAFC9E7DBF848000568C5E7FB
:10E4500070B549F2A825C1F6FF750C4695F8223033
:10E46000064623B1984202D009F060FDC0B149F2DE
:10E47000A423C1F6FF731C70F9F7DEFB43F6F043EB
:10E48000C2F200034DF6003293F8AD1053F821307C
:10E49000597B03EB8103C1F6FF725B6893422DD079
:10E4A0004FF61C00C0F20E00122108F037FF95F85D
:10E4B0002330FBB1214633460022C020FDF7B6FAD7
:10E4C0004FF20850C0F20E00240409F009FC04F4D5
:10E4D000FE04701E44F44044000244F00C0400F4B6
:10E4E0007060204309F002F84FF2A450C0F20E0011
:10E4F00009F0F6FBBDE87040FCF7F4B8FCF7BCF897
:10E50000CEE700BF2DE9F04149F2A826C1F6FF761B
:10E510000C4696F8223015460746B3B3984234D0DD
:10E5200009F004FD88BB4FF63000C0F20E00122146
:10E5300008F0F4FE96F823301BB32A4621463B46EA
:10E54000B020FDF773FA2D064FF20850C0F20E000E
:10E5500005F0FE4509F0C4FB45F430452404781E5F
:10E5600045F00B0504F4FE0400022C4300F4706037
:10E57000204308F0BBFF4FF2A450C0F20E0009F098
:10E58000AFFBBDE8F041FCF7ADB85C2CCBD00CD8AC
:10E590000A2C29D05B2C50D105EB850000EB8000C4
:10E5A000C0F34710FBF71AFCBDE75D2C33D05E2C9F
:10E5B00043D107EE905A0023C4F2FE2306EE903AB0
:10E5C000B8EE676A0023C6EE267A07EE103A4BF2E1
:10E5D0002003C1F6FF7377EE877A18684368C3EDAE
:10E5E0000A7A02F051FE9EE707EE905A0023C4F229
:10E5F000FE2306EE903AB8EE676A0023C6EE267A4E
:10E6000007EE103A77EE877AFDEEE77A17EE903A4A
:10E6100086F8253087E705EB850808EB88084FF674
:10E620004410C8F34718C0F2010009F059FB4046F6
:10E63000FCF7BAF986F81C8075E74BF22003C1F6A7
:10E64000FF732A461868036821465B6898476AE7A3
:10E650002DE9F04F49F2A826C1F6FF7687B096F86B
:10E660002230029104920390D3B3984238D009F03B
:10E670005DFCA8BB4FF64400C0F20E00172108F065
:10E680004DFE96F8233033B3039E049D029C33461F
:10E690002A4621468020FDF7C9F94FF20850C0F202
:10E6A0000E0009F01DFB2B0603F0FE4343F400436C
:10E6B0002204701E02F4FE0243F00803000213431A
:10E6C00000F47060184308F011FF4FF2A450C0F23C
:10E6D0000E0009F005FB07B0BDE8F04FFCF702B8EB
:10E6E0004BF22003C1F6FF7396F909A0D3F800B0EE
:10E6F000029B9BF81020DBF804809A44002AB9D0D2
:10E7000005965C4600258027464604E00135AA426E
:10E7100004F134040FDDD4F8EC329A45F6D1DBF87D
:10E720008C3C53B1C4F8EC729BF810200135AA421E
:10E7300004F13404EFDC059E9CE7DBF80C0080F06C
:10E7400000400AF05DF9CDE9000150460AF046F9B3
:10E7500047F6E1234FF08042C3F684730AF0F4F9E0
:10E7600000230022C4F2180309F0ECFF736807EEDF
:10E77000103AF1EE047A67EE277A804617EE900A97
:10E7800089460AF03DF902460B464046494609F0E3
:10E79000D7FF41EC100B0EF0BFFEDDE9000153EC9A
:10E7A000102B0AF0D1F941EC100B0EF0B5FE51EC34
:10E7B000100B0AF079F9C4F8D4029BF81020A5E7F1
:10E7C00010B44FF48043C4F20C035A68940218D575
:10E7D00042F64702C2F20102D868137842F64801B5
:10E7E000C2F2010101333F2B0978C8BF00238B42DD
:10E7F00007D042F28801C2F20101C0B2DCB2C854B3
:10E8000014704FF48043C4F20C039A68100202D5CE
:10E810005B68190217D4520212D54FF48043C4F238
:10E820000C035B685B020BD542F288034FF4AC72B9
:10E83000C2F20103C4F28832002183F86C10116027
:10E840005DF8044B704742F28801C2F2010191F871
:10E85000400091F84130DBB2984211D00133272BB0
:10E8600086BF00242346DCB20B444FF4804093F86B
:10E870004430C4F20C00DBB2C36081F84140CAE707
:10E880004FF4AE714FF4AC73C4F28831C4F28833E4
:10E89000002401200C601860BDE700BF10B44FF4E5
:10E8A0002043C4F20E031A7992061AD542F64502A5
:10E8B000C2F20102D879137842F64601C2F2010190
:10E8C00001333F2B0978C8BF00238B42C0B208D068
:10E8D00042F28801C2F201011944DBB281F87000F2
:10E8E00013704FF42042C4F20E02D378DBB21C0640
:10E8F00014D459060FD54FF42043C4F20E031A79ED
:10E90000520608D542F28802C2F2010200202C21F0
:10E9100082F8DC00D9705DF8044B70471179080665
:10E92000E7D542F28800C2F2010090F8B04090F8BA
:10E93000B110C9B28C4211D04A1C272A86BF0024CC
:10E940002246D4B202444FF4204192F8B420C4F2DB
:10E950000E01D2B2CA7180F8B140CAE76C21D17001
:10E96000C7E700BF10B44FF45043C4F206031A794E
:10E9700092061AD542F64302C2F20102D879137800
:10E9800042F64401C2F2010101333F2B0978C8BFAE
:10E9900000238B42C0B208D042F28801C2F20101CA
:10E9A0001944DBB281F8E00013704FF45042C4F216
:10E9B0000602D378DBB21C0614D459060FD54FF4E7
:10E9C0005043C4F206031A79520608D542F288026F
:10E9D000C2F2010200202C2182F84C01D9705DF8AE
:10E9E000044B704711790806E7D542F28800C2F25D
:10E9F000010090F8204190F82111C9B28C4211D049
:10EA00004A1C272A86BF00242246D4B202444FF46F
:10EA1000504192F82421C4F20601D2B2CA7180F8A2
:10EA20002141CAE76C21D170C7E700BF10B44FF491
:10EA30004043C4F206031A7992061AD542F64102FF
:10EA4000C2F20102D879137842F64201C2F2010102
:10EA500001333F2B0978C8BF00238B42C0B208D0D6
:10EA600042F28801C2F201011944DBB281F850017F
:10EA700013704FF44042C4F20602D378DBB21C0696
:10EA800014D459060FD54FF44043C4F206031A7943
:10EA9000520608D542F28802C2F2010200202C215F
:10EAA00082F8BC01D9705DF8044B704711790806F3
:10EAB000E7D542F28800C2F2010090F8904190F848
:10EAC0009111C9B28C4211D04A1C272A86BF00245A
:10EAD0002246D4B202444FF4404192F89421C4F249
:10EAE0000601D2B2CA7180F89141CAE76C21D17097
:10EAF000C7E700BFF0B54FF43043C4F206031A79FC
:10EB000012F0300F2BD072B6997D01F0FF02002970
:10EB100040D062B642F63F0742F64001C2F201071A
:10EB2000C2F201013C780E7842F2880E1846E4B237
:10EB3000F6B2C2F2010E631C402BC17928BF00233C
:10EB4000B34202F1FF32C9B204D00EEB03051C46FA
:10EB500085F8C01112F0FF02EDD1E4B23C704FF421
:10EB60003042C4F20602D178C9B20D0617D4490664
:10EB70000FD54FF43043C4F206031A79520608D574
:10EB800042F28802C2F2010200203C2182F82C02EB
:10EB9000D970F0BD4022D9795A7462B6DFE7137993
:10EBA0001C06E4D542F28804C2F2010494F8005233
:10EBB00094F80132EDB2DBB29D4202D10EE0AB42DD
:10EBC0000CD00133282B28BF0023E018167990F8C9
:10EBD0000402C0B2D071107D0728F0D94FF4304242
:10EBE000DBB2C4F2060284F801321379180644BF7E
:10EBF0007C23D370BBE700BF2DE9F04F42F63C0306
:10EC00008DB042F2900242F2940142F298004FF429
:10EC100003544FF4025BC2F20103C4F20702C4F2D0
:10EC20000701C4F20700C4F20704C4F2070B0493FF
:10EC3000029207910B90099461E09908C1F6FF7563
:10EC400005EBC10602F1FF395FFA89F9726801919B
:10EC5000B9F1050FA2F1080000F0CA80B9F1060F62
:10EC600000F03981B9F1070F00F068811F0700F14A
:10EC70003581019B55F833301B0C99B222F8081CE2
:10EC8000002B00F01A8141F20003C2F201030024BC
:10EC900053F829E022F8064C42F8044C42F288046A
:10ECA000BEF1000F00F08A83C2F201044FEA89032B
:10ECB000E218D2F84C22506041F22008C2F201085A
:10ECC0001C4438F81930C4F84C02194428F81910BB
:10ECD00008F000FB002800F06683C822C0F2400262
:10ECE000882316F0080FC0F2400318BF1346019A9C
:10ECF0000830706045F8323008238BF800309BF8FC
:10ED00000040E4B2620735D5049B1B787BB342F226
:10ED10008803C2F2010393F8381201F0FF0229B10F
:10ED2000013AD2B283F8382202B900BE42F6590540
:10ED3000C2F201052A7802F0FF032AB1013BDBB2DF
:10ED40002B70002B00F0C58242F65A03C2F2010379
:10ED50001E7866B942F65C05C2F20105286830B13A
:10ED6000438823B19B000380FBF708FD2E6004233A
:10ED70008BF8003004F0080303F0FF02002B00F0D2
:10ED80004181029B1B78DBB21A0940F200057FF437
:10ED900054AF9B08C1F6FF7505EBC30055F833105F
:10EDA0004068C1F38301092900F04C8100F2DD8045
:10EDB0000139012918D842F28804C2F2010442F252
:10EDC0002102B4F83C12914200F01C8394F83C12EA
:10EDD00042F288022129C2F2010200F03382C822E5
:10EDE000C0F2400245F83320079A0123137083E7ED
:10EDF00019077FF53EAF49F2B843C1F6FF731A6AAF
:10EE00000132082A00F215828021C0F2B0011A6294
:10EE100003914FF02C0A42F28804C2F2010448F632
:10EE20008803C1F6FF73D4F88002CDF818B04FF014
:10EE30000009019305969B46C9EB0A03002800F0E0
:10EE4000A782B4F888C2D4F88482CCF180029342BD
:10EE500028BF1346061D4FEA4C0208F1040E164463
:10EE600096444FEA890763B1043F5F441D463EF96B
:10EE7000021B36F8022B013D42EA014247F8042FFB
:10EE8000F5D19C44BCF17F0F994400F20B82A4F8A9
:10EE900088C2D145D0D3059EDDF818B0019A86F01E
:10EEA000080640F64C737260C2F20103039A3260A6
:10EEB0005A7982F001025A711EE7C822C0F240025C
:10EEC000882316F0080FC0F2400318BF1346019ABA
:10EED00045F8323010E71B0740F1F98008F04EF991
:10EEE00040F65473C2F2010353F82920002A00F0BF
:10EEF000788240F64C70C2F20100516810F8094067
:10EF000043F82910012C02F10803736000F05D82C0
:10EF1000C0F06382022C00F05C82032C02D1042337
:10EF200000F80930128816F0080F0CBF8823C82398
:10EF300043EA0243019A45F83230DDE61C077FF5CB
:10EF400098AE86F0080648F68403C1F6FF73736036
:10EF5000802240F64C73C0F20302C2F20103326019
:10EF6000DA7982F00102DA71C6E60D297FF43CAF4E
:10EF700090E84200C820C0F2400042F28804C2F289
:10EF8000010445F833008BB20120B3F5086F2A6104
:10EF9000AA61C4F84062C4F83C12C4F8442284F860
:10EFA000480200F0A48340F21C8142F221329342D5
:10EFB00000F09A8300F2AD8240F60132934200F0F5
:10EFC000958200F2F982B3F5106F00F0FF8340F6EE
:10EFD0008122934240F02281B4F8403242F288020A
:10EFE000042BC2F2010200F01D85052B40F01681B2
:10EFF00092F8723282F830320120B2F8423202F5D1
:10F000000C727CE3E00700F17C81210600F1308284
:10F01000A2070CD542F28803C4F207034FF4025151
:10F020001A78C4F20701D2B202201A700870E306FF
:10F0300005D54FF40253C4F2070310221A700DB025
:10F04000BDE8F08F42F28804C2F20104D4F84432E1
:10F050005BB3B4F8742294F8480294F87312402A0F
:10F06000164641F0020728BF4026002880F0010024
:10F07000A2EB06020CBF4FF0880E4FF0C80E84F8CA
:10F08000480205EBC70092B24EEA064E81F001013C
:10F090004360A4F8742245F837E0334484F87312CF
:10F0A000002A00F0C280C4F84432B4F83C2242F294
:10F0B0008803B2F5A06FC2F201037FF495AE002180
:10F0C00093F83E2283F83D120B9B1A708CE642F2B5
:10F0D0008804C2F2010455F83130D4F89892B4F89B
:10F0E000942203929B0CD4F89C8205921F46B9F19E
:10F0F000000F00F06E84B8F1000F00F06084002F64
:10F1000000F01285039BC3F1800A574548F2D07383
:10F11000C1F6FF73C0F0EC8442F288020A930893B0
:10F12000C2F20102D4F8A03206920393BAF1000FA2
:10F1300029D11BB9D4F8A432002B3FD00A9A7260AF
:10F140008023019AC0F2B40345F83230D4E503902D
:10F1500005F0A6FD039B8046002800F01282069968
:10F160000A46C1F89832C2F89C02002F00F01382C0
:10F1700000227F2FCDF80C9005924FF0800A88BFB7
:10F18000994640F2ED81059B08985B0008F1040266
:10F1900009F104011A441944534607F085FF089BFE
:10F1A00003EB8A030893039BCAEB0707002B40F08D
:10F1B0008482D4F8A432002B40F07F82C4F8A0925D
:10F1C000C4F8A48205F06CFD42F2880AC2F2010A7A
:10F1D0000028BCD1CAF89802CAF89C02AAF8940286
:10F1E000ACE740F20232934200F0D78200F2508145
:10F1F000B3F5817F00F0C78300F25D84802B00F0BF
:10F20000B583822B0AD1B4F8403203F07F0342F277
:10F210008802082BC2F2010240F2E883099A0F2308
:10F220001370079A01231370DEE5402E18BF0023E8
:10F2300039E780210022C0F2B4011A6203914FF035
:10F240002D0AE8E592F83F1292F83D22012900F0DC
:10F25000A88102297FF4C3AD012A7FF4C0AD4678AE
:10F26000007849F2B841C1F6FF7100EB06204A610F
:10F27000C86194F8731294F8482241F0020081F0BA
:10F280000101002A84F8731282F0010205EBC0012B
:10F2900084F8482214BFC8248824002245F830404E
:10F2A0004A609CE505F0D2FC404605F0CFFC4FF0EB
:10F2B0000002D4F88C02D4F89032A4F888220022FC
:10F2C000C4F88002C4F88C22C4F88432C4F89022B6
:10F2D000DFE542F65203C2F201031B7803F0FF0799
:10F2E000002B7FF431AD42F65406C2F201063068BD
:10F2F000002800F0E78143880380FBF703FA3760BA
:10F3000022E542F2940042F28801C4F20700C2F200
:10F31000010140F20003C1F6FF730224047081F87A
:10F32000732201F52A7401F53A71D9604FF4035C38
:10F330008821C0F24001C4F2070C42F2880E5C60E2
:10F34000196099601A619A61C4F2070E0D234FF497
:10F35000025742F2980642F28C0542F284048CF87D
:10F360000030C4F20707FF23C4F20706C4F2070502
:10F37000C4F207048EF8003001214FF09F0E3B705D
:10F3800032702B7084F800E001700DB0BDE8F08F92
:10F390009A00019B059EDDF818B0014603EB490079
:10F3A00009F03EFE7AE542F65103C2F20103019AEA
:10F3B00045F832001A7801321A709DE443F82900AA
:10F3C000C2F201044FEA890376E4022300F809300F
:10F3D000A8E5052300F80930A4E5032300F8093067
:10F3E000A0E540F64C77C2F2010717F80930022B6E
:10F3F00079D0FFF481AC032B40F06D81012307F835
:10F40000093079E402784678817884F87822C278E5
:10F4100084F8796284F87A1284F87B220179D4F82E
:10F420007822467984F87C12817984F87D62862A74
:10F4300094F8486284F87E1294F8731204BF0F2285
:10F4400084F8382241F00202002E81F0010184F894
:10F4500073120CBF8821C82145F8321005EBC20297
:10F4600086F001060021073084F848625160ADE45F
:10F470004FF40352C4F207024FF40253C4F20703DD
:10F480000D2010708021A20719707FF5D0ADC1E565
:10F49000B3F5A06F00F0288140F20183A3F5D0639B
:10F4A000012B3FF6BBAE49F2B8424FF65C03B4F80D
:10F4B0003E02B4F84062C1F6FF72C0F20E0304E0EF
:10F4C0000C335A68002A3FF4A9AE19888142F7D15B
:10F4D0005988B142F4D1000A032814BF1889107862
:10F4E000B4F842320BE107F8092005E4B4F84022F1
:10F4F00042F28803042AC2F2010300F09D82052A29
:10F500007FF48CAEB3F83E2283F8722200210120F2
:10F5100069E048F2A122934200F0138100F20881D1
:10F5200048F2A112934200F00C8148F2A2129342D9
:10F530007FF474AEB4F8423242F28802022BC2F277
:10F5400001027FF66BAE4421AC2082F8301200211C
:10F5500082F8310282F83212032002F50C72CEE0FA
:10F56000002203921146043308F104020A44089869
:10F5700019443B4607F098FD039B3B44A4F89432A2
:10F58000DCE5184605F062FBCAF89882CAF89C824E
:10F59000AAF89482D2E50397BDF80C30A4F894320F
:10F5A000CCE5012A7FF41BAC49F2B841C1F6FF71EA
:10F5B000007888614A615CE642F2210293423FF49E
:10F5C00030AE42F2212293427FF428AE4DF27443D2
:10F5D000C1F6FF7394F83E221B68C4F86C32002118
:10F5E00084F87022012000239C461F469E461A463E
:10F5F00094F8736246F0020805EBC8090028C9F8C0
:10F6000004200CBF8822C8223A4342F2880940F203
:10F61000000745F8382086F0010284F84812C1F648
:10F62000FF77C2F2010984F8732213BBBEF1400FC9
:10F630007FF4F7AD42F0020205EBC20540F200078D
:10F64000C5F804C0C1F6FF7749BB190441F0880131
:10F6500047F8321084F8480284F873620CEB030018
:10F66000402B7FF4DEAD0023C4F84402A4F87432CA
:10F67000D7E5402BDED942F0020207EBC205C5F800
:10F6800004C0C1B1C821C0F2400189F84802403B22
:10F6900089F873620CF1400047F83210E4E719046E
:10F6A00041F0C80184F8480284F873620CEB03004F
:10F6B00047F83210D4E78821E5E7059B5344A4F8C6
:10F6C00094323BE507F006FE002800F0A781FBF727
:10F6D00019F8FFF739BB16F0080F0CBF02230323FC
:10F6E00007F80930FFF708BB002101207BE7049BE6
:10F6F0001B7884F83032B4F8423204F50C7283423D
:10F7000080F0FD8194F8736246F0020805EBC801B1
:10F71000402B9E4628BF4FF0400E4A6002EB0E0C75
:10F72000CEEB03034FEA0E4700210120C8226BE70E
:10F7300048F2A132934204D048F2A14293427FF4AE
:10F740006DAD94F83C3242F28802A12BC2F2010264
:10F750007FF464AD92F83F02012800F0F1810228A5
:10F760007FF45CAD92F83D32812B00F0F181822B69
:10F7700000F02782832B00F01D82842B7FF44EAD96
:10F780000121002382F8301282F8313242F2B8228D
:10F79000B4F84232C2F20102B1E7B4F8403203F0E9
:10F7A0007F03082B3FF63AADB4F83E22002A7FF4DF
:10F7B00035AD4FF403529B00C4F207021A440021F6
:10F7C000137843F00203137001200CE740F20006A7
:10F7D000049A94F83E321370C1F6FF7606F58077EE
:10F7E00002E00836B74207D0336A1B06F9D5706AC3
:10F7F000083807F0C3FCF4E740F64C7340F670722B
:10F8000041F2000940F6547A41F22008C2F20102A6
:10F81000C2F2010301950027C2F20109C2F2010AF6
:10F82000C2F2010816461D460394D9F8000028B11B
:10F83000446807F0A3FC2046002CF9D10023C9F846
:10F84000003042F2D423C2F20103DAF800000022B1
:10F8500043F8272028B1446807F090FC2046002C8C
:10F86000F9D12B780022032BCAF8002046F8042F88
:10F8700028F8172004D06DD9042B6DD0052B02D1A8
:10F880004FF001032B700137082F09F104090AF129
:10F89000040A05F10105C8D142F65103C2F2010381
:10F8A000039C019D01931A4642F2C40A00234FF6BD
:10F8B000E869C8218820C4F2070AC0F20E09137053
:10F8C000C0F240012346C0F2400054460391CA46AC
:10F8D00005904FF002080127994616E0BE0046F059
:10F8E000020246F00306002040F20003082F45F80C
:10F8F0003200C1F6FF7345F8360000F03481B8F1EC
:10F90000090F2DD0013708F101081AF8013B04F85E
:10F91000043B072F00F039811E07DFD507F0DAFC22
:10F92000002800F0DD8005EB4713BE00083058606A
:10F93000059B45F8363007F0CDFC002800F0C78065
:10F9400046F0010305EBC3020830039945F8331074
:10F950005060C4E7022B96D14FF000032B7092E762
:10F9600099F848024C4680F001013CE6002342F23F
:10F97000B82284F8303284F83132C2F20102B4F88D
:10F9800042320220BBE6B4F8403203F07F0342F279
:10F990008802082BC2F201023FF640ACB2F83E12D8
:10F9A00000297FF43BAC4FF403529B00C4F20702E2
:10F9B0001A440120137823F00203137013E605F0B4
:10F9C0006FF98046002800F0A880C4F89C02FFF779
:10F9D00096BB05F065F98146002800F09E80C4F8CA
:10F9E0009802B8F1000F7FF48AABE8E74FF40351B7
:10F9F0009B00C4F207011944002382F8303282F8D8
:10FA000031320B78980740F19580012382F830322B
:10FA10000220B2F8423202F50C7270E601232B701C
:10FA2000FFF792B992F8713282F830320120B2F8C1
:10FA3000423202F50C7262E693F83E1283F87112BC
:10FA400000293FF452AE40F64C77C2F2010740F273
:10FA5000D803C1F6FF7397F80590A3F10806B9F132
:10FA6000000F18BF1E46316811F080087FF43CAECD
:10FA700048F68803C1F6FF7318464146B0229A46FD
:10FA800009F0CEFA802389F00109C0F2B003C6F86C
:10FA900004A087F80590414633600120A3E540F2B9
:10FAA000213293423FF4BDAB40F2214293423FF4F6
:10FAB000B8ABFFF7B3BB40F2211293423FF4B1ABB6
:10FAC00040F2212293423FF4ACABFFF7A7BB019970
:10FAD0000B7846F00102013345F832000B70FEE668
:10FAE000019A1378BE00013345F83600137022E7FF
:10FAF0001A460892039A0A9351004B4633E5402870
:10FB0000864628BF4FF0400ECEEB00034FEA0E476B
:10FB100002EB0E0C002101206AE548F2D073C1F619
:10FB2000FF730A93FFF70ABB48F2D073C1F6FF7365
:10FB30000A9331E5B2F84232022002F50C72DEE59A
:10FB400049F2B843C1F6FF739B6982F830321DE673
:10FB500049F2B843C1F6FF73DB6982F830321B12F9
:10FB600082F8313212E68021C0F2030103EBC206B3
:10FB700043F8321099F8480248F68403C1F6FF733F
:10FB80004C46736080F001012DE548F2D073C1F658
:10FB9000FF738022C0F2B402C5F8E430C5F8EC303F
:10FBA0000023C5F8E020C5F8E820C5F8F030C5F816
:10FBB000F830A7E6FF210F2382F8301282F83132A5
:10FBC000E4E5002382F8303282F83132DEE500BF0E
:10FBD00041F23801C4F20B0141F230020B6823F00C
:10FBE000805323F00A030B60C4F20B0213689907D9
:10FBF000FCD541F22C03C4F20B031A68920703D51B
:10FC00001A6822F002021A6041F22803C4F20B03C0
:10FC100042F2B832196821F0080119601968C2F27D
:10FC2000010241F00801012019601060704700BF17
:10FC30000020704770B449F26073C1F6FF7348F258
:10FC40001F02996BC4F2000208791070586B48F2D9
:10FC50001C02C4F2000204791470097911701A6B45
:10FC6000002A4FD05968C9688A4247D80168CC8BAE
:10FC7000240402F1FF3069D4C0F30E00C883C88B9E
:10FC800080B2C882996B0968C88B000456D4C2F34D
:10FC90000E00C883C88B002480B212F1FF32C882E4
:10FCA00018BF01221C63596B086849F2607105682E
:10FCB000C1F6FF7101F12C04A54237D00968CC6868
:10FCC00014F0804F0468056815BF24882478023535
:10FCD000013544F0004405604C63996B48F21B0306
:10FCE000C4F200030979197049F26071C1F6FF711D
:10FCF00012B14A6B12791A7070BC7047521A1A63AB
:10FD00000122D0E71968D86B0A630024CFF60F747C
:10FD1000CC62CC68066824F08044CC60346803254B
:10FD200083F82D501146234670BC1847086891F897
:10FD30002C10C46841F000414163CEE7CC8BC2F384
:10FD4000080004F47E442043C883A3E7CC8BC0F3AF
:10FD5000080004F47E442043C88390E700B583B0D4
:10FD600002A800F8011D012107F0D8FA03B05DF8E0
:10FD700004FB00BF90F89D3090F89C20DBB29342CA
:10FD800014D001331F2B84BF00210B4610B598BF40
:10FD9000D9B2063350F8234080F89D102146FBF776
:10FDA000CBFE2046BDE8104004F050BF704700BFB6
:10FDB0002DE9F04F436AC469866985B02BB906EB1B
:10FDC000C414846105B0BDE8F08F0546076A04F0ED
:10FDD00067FF0290002800F0E680F219B5F9323092
:10FDE0000192029A042B02F1040E00F0EE8054DD21
:10FDF000062B00F07A81C0F26381072B00F00881A6
:10FE0000082B73D1AA6ACDF80CE04FEA520C130C00
:10FE10006FEA0C021146029AD5F82480C3F57F4B95
:10FE20004FF0FF39901D764602F5837A0BF1FF0BF8
:10FE3000019AB9FBFBFB8E46B9FBF3F921E0CCEB51
:10FE400002073F0C4FF6FF710BFB07F7C7F6FF7178
:10FE500002EB0C03C91B1B0C091409FB03F308FB81
:10FE600001F103F1004396454FEA21414FEA234354
:10FE700070D9318002305045224406F1020600F06C
:10FE80004281130C09FB03F31B0C08FB03F36245CF
:10FE90004FEA1343D3D23380ECE7012B00F0888084
:10FEA0005DDD022B43D0032B20D16F6A019802F550
:10FEB000827C7646C30BC3F57F43C113FF3307FB38
:10FEC00003F34FEA907807FB01F11A0C091408F1CB
:10FED000FF33012B94BF13460B4626F8023B6645C1
:10FEE0002044E7D1019B03EBC41301932C6A019AD0
:10FEF000B5F93430141BAC6173B1029A02F582710A
:10FF000001E0B5F93430BEF90020134403F30F03C8
:10FF10002EF8023B7145F4D8029C28462146FBF797
:10FF20000BFE204605B0BDE8F04F04F08FBE686AB6
:10FF300020F34F0002F58276019A07B273464042E1
:10FF400037EA220128BF014623F8021BB3422244AC
:10FF5000F6D1C7E708FB03F31B1433808AE7002BB5
:10FF6000C4D14FF6B806D5F824C00199C0F20E06E8
:10FF700002F5827770460B0E5A1C36F9138036F95B
:10FF80001220C1F30F29C9F5803308FB03F309FBE5
:10FF9000023353FB0CF320F8023BB8422144EAD170
:10FFA000A0E704F053FEAB6903EBC413AB6109E7B0
:10FFB00002F582706E6A019A734636FB12F123F8DD
:10FFC000021B83422244F8D18CE7EE6A002EE8D06F
:10FFD000D5F824C0019902F5827770460A0E531CA9
:10FFE000B3F5807F14BF5B000023C1F30F28F35EDD
:10FFF00036F9122008FB03F3C8F5803808FB0233FA
:020000021000EC
:1000000053FB0CF320F8023BB8422144E6D169E7E8
:1000100042F2B033C2F2010303931E68029B0199BE
:1000200040F65F384FF21D3A4FF2EC4BC8F24E38B3
:10003000C0F2010ACFF6FF7B03F5827C77460022EF
:1000400001E0674532D0B5F9303027F8023B61183E
:10005000F7D3686A18B326B386FB082388FB069299
:1000600033444FEAE6793244C9EB2343C9EB2242D9
:100070000AFB13660BFB02F244F2A71303FB0626EE
:10008000002E02DA06F10046013EB6FBF0F300FB5B
:1000900013639BB20122A3EB60032B86D1E70346D7
:1000A000F9E74CF64266C1F60C76EEE7019B03EBEE
:1000B000C4130193002A3FF419AF039B1E6015E798
:1000C000686A20F34F0002F58276D5F828C0019ABD
:1000D00007B273464042624534BF3946014623F8B1
:1000E000021BB3422244F6D1FCE6686A02F582762E
:1000F000019AC043734630FB12F123F8021BB3424E
:100100002244F8D1EEE6019BDDF80CE003EBC413CA
:100110000193EBE602783F2A0BD84EF6D023C0F2CB
:100120000E0353F8321091F8800270B3012381F866
:10013000803042F2B433C2F201031A7822B349F29A
:100140006072C1F6FF720020D17A18700B46D9B1E7
:10015000C80706D54FF46143CEF20003D06918609A
:100160000B46880706D54EF20413CEF20003116A3F
:100170001960D37A590710D41B0705D54EF20C131A
:10018000CEF20003926A1A60704703EBC2035A680A
:10019000136843F003031360CBE74EF20813CEF26B
:1001A0000003516A1960D37AE6E700BFF0B54DF25B
:1001B0007446C1F6FF7683B0336801934FF4404430
:1001C000C4F20204019F0546A4464FF0004EFF20F2
:1001D000236843F480632360C4F82CE06063E36A1F
:1001E000002BFCDADCF83830DBB2FF2B06D03368AA
:1001F0000093009BDB1BB3F5967FE9D34FF440439C
:10020000C4F202034FF00046186841F0400440F485
:1002100080601860DE6218465C63C36A002BFCDAFB
:100220004FF44044C4F2020418204FF000472668FF
:1002300022FA00F346F48066DBB22660E76263636D
:10024000E36A002BFCDA083810F1080FEFD100291F
:1002500032D008290CBF8721FF214FF44043C4F25C
:1002600002034FF000401A6842F480621A60D862BC
:100270001A465963D36A002BFCDA4FF44042C4F2A9
:100280000202164600274FF00044FF21136843F492
:1002900080631360D4625163D36A002BFCDAB36BC2
:1002A000D8B21B06687001D403B0F0BD0137B7F5B2
:1002B000807FEBD103B0F0BD9521CEE72DE9F04171
:1002C000064682B0002900F0D08042F2B43583782F
:1002D000C2F20105032B2B78144618BF4902002BEC
:1002E00060D032783F2A0DD84EF6D023C0F20E03EC
:1002F00053F8320090F88072002F00F0BB80012389
:1003000080F800310A4630461821FFF74FFF0028D9
:1003100000F0BF8032783F2A0CD84EF6D023C0F2CE
:100320000E0353F8321091F88002002832D00123D6
:1003300081F880302B7842F2B432C2F201022BB342
:1003400049F26073C1F6FF730020D97A10700A4633
:10035000E1B1CC0706D54FF46142CEF20002D86974
:1003600010600A46880706D54EF20412CEF200024B
:10037000196A1160DA7A510700F1BE80120705D5BB
:100380004EF20C12CEF200029B6A1360002002B003
:10039000BDE8F08103EBC2035A68136843F003031E
:1003A0001360C7E749F26073C1F6FF734DF2803204
:1003B000C1F6FF72D87A126801272F7000283DD04D
:1003C00072B6DF7A17F0010F38460DD04EF2801C5E
:1003D000CEF2000CD868DCF800E00EEA000EC3F89C
:1003E0001CE03846CCF800E0BF070BD54EF2841E67
:1003F000CEF2000E1F69DEF8000038401862CEF819
:100400000000D87A47070BD54EF2881ECEF2000EB8
:100410005F69DEF8000038405862CEF80000D87AF4
:1004200007070AD54EF28C1ECEF2000E9F69DEF849
:10043000000038409862CEF8000062B61B68D868A9
:1004400090423FF44EAF44F20107C0F23F07002054
:100450001F60C8F23F0042F08047DA601F611860F9
:1004600032783F2A7FF640AF4CE742F2B435C2F211
:1004700001054FE703EBC20330465A68136823F0C7
:10048000020313600A461821FFF790FE00287FF44C
:1004900041AF21463046FBF76BFB00283FF43AAFF3
:1004A0004DF27441C1F6FF714FF440420B68019365
:1004B000C4F20202DDF8048094464FF0004EFF20A3
:1004C000136843F480631360C2F82CE05063D36A6E
:1004D0004FF44044002BC4F20204F8DADCF8387020
:1004E000FFB2FF2F10D00B680093009BC8EB0303F3
:1004F000B3F5167FE4D30DE74EF20812CEF20002F8
:10050000596A1160DA7A39E700220D213046FFF787
:100510004DFE00287FF4FEAE23684FF0004243F406
:10052000806323602146E2626763CA6A4FF44043F6
:10053000002AC4F20203F8DA9B6B13F0FF0F7FF47A
:10054000E9AE3046FFF7E6FD012020E7830740F0E3
:10055000B2802DE9F04142F2BC35C2F2010582B011
:100560002B781BB1032002B0BDE8F08141F22402D8
:10057000C4F20B0214461368DF07FCD423689E07FD
:10058000F9D46B7803B9490241F23003C4F20B038A
:1005900041F234021C681C60C4F20B0241F23804C0
:1005A000136823F4081323F0310343F0805341F21E
:1005B0002C06C4F20B0643F00A03C4F20B041360CA
:1005C0002368376842F2B83247F002074FF4805E82
:1005D0003760C2F20102C4F20B0E41F20807C4F206
:1005E0000B0700261660CEF8000041F2040641F227
:1005F0000C00396043F08053C4F20B06C4F20B00C8
:10060000012143F00A034FF48137C1F6220137601C
:10061000236001601368002BFCD041F23003C4F268
:100620000B0341F22402196801F003011960C4F2BE
:100630000B0213685907FCD441F2240141F2300245
:10064000C4F20B01C4F20B0241F2340741F2080874
:1006500041F20C0C41F210068E461446C4F20B0710
:10066000C4F20B08C4F20B0CC4F20B060B68DB07D8
:10067000FCD4DEF800309807F8D438686B68019332
:1006800040F001003860136813600020019BC8F837
:100690000030C0F60250CCF800001368DB07FCD530
:1006A000236803F001032360306810F40070DDD18B
:1006B00002B0BDE8F0814FF0FF3070472DE9F04FF8
:1006C000827987B0012A83468DF80F1006D0012267
:1006D0008BF80420002007B0BDE8F08F4279900726
:1006E000F5D55307DBF80C4030D5DBF81860B44281
:1006F0002CD0002E00F00E81DBF820E09EF81020B8
:10070000611E02F10900721EC140C240914200F216
:100710000981002C00F00681DBF80850521A1446BB
:100720000BF1080708E001F0E5FC013C0028CED001
:10073000DBF820E0DBF8085029463A467046002CEA
:10074000F1D1CBF80C6034462E4603E0DBF80860AC
:10075000DBF820E041F2300342F2840249F2B44A6D
:10076000C2F20103C2F201020193C1F6FF7A0292C2
:100770000DF10F0801279EF80450013D05EA5425AC
:1007800015F0FF05C4F308040AD14CB9002E40F05F
:100790009680DBF81C60002E00F0AA80CBF8086081
:1007A000C4F500721FFA82F9B94530D99EF81010CD
:1007B000DEF81420023E06FA01F115440D441FFA3A
:1007C00087F92CB9DBF80C60DBF81800864269D297
:1007D0002846012101F02CFC00283FF478AF019B52
:1007E0004D46E0184219904205D0141A414622465F
:1007F00009F0ECF8A044DBF80C407F1B2C44CBF84C
:100800000C4031D0DBF80860DBF820E0B3E79EF85D
:100810001000DEF81410023E86400D44B9F5007F4A
:100820003544CED1DAF80020954204BF4FF0FF32B4
:10083000CAF8002042F2CC32C2F201022946106806
:100840000278FE2A5FD04246FFF738FD00283FF4C9
:100850003EAFDBF80C404FF400752C447F1B08F5CD
:100860000078CBF80C40CDD1DBF8182094429BF8EF
:10087000052005D942F08002CBF818408BF80520FE
:1008800011070BD59BF8061000293FF420AF120684
:100890004DD401F0C1FB00283FF419AF012007B08F
:1008A000BDE8F08F01F0B8FB00283FF410AF029ACA
:1008B000CAF80050117841F0010111708FE73146FC
:1008C000704605AA01F016FC00283FF404AFDBF8DF
:1008D00020E0059E9EF820004FF6F872C0F6FF72E9
:1008E0004FF6F871102808BF0A469642FFF456AF3B
:1008F0005846FBF7B3F900283FF4E9AEDBF820E0F7
:10090000DBF808604CE74046FFF720FEB0FA80F0C5
:1009100040099BE7CBF80860CBF80C60DBF820E0DF
:10092000344617E7DBF81C50CBF80850F7E60121F6
:10093000DBF8100001F07CFB00283FF4C8AE41F268
:1009400030029BF81410C2F2010212EB41123FF484
:10095000BEAE9BF8061001299CBFDBF81810D161D0
:10096000DBF81C105183090C91829BF8052002F0E2
:100970007F028BF805208CE72DE9F04F2DED048BDD
:10098000844685B00CF6984300F6A84400F6C445AA
:1009900000F6AC4900F54B6893ED001A94ED000A9F
:1009A000D5ED004A99ED003AD8ED003ADCF87CEC40
:1009B0009FED9E5ADFED9E9A0CF6944300F6A440FC
:1009C0001C460CF5496BD0ED000A02930CF69C40D6
:1009D0000CF54A6393ED008ADBED002A94ED004AA2
:1009E000D0ED008A02F1FE030239A2F1020A01935E
:1009F000F6EE001AB7EE002ABFEE009ABEF1000F25
:100A00009FED8C6A40F30481DCF8806CF0EE465A6E
:100A10000CF53C70002550F8307C50F8343C50F810
:100A20002C2C50F8284C3B4402EB234201359BB25E
:100A3000A2422DB240F82C2C40F8303C04DD50F896
:100A4000244C121B40F82C2C06EB420436F91220E1
:100A5000B4F9027010ED087A50ED076ABF1A03FB73
:100A600007F302EB234307EE903AF8EEE77A67EEDE
:100A7000266A67EE877A40ED086A67EE857AF5EEBA
:100A8000C07AF1EE10FA0EDD24EEA77AE7EEC77A0F
:100A9000B0EE677AF1EE667AB4EEE77AF1EE10FA2C
:100AA00058BFF0EE477A50ED036A10ED027A7545B3
:100AB000E7EEA65A00F13400A7EE876AABDB36EE0C
:100AC000637A75EEC37AE7EE003A029BA7EE803AAE
:100AD000E1EE042A36EE637AA2EEC14AA7EE206A5E
:100AE00075EEC37A26EE087AE7EEA05AA4EE076AFE
:100AF00065EEA87A26EE216AE4EE275AB4EEC26AC1
:100B0000F1EE10FA89ED003A65EEA15AC8ED003A0F
:100B1000CBED002A83ED004A6CDD47F6FF73F4EE5F
:100B2000C25AF1EE10FA57DD47F6FF722AF8022F8B
:100B300021F8023F019B9A457FF460AFDFED3E7ADA
:100B4000B0EEC33AB4EEE73ADFED3B7AF1EE10FADD
:100B5000F0EEE33A48BF0023F4EEE73A48BFC9F8A5
:100B60000030F1EE10FA44BF0023C8F80030BEF1A7
:100B7000000F2CDD00239FED317A1E46342706E05E
:100B8000DCF87CEC013636B2764533461FDA07FBDB
:100B900003C3D3EDB47A0EF1FF3EF4EEC77A07FB40
:100BA0000EC4F1EE10FA04F52F7403F52F75E7D596
:100BB0000FCCCCF87CEC0FC50FCC0FC50FCC0FC5FC
:100BC000013636B223682B6076453346DFDB05B04D
:100BD000BDEC048BBDE8F08FF4EEC95AF1EE10FACB
:100BE00019D465EEA95AFDEEE57ACDED037ABDF98B
:100BF0000C209BE7B4EEC96AF1EE10FA10D426EE91
:100C0000296AFDEEC67ACDED037ABDF90C3086E790
:100C1000F0EE465A53E748F20102CFF6FF7285E73D
:100C200048F20103CFF6FF7379E700BF00000038F8
:100C300000FEFF4600000000FFE6DB2E17B7D138AC
:100C400049F63003C1F6FF73012270B5596902718C
:100C5000002283F8382083F8392083F85C2083F859
:100C60005D2083F85E2083F85F200D6804462E68BF
:100C700048685A6630439A6628601869827093F80B
:100C800061200D680A444EF6D020167A527BC0F2DD
:100C90000E0000EBC6061202766802F4E06242F033
:100CA0006402326093F862200A44967CD27D00EBA5
:100CB000C6001202406802F4E06242F06402026080
:100CC00028684A68104205D01A692C2151701A69A7
:100CD000042191711A69202151711B6980229A7037
:100CE000052002F089FF44F260023021204605F021
:100CF000D3FD0546002859D06C222621204605F058
:100D0000CBFD4FF4F9722821204605F0C5FD40F6D1
:100D100022722C21204605F0BFFD44F246423C21C0
:100D2000204605F0B9FD40F237122421204605F097
:100D3000B3FD44F2FF023021204605F0ADFD7322E1
:100D40000221204605F0A8FD4FF4C87002F054FFC0
:100D500041F61D522E21204605F09EFD042211462B
:100D6000204605F099FD4FF498720621204605F0C3
:100D700093FD10220A21204605F08EFD00220E214F
:100D8000204605F089FD43F63C421021204605F03F
:100D900083FD47F67F722221204605F07DFD362235
:100DA0002421204605F078FD01236372284670BD9A
:100DB000437AFBB1036970B40646186800221A60D2
:100DC000B8B1B6F91E40B6F92010031D00F58275C2
:100DD00033F9022B9442A8BF14469142B8BF114682
:100DE0009D42F5D80123F4833184337770BC03F03E
:100DF0002DBF70BC704700BF41689FED157AD1EDE3
:100E0000056ADFED147AE6EE877A45F2A65242F2E1
:100E10004B43C4F22C72C3F2BE7310B58260C36040
:100E2000044617EE900A07F0EBFD41EC100B0CF0B6
:100E300073FB51EC100B07F037FEDFED077A07EE7E
:100E4000100A67EE277A04F69844C4ED007A10BDC4
:100E50003D0AC7403D0A27C025551539036A002BB6
:100E600000F009822DE9F04F044691B0002103F013
:100E70006DFF637A012B054640F2FE812369002253
:100E8000D3F804C05A600430002D00F0FB81BCF19F
:100E9000000F00F0F5814FF0000BB4F92430216A07
:100EA0009FEDEB3ADFEDEB3A96460CF1020605F5C5
:100EB0008277F6EE004AB7EE005AB0EE004AC4F26E
:100EC000400B4FF0814A90E09DED0A6AF4EEE67A1D
:100ED000F1EE10FA07D8F4EEC67AF1EE10FAB0EEA1
:100EE000467A80F25881F4EEC67AF1EE10FAF0EE0E
:100EF000466A80F27681DDED0B5AF4EEC67AF1EEA9
:100F000010FA07D8F4EEE75AF1EE10FAB0EE657A6F
:100F100040F27181F4EEE75AF1EE10FAF0EE656AF4
:100F200040F26C819DED0C6AF4EEE75AF1EE10FA96
:100F300007DBF4EEC67AF1EE10FAB0EE467A80F2F4
:100F40006781B4EEE76AF1EE10FAF0EE466A40F21D
:100F50006281DDED0D5AB4EEE76AF1EE10FA07DBBF
:100F6000F4EEE57AF1EE10FAB0EE657A80F25D818A
:100F7000F4EEE75AF1EE10FAF0EE656A40F25881AD
:100F80009DED0E6AF4EEE75AF1EE10FA07DBB4EECF
:100F9000E76AF1EE10FAB0EE467A40F25381F4EED1
:100FA000C67AF1EE10FAF0EE466A07DB9DED0F7A95
:100FB000F4EEC77AF1EE10FA40F24781F4EEC67A09
:100FC000F1EE10FA07D89DED0F7AF4EEC77AF1EE44
:100FD00010FA80F23A81002320F8023BA38C0133FF
:100FE0001BB2B842A38400F03781E28C9342AABFBF
:100FF000A4F824E05B000023B0F90020CA5236F9BF
:10100000023FA28C06EE903AF8EEE66A238D86EE59
:10101000837A07EE903AF8EEE77AE38C27EE277AA8
:1010200077EE247AFDEEE77A17EE908A424412B208
:10103000A2F1030999FBF3F803FB18980FFA88F85B
:10104000B8F1000FB8BF9844A2F1020931F9188035
:10105000CDED093A06EE908A99FBF3F803FB189858
:101060000FFA88F8B8F1000FB8BF9844F8EEE66AB6
:1010700031F91880CDED026A02F1FF3906EE908A4F
:1010800099FBF3F803FB18980FFA88F8B8F1000FF2
:10109000B8BF9844F8EEE66A31F91880CDED036ADE
:1010A00006EE908A92FBF3F803FB18280FFA88F8F3
:1010B000B8F1000FB8BF9844F8EEE66A31F918802D
:1010C000CDED046A02F1010906EE908A99FBF3F86E
:1010D00003FB18980FFA88F8B8F1000FB8BF9844CE
:1010E000F8EEE66A31F91880CDED056A02F10209E1
:1010F00006EE908A99FBF3F803FB18980FFA88F82C
:10110000B8F1000FB8BF9844F8EEE66A31F91880DC
:10111000CDED066A033206EE908A92FBF3F803FBEC
:10112000182212B2002AB6BF9B1831F9123031F9D9
:1011300013308DED0A5AF8EEE66AF8EEE77A06EE1D
:10114000103ACDED076A77EE677ADDED096A8DED2D
:101150000B4A4FF00008B8EEC66A0023F4EEE67AB8
:10116000C4F2A008C4F2C003F1EE10FACDF830B01A
:10117000CDF834A0CDF838808DED086A0F93FFF6D6
:10118000A3AE9DED0A7AF4EEC77AF1EE10FAB0EE56
:10119000476A3FF69BAE0422002377EEE67A36EEEE
:1011A000C77A0DF10808C7EE876A42444344D2ED7E
:1011B000007A93ED007AF5EEC06AF1EE10FA48BFBE
:1011C000F1EE666A66EEA77A75EE666AE7EE267A53
:1011D00077EEA47AFDEEE77ACDED017ABDF9043021
:1011E000FAE69DED0B7AF4EEC77AF1EE10FAF0EE26
:1011F000475A3FF682AE08220423CEE79DED0C7AD3
:10120000B4EEE77AF1EE10FAB0EE476AFFF68CAE74
:101210000C220823C1E79DED0D7AF4EEC77AF1EEBA
:1012200010FAF0EE475A3FF696AE10220C23B4E7C0
:101230009DED0E7AB4EEE77AF1EE10FAB0EE476A61
:10124000FFF6A0AE14221023A7E718221423A4E768
:1012500000FEFF4600000000664620462946FAF7D9
:101260006BFC284603F0F2FC3EB1304611B0BDE8FD
:10127000F04F03F0EBBC704710B911B0BDE8F08F30
:101280000026EAE76646EFE770B54568D0ED035AF9
:1012900095ED024A95ED036A9FED697A9FED695AD3
:1012A000F2EE084AF9EE087AE4EE247A00F6A44356
:1012B00000F6A846F1EE006A2DED028B66EE266A76
:1012C000BFEE008AF0EE484AE6EE264A0446FDEEFE
:1012D000E77AF6EE008A17EE902AC0F8882CC3ED64
:1012E000004AD5ED037AF4EEE87AF1EE10FAD4BFB5
:1012F000F0EE457AF0EE477AC6ED007A65EEE77AD1
:1013000017EE900A07F07CFB41EC100B0CF004F98F
:1013100051EC100B07F0C8FB07EE100AF7EE007A4D
:1013200077EEC77AB0EE007AC6ED007AD5ED047A92
:10133000A7EE878A04F69C4204F54A6382ED008A90
:1013400083ED008A95ED047AB4EEE87AF1EE10FAB6
:1013500003D5F1EE487AC3ED007ADFED3B6A95EDF7
:10136000056A9FED3A7AD4ED037A9FED398AA6EEAD
:10137000267A04F6984627EE888A17EE100A07F0B8
:101380003FFB41EC100B0CF0C7F851EC100B07F0D1
:101390008BFB07EE900A27EE888AF7EE007A86ED3F
:1013A000008A95ED067A77EE277A04F6D44377EE35
:1013B000877AF5EE006AC3ED007A95ED067AB4EE11
:1013C000E67AF1EE10FA09D5B0EE086AF6EE086A90
:1013D000E7EE466A77EEE67AC3ED007A95ED077A96
:1013E0009FED1C6ADFED1C7ADFED1C6A27EE067AA2
:1013F00004F6844383ED007A95ED097AB6EE006A2F
:1014000037EE467A04F6B84383ED007A95ED0A7A12
:1014100067EE277A04F54C6367EE877A04F6BC41E1
:101420000022C1ED007ABDEC028B1A60D5ED0B7A7B
:1014300067EEA67A04F6C444C4ED007A70BD00BF1E
:1014400000C05A4600409C453D0AC7403D0A27C09F
:10145000560EC9408FC2F53C2DB29D3D6666E63FF3
:101460002DE9F84378292DED028B0546476800F0F9
:101470009C8012D97B2956D06FD97E294CD07F29E8
:1014800045D149F2A823C1F6FF7393F824300374C1
:10149000BDEC028B0120BDE8F883072978D02AD85B
:1014A000012934D107EE902ADFED7D6A9FED7D7A28
:1014B000F8EE677A00F6D84367EEA67AF4EEC77ABC
:1014C000F1EE10FAC3ED007A21DD00F69C4300F541
:1014D0004A65C3ED007AC5ED007AD7ED046AB6EE31
:1014E000007AF4EEC76AF1EE10FA10D5F1EE677AE1
:1014F000C5ED007A0BE0402901D0422907D102F066
:101500004004E4B2C5F88C4C002C00F08380BDECA4
:10151000028B0120BDE8F88301230374BDEC028B2C
:101520000120BDE8F8830021034600F51C62C3F8E2
:10153000D01234339A42FAD105F6C8420021C4F2DF
:101540002031002311602846C5F87C3CFFF79CFE43
:10155000BDEC028B0120BDE8F8837929D7D100F6D4
:10156000984700F5496600F54B6400F6AC4100F67B
:10157000944500234FF07E523B60336023600B6044
:101580002A60FFF781FEBDEC028B0120BDE8F883E5
:1015900002EB820202EB8200C0F3471006F0B0FDBE
:1015A000BDEC028B0120BDE8F88347F2A4000024C3
:1015B000C3F67D702B4605F51C61C3F8D042C3F815
:1015C000D402343399424FF00002F6D105F6C841F7
:1015D0000024C4F220340C60002305F6984005F680
:1015E000944105F5496705F54B6605F6AC44C5F829
:1015F0007C3CC5F88C3C4FF07E5302603A60284634
:10160000326022600B60FFF73FFEBDEC028B0120D1
:10161000BDE8F8832A7C002A3FF479AF2E46B1EE6C
:10162000048A04E0A24206F134067FF770AFD6F8D0
:10163000EC32802B04F10104F4D1D5F88C3C002B62
:10164000F0D1E86880F0004007F0DAF9D7ED017AD0
:1016500067EE887A804617EE900A894607F0D0F93F
:101660000B4641F6B8610246C4F21D014FF0A0409E
:1016700007F066F841EC100B0BF04EFF404653ECC0
:10168000102B494607F060FA41EC100B0BF044FFB9
:1016900051EC100B07F008FAC6F8D4022A7CC1E717
:1016A0002497FF3BCDCC4C3D0068026848F2A5531F
:1016B0001268C0F200039A427FD148F23403C4F2A8
:1016C00004031B685A0565D542F25C43C2F201036C
:1016D0002DE9F0471B6888460BB101221A7042F2CF
:1016E0001449C2F2010942F2154599F8004001344B
:1016F0003F2C88BF4FF0000A42F218474FF42046B3
:1017000094BF5FFA84FA5446C2F20105C2F201079F
:10171000C4F206062B78A3422AD1EFF31383002BE1
:1017200039D1EFF31083002B35D1EFF30582002A76
:1017300040D00F2A05D94EF2F033CEF20003134405
:101740001B78EFF3118212B1934228BF1346402B4E
:1017500021D9B3F5807FDDD142F64903C2F20103FE
:101760001B78002BD6D105F0D9FC2B78A342D4D01E
:1017700042F258434FF42042C2F20103C4F206027F
:1017800007F804800120BC21187089F800A0D170EE
:10179000BDE8F087704733791B06BBD52B78013342
:1017A0003F2B86BF00221346DAB2FB5CDBB2F3713B
:1017B0002A70AFE74FF48073C3E710472DE9F04F6D
:1017C0004BF220022DED028B49F2A823C1F6FF72E5
:1017D000C1F6FF73166893F90970D6F804A083B0B8
:1017E00007440C46002900F0CF81D6F87C5C317CA0
:1017F0008D4280F29881342303FB05630022691C2B
:10180000C6F87C1CC3F8DC22C3F8D822A7F13C0937
:101810004EF64F4309FB09F2C4F6C46383FB023161
:10182000D317C3EBA10303EB430103EB8103D31AEB
:1018300007EE903AF8EEE77AB1EE0A7A06F6BC4186
:1018400006F6B84377EEC77AD3ED006A91ED007AD9
:101850003C2FE7EE276A09DD07EE102A06F54C63F8
:10186000D3ED007AB8EEC77AE7EE876AD6F8883CFF
:10187000B2691A44974240F3FD81726D1A4497424F
:1018800040F32B82D6F890201A44974240F32282EC
:10189000D6F8CC201A44974240F30182D6F80821AA
:1018A0001A44974240F3F881D6F844211A449742EB
:1018B00040F3EF81D6F880211A44974240F3E68145
:1018C000D6F8BC211A44974240F3DD81D6F8F821BE
:1018D0001A44974240F3D481D6F834221A449742EE
:1018E00040F3CB81D6F8702213449F42CCBF4FF017
:1018F00021084FF01E084FEA880B0BEB080306EB9C
:101900008303D6ED037A5B699FEDE68A9FEDE66A75
:10191000FB1A07EE103AB8EEC77A27EE888A77EE00
:10192000267A67EE867A17EE900A07F069F841EC9E
:10193000100B0BF0F1FD342303FB056351EC100B8E
:10194000009307F0B1F807EE900A27EE888A009B13
:10195000BEEEC88A0022302CC3F8C02283EDAF8AC5
:1019600007DD502CD4BF08F1010808F102084FEA46
:10197000880BD84406EB88084FF0340E06F6D442A4
:10198000D8F82030D2ED008AD8F81C00D8F82410FE
:101990000EFB0568013BC8F8C832C8F8C402C8F895
:1019A000CC1218EE900A07F02BF807EE904A9FED44
:1019B000BF7AF8EEE77ACDE9000167EE877AB0EEFC
:1019C000088A17EE900A07F01BF89DED001B41EC0A
:1019D000100B0BF025FEF0EE007A51EC100BA8EE88
:1019E000A78A07F061F807EE900A28EE278A3C2FB5
:1019F00088EDB48A00F31F81DAED046A9FEDAC7ABA
:101A0000DFEDAC5ADFEDAC7A9FEDAC6A96ED038A60
:101A100006F6C84393ED005A66EEA66A403CA6EE71
:101A2000857A06F6CC4306F6DC4106EE904A05EED2
:101A3000107AD3ED004AF8EEE66AB8EEC55AA4EE85
:101A4000A67A342303FB0563E5EE257AC3F8EC722E
:101A500006F68442B4EEE77AF1EE10FA58BFF0EEE3
:101A6000477AF4EEC67AF1EE10FAD4BF67EEA77AA1
:101A7000DFED937A68EE277A0B2FC3EDB87A6CDD31
:101A80006C2F40F32F81D1ED007A92ED007A9FED1B
:101A90008D6A27EE877AF0EE675AE7EE065A4EF621
:101AA00085394FF0A858F0EE006AB0EE657AC4F2BE
:101AB0000109B0EE476A97EEA66A83EDBA7A83ED24
:101AC000B96ADAED007A77EEA77A17EE900A06F097
:101AD00097FF02460B464046494606F031FE41EC70
:101AE000100B0BF019FDF1EE487A53EC102B17EEAA
:101AF000900ACDE9002306F083FFDDE9002307F01B
:101B000023F841EC100B0BF007FD342351EC100BC4
:101B100003FB056606F0C8FFC6F8D40203B0BDECAF
:101B2000028BBDE8F08F002900F0DA800025DFEDA0
:101B3000667A2B46324692EDB47AB4EEE77AF1EE4D
:101B400010FA48BF1D4603F1010348BFF0EE477A83
:101B5000994202F13402EED158E6D1ED007A92EDCD
:101B6000007A9FED5A6A27EE877AF0EE675AE7EE21
:101B7000065A47F6E1294FF02058F0EE006AB0EE21
:101B8000657AC3F6D47994E7327C002AC6D035460C
:101B90004FF0800B04E00134A24205F13405BDDDB5
:101BA000D5F8EC329F42F6D1D6F88C3C1BB1C5F883
:101BB000ECB2327CEFE7F06880F0004006F020FFE6
:101BC000CDE90001384606F009FF47F6E1234FF062
:101BD0008042C3F6847306F0B7FF00230022C4F2EC
:101BE000180306F0AFFD9AED017AF1EE047A67EE84
:101BF000277A804617EE900A894606F001FF0246D2
:101C00000B464046494606F09BFD41EC100B0BF09D
:101C100083FCDDE9000153EC102B06F095FF41EC4D
:101C2000100B0BF079FC51EC100B06F03DFFC5F8E2
:101C3000D402327CAFE7C7F13C0307EE903A9FED48
:101C4000247AF8EEE77A67EE877A17EE900A06F0C4
:101C5000D7FE41EC100B0BF05FFC51EC100B06F0C3
:101C600023FFD8EDB47A07EE100A67EE877AC8ED45
:101C7000B47AC1E64FF000083DE64FF01B083AE6A3
:101C80004FF0180837E64FF0150834E64FF0120809
:101C900031E64FF00F082EE64FF00C082BE64FF020
:101CA000090828E60000FA4620986C3D2497FF3B7F
:101CB00000004842CDCCCC3E00005C4200005243C4
:101CC00000442C47000040420000C642000040C2D1
:101CD0000AD7233C4FF006080DE64FF003080AE64A
:101CE0000D4693E591ED007AD2ED006A07EE909AE9
:101CF00067EE266AF8EEE77AF0EE475AE6EEA75A64
:101D00002B2FB0EE006AF0EE656AD7EE066AC3EDDF
:101D1000BA5AC3EDB96A06DC47F6E1294FF02058FC
:101D2000C3F6D479CDE6384606F058FE4BF651039B
:101D30004FF06042C3F69E7306F006FF00230022B8
:101D4000C3F6F07306F0FCFC80468946B9E600BF96
:101D5000B0F85E306BB190F85D30202B07D8C21818
:101D6000013380F85D30012082F83B107047012379
:101D700003710020704700BF704700BF90F83830F3
:101D800090F839209A4286BF1B18187E4FF0FF301A
:101D9000704700BF90F8383090F839209A4205D942
:101DA0005A1C034480F83820187E70474FF0FF30EB
:101DB000704700BF90F8392090F83800101A70472B
:101DC00049F28860C1F6FF70F9F7E0BF49F2F460AC
:101DD000C1F6FF70F9F7DABF49F63000C1F6FF70BF
:101DE000F9F7D4BF38B50546B0F85E0090B195F864
:101DF0005D301446C3F1210294420CD805F13B003A
:101E00001844224607F0E2FD95F85D30234485F83A
:101E10005D30204638BD012014462871EEE700BF32
:101E2000037B012B024601D90020704700EB8300A1
